:100000000C94A0060C94E6060C94E6060C94E60606
:100010000C94E6060C94E6060C94E6060C94E606B0
:100020000C94E6060C9461180C94E6060C94E60613
:100030000C947A2D0C94E6060C94E6060C94E606D5
:100040000C94E6060C94E6060C94F6160C94E60660
:100050000C94650E0C94E6060C942F0E0C94E60698
:100060000C946D1D0C94E6060C94352C0C94E6064D
:100070000C94526B0C94E6060C943E69981D9D1DE1
:10008000A21DAB1DC21DD91DE91DF91D161E702034
:10009000D91D321F431F721F901FAD1F0720622002
:1000A0004022B9227523EC235524F82403276A271C
:1000B000E4272E287928C62813296D29DA29742ADD
:1000C0006E2B582C8A2C992CC42CF62C062D462DE0
:1000D000462D332D1E2D202D3A2D282D332D232D49
:1000E000252D3A2D282D332D352D372D3A2D3E2D0A
:1000F0000A0D426174743A0020332043656C6C73BE
:1001000020200020342043656C6C73202000204C9C
:100110006F77207761726E696E67206C6576656CAB
:100120003A2025642E2564000A0D47656E657261CC
:1001300074696E672064656661756C74204D6978BA
:100140006572205461626C65000A0D4D69786572B4
:100150002D436F6E6669673A20272573272028256F
:1001600075204D6F746F727329000A0D466F756E9E
:100170006420424C2D4374726C3A200025642000A8
:100180000A0D0A0D2121204D495353494E47204263
:100190004C2D4354524C3A202564202121000A0D55
:1001A0003D3D3D3D3D3D3D3D3D3D3D3D3D3D3D3D7F
:1001B0003D3D3D3D3D3D3D3D3D3D3D3D3D3D3D3D6F
:1001C0003D3D3D000A0D496E69742E204545505253
:1001D0004F4D003A2047656E65726174696E672005
:1001E00044656661756C742D506172616D657465EE
:1001F00072207573696E67206F6C64205374696335
:100200006B2053657474696E6773000A0D466C69E0
:100210006768742D74696D65202575206D696E2081
:1002200020546F74616C3A2575206D696E000A0D5B
:10023000414343206E6F742063616C696272617424
:1002400065642021000A0D5573696E672070617224
:10025000616D65746572736574202564000A0D43D1
:10026000616C6962726174696E6720707265737324
:100270007572652073656E736F722E2E004F4B0A78
:100280000D000A0D436F6E74726F6C3A2000486562
:100290006164696E67486F6C64004E6F726D616C6B
:1002A00020284143432D4D6F646529000A0D3D3DD3
:1002B0003D3D3D3D3D3D3D3D3D3D3D3D3D3D3D3D6E
:1002C0003D3D3D3D3D3D3D3D3D3D3D3D3D3D3D3D5E
:1002D0003D0A0D00416E676C654E69636B202020FE
:1002E00020202020416E676C65526F6C6C202020AE
:1002F000202020204163634E69636B202020202052
:1003000020202020416363526F6C6C20202020202D
:10031000202020205961774779726F2020202020EB
:10032000202020204865696768742056616C7565D7
:10033000202020204163635A2020202020202020DC
:1003400020202020476173202020202020202020F2
:1003500020202020436F6D706173732056616C758F
:1003600065202020566F6C74616765205B302E31EC
:10037000565D20205265636569766572204C65760E
:10038000656C20204779726F20436F6D70617373C5
:10039000202020204D6F746F7220312020202020DB
:1003A000202020204D6F746F7220322020202020CA
:1003B000202020204D6F746F7220332020202020B9
:1003C000202020204D6F746F7220342020202020A8
:1003D000202020202020202020202020202020201D
:1003E000202020202020202020202020202020200D
:1003F00020202020566172696F4D6574657220203F
:10040000202020204D4B334D61672043616C537495
:1004100061746520536572766F2020202020202093
:1004200020202020486F766572676173202020208D
:100430002020202043757272656E74205B302E314F
:10044000415D20204361706163697479205B6D4177
:10045000685D202020202020202020202020202017
:10046000202020202020202020202020202020208C
:10047000202020202020202020202020202020207C
:10048000202020202020202020202020202020206C
:10049000202020204932432D4572726F7220202087
:1004A000202020202020202020202020202020204C
:1004B000202020204750535F4E69636B202020206E
:1004C000202020204750535F526F6C6C202020204A
:1004D0002020202021212120494E434F4D504154BE
:1004E00049424C4520212121002E000A0D20444183
:1004F00043206F7220493243204552524F522120EF
:10050000436865636B204932432C2033567265661D
:100510002C2044414320616E6420424C2D43747270
:100520006C005B25695D005B25695D002B204D69D2
:100530006B726F4B6F70746572202B0048573A5680
:1005400025642E25642053573A25642E256425639F
:100550000053657474696E673A25642025730049F9
:100560003243204552524F52212121004D6973736D
:10057000696E6720424C2D4374726C3A25642121C8
:10058000004865696768743A20202535690053651D
:1005900074706F696E743A253569005072657373B3
:1005A0007572653A253569004F66667365743A2041
:1005B000202535690048656967687420636F6E742B
:1005C000726F6C0044495341424C45440048656990
:1005D00067687420636F6E74726F6C004449534196
:1005E000424C4544006163742E2062656172696EFD
:1005F00067004E69636B3A20202020202025356952
:1006000000526F6C6C3A2020202020202535690094
:10061000436F6D706173733A202020253569004B5C
:10062000313A25346920204B323A25346920004B79
:10063000333A25346920204B343A25346920004B65
:10064000353A25346920204B363A25346920004B51
:10065000373A25346920204B383A25346920004E3A
:10066000693A2534692020526F3A253469200047C1
:10067000733A253469202047693A253469200050AF
:10068000313A253469202050323A2534692000500F
:10069000333A253469202050343A25346920004704
:1006A00079726F202D2053656E736F72004E6963EF
:1006B0006B25346920282533692E25692900526F5E
:1006C0006C6C25346920282533692E25692900475B
:1006D000696572253469202825336929004E6963CC
:1006E0006B2025346920282533692E25782900526E
:1006F0006F6C6C2025346920282533692E257829D4
:100700000059617720202534692028253369290084
:100710004E69636B202534692028253369292825F3
:1007200033692900526F6C6C2025346920282533E9
:1007300069292825336929005961772020253469E2
:10074000202825336929282533692900414343207E
:100750002D2053656E736F72004E69636B202534D4
:100760006920282533692900526F6C6C2025346973
:10077000202825336929005A20202020253469208B
:10078000282533692900566F6C746167653A20200B
:10079000202533692E253169560043757272656EC6
:1007A000743A2020202533692E2531694100506F8D
:1007B0007765723A2020202020253469570044694B
:1007C000736368617267653A202535696D41680019
:1007D00052656365697665720052432D52535349E1
:1007E0003A202020202534690052432D5175616C38
:1007F0006974793A202534690052432D4368616E4B
:100800006E656C733A25346900436F6D7061737364
:100810000048656164696E673A2020253569005695
:10082000616C75653A20202020253569005374617C
:1008300072743A2020202025356900506F74693188
:100840003A202025336900506F7469323A20202500
:10085000336900506F7469333A20202533690050A2
:100860006F7469343A202025336900506F746935FC
:100870003A202025336900506F7469363A202025CC
:10088000336900506F7469373A202025336900506E
:100890006F7469383A202025336900536572766F8A
:1008A000202000536574706F696E742020253369B1
:1008B00000506F736974696F6E3A20253369005276
:1008C000616E67653A2533692D2533690045787473
:1008D00065726E436F6E74726F6C2020004E693AC1
:1008E0002534692020526F3A253469200047733A35
:1008F000253469202047693A253469200048693A3F
:10090000253469202043663A2534692000424C2D65
:100910004374726C204572726F72732000253364C9
:1009200020253364202533642025336420002533BB
:10093000642025336420253364202533642000257A
:10094000336420253364202533642025336420005C
:10095000424C2D4374726C20666F756E64200020CB
:1009600025632020202563202020256320202025AA
:10097000632000202563202020256320202025637C
:10098000202020256320002025632020202D2020EA
:10099000202D2020202D2000313000313100313237
:1009A00000466C696768742D54696D652020005499
:1009B0006F74616C3A2535756D696E004163743AE8
:1009C00020202535756D696E002872657365742960
:1009D000000A0D506C6561736520636F6E6E656310
:1009E00074205370656B7472756D207265636569F0
:1009F00076657220666F722062696E64696E672028
:100A00004E4F572E2E2E006F6B2E0A0D0054696D1F
:100A1000656F75742E0A0D0000008F001E01AD0178
:100A20003B02CA025803E603740402058F051B0645
:100A3000A7063307BE074808D2085B09E3096B0A1B
:100A4000F20A780BFD0B810C040D860D070E870E44
:100A5000060F840F00107B10F5106E11E5115B126C
:100A6000CF124213B31323149214FE146A15D31534
:100A70003B16A11605176717C81727188318DE1825
:100A800037198E19E319361A871AD61A231B6E1BCB
:100A9000B61BFD1B411C831CC31C001D3C1D751D8A
:100AA000AB1DE01D121E421E6F1E9A1EC31EE91EC4
:100AB0000D1F2E1F4D1F691F841F9B1FB01FC31FBB
:100AC000D31FE11FEC1FF51FFB1FFF1F00200301B9
:100AD0000000156500020101D565010302024466AC
:100AE00002000303A1662532692E253169560025CF
:100AF0003033646D20253033642563005374617492
:100B000075730025346920202532693A2530326911
:100B1000002534696D004E69636B20526F6C6C2048
:100B200020596177002534692025346920253469EE
:100B3000002532692E2531695620202533692E255E
:100B40003169410025346957202536696D416800B7
:100B50005361743A25303264004E6F466978003232
:100B600044466978003344466978003F3F466978D7
:100B7000002F4447505300486F6D653A2530336469
:100B80006D20253033642563004E6F204E617669F9
:100B90004374726C21000A0D7777772E4D696B7262
:100BA0006F4B6F707465722E64652028632920482E
:100BB0006953797374656D7320476D6248000A0D3F
:100BC00074686520757365206F662074686973208A
:100BD000736F667477617265206973206F6E6C79CC
:100BE000207065726D6974746564200A0D6F6E20E3
:100BF0006F726967696E616C204D696B726F4B6FC4
:100C0000707465722D48617264776172650041434A
:100C1000542044534C004A65746920736174656CB8
:100C20006C6974005370656B7472756D20736174B8
:100C3000656C6C697420284C6F77207265736F6CDB
:100C40007574696F6E29005370656B7472756D20D1
:100C5000736174656C6C69742028323034382900F3
:100C60005370656B7472756D20736174656C6C691B
:100C700074004D756C74697369676E616C205050B7
:100C80004D000A0D52656365697665723A200075FC
:100C90006E6B6E6F776E2E205573696E67205050A5
:100CA0004D2E2E2E006E6F7420737570706F7274DF
:100CB00065642062792068617264776172652100E1
:100CC0000A0D3D3D3D3D3D3D3D3D3D3D3D3D3D3DB7
:100CD0003D3D3D3D3D3D3D3D3D3D3D3D3D3D3D3D44
:100CE0003D3D3D3D3D000A0D466C69676874436FAC
:100CF0006E74726F6C0A0D48617264776172653A46
:100D000025642E25640A0D536F6674776172653A07
:100D10005625642E2564256320000A0D3D3D3D3D8A
:100D20003D3D3D3D3D3D3D3D3D3D3D3D3D3D3D3DF3
:100D30003D3D3D3D3D3D3D3D3D3D3D3D3D3D3D0020
:100D400011241FBECFEFD0E1DEBFCDBF11E0A0E088
:100D5000B1E0E8E4F6EE02C005900D92A03DB107C7
:100D6000D9F718E0A0EDB1E001C01D92A333B1079F
:100D7000E1F76AEAE2E0F0E081E2809357007491E3
:100D8000AE014F5F5F4F20EF3FEFDA019FE0F901C7
:100D90002F5F3F4F84918D93915097FFF8CF773914
:100DA00011F40000FECFFA019EE081916827609562
:100DB000915097FFFACF8889681721F0773911F49D
:100DC0000000FECF0E9446080C9423730C94000090
:100DD000F999FECF92BD81BDF89A80B59927089503
:100DE000F999FECF1FBA92BD81BD60BD0FB6F894D0
:100DF000FA9AF99A0FBE0895282FFB018150853089
:100E000008F023E0842F9927332721503040829F18
:100E1000B001839F700D929F700D11246C597F4F0C
:100E200028EE36E0AC01CF010E94C0700E945F61E5
:100E30000895282F863010F025E002C0882369F03D
:100E4000F999FECF1FBA82E090E092BD81BD20BD2E
:100E50000FB6F894FA9AF99A0FBE0895FF920F937D
:100E60001F93CF93C82F8B01F42E863010F0C5E06E
:100E700002C0882389F18F2D99272C2F33272150E9
:100E80003040829FF001839FF00D929FF00D11245E
:100E900020EF36E0AC01B801CF018C599F4F0E9482
:100EA000E570F999FECF1FBA82E690E092BD81BD50
:100EB000F0BC0FB6F894FA9AF99A0FBE20EF36E01C
:100EC0004CE050E0B80180E590E00E94E5708C2F86
:100ED0000E9419070E945F61CF911F910F91FF90AF
:100EE0000895CF93F999FECF82E090E092BD81BD45
:100EF000F89A80B5C82F8150853020F0C3E08C2F40
:100F00000E9419078C2F9927CF9108958091C306CD
:100F1000E82FFF27EE0FFF1FEC5AF94F80819181D8
:100F20008D5E9F4F14F010920301808191818A5B46
:100F30009F4FCCF4809103018823A9F481E0809332
:100F40000301809180048F5F80938004853038F0A6
:100F500088EE93E09093FF018093FE0104C066E960
:100F600070E00E947E328091800499279093FA0568
:100F70008093F90508951F93CF93DF93182F88234B
:100F800089F080EF90E09F938F938FE094E19F939F
:100F90008F93E091FF03F091000409950F900F905B
:100FA0000F900F908091E506823308F046C084EFE1
:100FB00091E00E94E117EC01112329F0CE010E947B
:100FC000EA178823D9F38091250190912601209179
:100FD000E5068238910584F433E0239FC001112493
:100FE00080930001112359F168EC70E0832F0E9477
:100FF0007E3288EF90E011C0822F9927880F991FC9
:10100000880F991F809300011123C9F068EC70E0EC
:1010100084E00E947E3283E091E09F938F938FE083
:1010200094E19F938F93E091FF03F0910004099561
:101030000F900F900F900F9002C08093000111232A
:1010400009F1809100016AE00E947672892F992748
:101050009F938F93809100010E94767299279F93AE
:101060008F938EE091E09F938F938FE094E19F9315
:101070008F93E091FF03F091000409958DB79EB71F
:1010800008968DBFDF91CF911F910895CFEFD0E1EA
:10109000DEBFCDBF88249924C0E0C4B9C5B9A7EE8E
:1010A000CA2EA3E0DA2E8EEC9FEFC80ED91ED7FE13
:1010B000FACF189B06C0199B02C08DE007C08BE0D9
:1010C00005C0199B02C084E101C08AE0809302013F
:1010D00081E887B93E9A8FEF88B98BE184B981E0C6
:1010E00085B98EE38AB987E48BB9469A84B7877F3E
:1010F00084BF8091600088618093600010926000DE
:1011000080ED97E09093FF018093FE011092E90239
:101110001092E80210925906109258061092EB02B3
:101120001092EA021092ED021092EC02209102015C
:10113000243128F088E894E0A0E0B0E004C08BE01F
:1011400095E0A0E0B0E08093790190937A01A093BC
:101150007B01B0937C012A3011F0243111F42898DE
:1011600001C0289A0E944A180E941B180E94171456
:101170000E945E2D0E942B1C0E94F42B0E94675D32
:101180000E94A1670E94856A809102018C3010F450
:10119000299A01C0299878944DE063EC76E083E0C9
:1011A0000E94FC06F999FECF88EE93E092BD81BDC6
:1011B000F89A80B5813001F5F999FECF81E090E091
:1011C00092BD81BDF89A80B58F3FB1F028EE36E030
:1011D0004DE450E068EE73E081E094E00E94C0705E
:1011E000EEE0F4E09FE08081349618160CF4CF5FB7
:1011F000915097FFF8CF56C088E291E09F938F936C
:101200008FE094E19F938F93E091FF03F0910004AE
:1012100009950F900F900F900F90E1E0F4E08FE0B0
:10122000158616861786108A8150349687FFF8CF68
:1012300080E480930E0480930F0410921004809336
:1012400011048093120490EC9093130410921404F0
:101250008093150480931604109217049093180439
:101260009093190480931A0410921B0480931C0419
:1012700090931D0481E08093010462E074E08BE0B0
:1012800024E031E0DB01F90101900D928A95E1F74C
:1012900020EF36E04DE450E06150704088EE93E07E
:1012A0000E94E5708C2F99279F938F9382E094E0A2
:1012B0009F938F9389E491E09F938F93FFE0AF2EEC
:1012C000F4E1BF2EBF92AF92E091FF03F0910004D2
:1012D00009958DB79EB708968DBF8AE691E09F93DA
:1012E0008F93BF92AF92E091FF03F09100040995B4
:1012F00010924802109202020E94533E0F900F90EB
:101300000F900F90809102028823E1F3109248021F
:1013100080ED97E00E94E1176C01C0E0D0E0E4E2CC
:10132000EE2EE6E0FE2E8E01109202020E94533E47
:10133000809102028823E1F3F801EF5FFB4F85857E
:101340001816ACF408C0909302020E94533E80919C
:1013500002028823E1F3C6010E94EA17982F88232E
:1013600031F4F801ED5DF94F8181882364F7D701ED
:101370008C9187FF13C02196DF93CF9321978CE741
:1013800091E09F938F93BF92AF92E091FF03F09112
:1013900000040995EDB7FEB73696EDBF21960C5FB8
:1013A0001F4F84E090E0E80EF91ECC30D10508F420
:1013B000BBCFC0E0D0E003E216E07EE0E72E74E0B1
:1013C000F72EF801818187FD1CC0D7018C9118167A
:1013D000C4F42196DF93CF93219780E891E09F9307
:1013E0008F938FE094E19F938F93E091FF03F091AF
:1013F0000004099581E08093FC01EDB7FEB73696B5
:10140000EDBFF801818180788183219684E090E0AE
:10141000E80EF91E080F191FCC30D10590F28EE9A5
:1014200091E09F938F930FE014E11F930F93E0914E
:10143000FF03F091000409950E94533E0F900F9016
:101440000F900F90F999FECF81E090E092BD81BDA1
:10145000F89A80B5823509F417C10E94F42F84EC04
:1014600091E09F938F931F930F93E091FF03F0916F
:1014700000040995C1E00F900F900F900F90C230BB
:1014800039F0C33019F40E949A3104C0C43010F00E
:101490000E94C83080910201843168F085E0809319
:1014A000E206109203078BE18093DE068EE48093C0
:1014B000000780930107F999FECF80E590E092BD87
:1014C00081BDF89A80B58C3008F0C1C0F999FECF83
:1014D00081E590E092BD81BDF89A80B58C3008F02E
:1014E000B6C0F999FECF82E590E092BD81BDF89A31
:1014F00080B58C3008F0ABC0F999FECF83E590E061
:1015000092BD81BDF89A80B58C3008F0A0C0F999E1
:10151000FECF80E590E092BD81BDF89A80B58093C2
:10152000C306F999FECF81E590E092BD81BDF89A9E
:1015300080B58093C406F999FECF82E590E092BD14
:1015400081BDF89A80B58093C506F999FECF83E5F1
:1015500090E092BD81BDF89A80B58093C606F99956
:10156000FECF84E590E092BD81BDF89A80B580936E
:10157000C706F999FECF85E590E092BD81BDF89A46
:1015800080B58093C806F999FECF86E590E092BDBC
:1015900081BDF89A80B58093C906F999FECF87E599
:1015A00090E092BD81BDF89A80B58093CA06F99902
:1015B000FECF88E590E092BD81BDF89A80B58F3F5F
:1015C00009F427C0F999FECF88E590E092BD81BD6E
:1015D000F89A80B58093CB06F999FECF89E590E023
:1015E00092BD81BDF89A80B58093CC06F999FECF63
:1015F0008AE590E092BD81BDF89A80B58093CD06D2
:10160000F999FECF8BE590E092BD81BDF89A80B547
:101610000AC089E08093CB068AE08093CC068BE0F9
:101620008093CD068CE08093CE06C13091F483ED9B
:1016300091E09F938F931F930F93E091FF03F0919D
:10164000000409950F900F900F900F9002C00E9418
:10165000CF2F4CE663EC76E08C2F0E942E07CF5FF5
:10166000C63008F40CCF83E00E941907F999FECF29
:101670001FBA81E090E092BD81BD82E580BD0FB6CA
:10168000F894FA9AF99A0FBEF999FECF8EE090E09D
:1016900092BD81BDF89A80B59927382F2227F999F4
:1016A000FECF8FE090E092BD81BDF89A80B5280F03
:1016B000311D3093D5012093D401F999FECF8AE0F2
:1016C00090E092BD81BDF89A80B59927582F4427A4
:1016D0008FB399279C012270307081FDF9CF8BE088
:1016E00090E092BD81BDF89A80B5480F511D50938E
:1016F000D3014093D2014F5F5F4F39F08091D40105
:101700009091D5018F5F9F4F41F43093D501209385
:10171000D4013093D3012093D2018091D2019091D2
:10172000D3019F938F938091D4019091D5019F9382
:101730008F938BE092E09F938F93CFE0D4E1DF9380
:10174000CF93E091FF03F09100040995EDB7FEB748
:101750003896EDBFF999FECF84E090E092BD81BD4F
:10176000F89A80B5853078F08EE292E09F938F935F
:10177000DF93CF93E091FF03F091000409950F9060
:101780000F900F900F900E9471074CE663EC76E08B
:101790000E94FC060E94710799279F938F9385E40E
:1017A00092E09F938F93CFE0D4E1DF93CF93E091CA
:1017B000FF03F091000409958DB79EB706968DBF83
:1017C0008DE592E09F938F93DF93CF93E091FF039A
:1017D000F0910004099588EE93E00E94E1176C01F6
:1017E0000E94311C0F900F900F900F90C6010E9425
:1017F000EA178823D9F38DE792E09F938F93DF93C5
:10180000CF93E091FF03F091000409950E94EA3B19
:10181000809102010F900F900F900F908A3011F07D
:10182000843111F4289801C0289A80ED97E09093B4
:10183000FF018093FE0185E58093820482E892E0B7
:101840009F938F93DF93CF93E091FF03F091000478
:1018500009958091CF060F900F900F900F90E09117
:10186000FF03F091000482FF07C08EE892E09F938F
:101870008F93DF93CF9308C08AE992E09F938F9371
:101880008FE094E19F938F9309950F900F900F90A5
:101890000F900E94B72188E893E19093A001809374
:1018A0009F0181E0809381040E94BB070E94E4694C
:1018B0008CEA92E09F938F93DF93CF93E091FF03A5
:1018C000F0910004099580ED97E00E94E1176C010A
:1018D0008AEF90E00E94E117EC010F900F900F90BB
:1018E0000F90CE010E94EA17882339F084E690E039
:1018F0000E94E117EC010E94416B80910202882353
:1019000009F499C180911701882309F494C11092B8
:10191000020280918004882319F00E94860702C089
:101920000E94A4400E94533E209102012A3011F0EF
:10193000243111F4289801C0289A8091EF0288235D
:1019400031F08091EF0281508093EF0205C08091C9
:101950006F00806280936F0080919F019091A00141
:1019600001979093A00180939F0180919F01909196
:10197000A001892B21F0809147028823A1F1809159
:101980009F019091A001892BB1F40E940A2C85E05F
:1019900090E09093A00180939F0180910B0690911D
:1019A0000C06019690930C0680930B068091BE0264
:1019B00080688093BE0280911001909111018F5F29
:1019C0009F4F19F58091E5028823F9F080E197E2B5
:1019D0009093FF018093FE0180E890E090931101C5
:1019E0008093100112C02A3011F0243111F428988C
:1019F00001C0289A8091FE019091FF01892B29F462
:101A00008091BE028F778093BE028091020288236C
:101A100021F08091E502882311F40E945B140E945A
:101A2000A310C6010E94EA17882309F400C1E4E16B
:101A3000F0E0CE0EDF1E80910D01882321F0815051
:101A400080930D0125C080938C041092CA021092DD
:101A5000C9021092C8021092C7021092C6021092D8
:101A6000C50280911001909111018F5F9F4F81F409
:101A70008091EF02882361F488E99AE39093FF0153
:101A80008093FE0180E09CE090931101809310010F
:101A90008091D403882339F081508093D4038091BE
:101AA000BE028F7B11C01092D2031092D10310920C
:101AB000D0031092CF038091FE019091FF01892BFA
:101AC00029F48091BE0280648093BE02809100015F
:101AD000282F3327809125019091260182179307A3
:101AE000CCF48091BE0280628093BE02809110018E
:101AF000909111018F5F9F4FC1F480E797E1909320
:101B0000FF018093FE0180E093E0909311018093A8
:101B100010010BC08091FE019091FF01892B29F4E7
:101B20008091BE028F7D8093BE020E94936084E00C
:101B30008093FD018091E502882329F44AEA842EEE
:101B400045E0942E12C08091D6018F5F8093D6011C
:101B5000813359F41092D6018091D0019091D10136
:101B600001969093D1018093D0010894811C911C1F
:101B700042E784164BE0940609F059C08824992462
:101B80008091D4019091D50101969093D5018093D5
:101B9000D4012091D2013091D3012F5F3F4F309378
:101BA000D3012093D201892F9927282FF999FECFAD
:101BB0001FBA8EE090E092BD81BD20BD0FB6F894B3
:101BC000FA9AF99A0FBE2091D401F999FECF1FBA63
:101BD0008FE090E092BD81BD20BD0FB6F894FA9AD7
:101BE000F99A0FBE2091D2013091D3014091D301D7
:101BF000F999FECF1FBA8AE090E092BD81BD40BD49
:101C00000FB6F894FA9AF99A0FBEF999FECF1FBA57
:101C10008BE090E092BD81BD20BD0FB6F894FA9A9A
:101C2000F99A0FBE84E190E00E94E1176C010E94D6
:101C30006E610E94B6678091FD01882309F051CE44
:101C40000E94D4604ECEF999FECF1FBA92BD81BDDD
:101C500060BD0FB6F894FA9AF99A0FBE08951F92D4
:101C60000F920FB60F9211248F939F93EF93FF93D0
:101C700080910F018823E1F48091F0019091F101AE
:101C800001969093F1018093F001FC01EF5CFA4F13
:101C9000E081ED3019F0803A910539F41092F101AC
:101CA0001092F00181E080930F01E093C60004C020
:101CB0001092F1011092F001FF91EF919F918F919D
:101CC0000F900FBE0F901F9018951F920F920FB696
:101CD0000F9211242F933F934F935F936F937F93B2
:101CE0008F939F93AF93BF93CF93EF93FF9390E026
:101CF0008091C6008093E8015091F601503A10F0AF
:101D00009093F7018091E8018D3009F065C08091D2
:101D1000F701823009F060C09093F701852F992771
:101D200081579B4FFC01329740812091F201309105
:101D3000F301241B3109DC0111978C91281B310917
:101D4000C9019F709093F3018093F20146E096954C
:101D500087954A95E1F7982F935C9093F4012F7340
:101D60003070235C2093F5018081981729F48C91C1
:101D7000281711F491E006C090E08091E5018F5F93
:101D80008093E501C091E701CC2309F074C0992349
:101D900009F471C081E08093E701580F5093E4018A
:101DA0005150E52FFF27E157FB4F8DE08083809155
:101DB0009104823509F05FC00E94B72188E190E06C
:101DC0002CE00FB6F894A895809360000FBE209386
:101DD0006000C093FC014FC02091F701822F99272A
:101DE00081309105F9F0823091051CF4892B21F0A6
:101DF00040C0029711F13DC08091E801833239F46F
:101E00008091E701882319F481E08093F7018091A4
:101E1000E80180938F0481E08093F6018091E801CE
:101E2000992722C02F5F2093F701E52FFF27E15765
:101E3000FB4F8091E801808309C0E52FFF27E15720
:101E4000FB4F8091E8018083503A20F45F5F50930C
:101E5000F60102C01092F7012091E8018091F20191
:101E60009091F301820F911D9093F3018093F20101
:101E700002C01092F701FF91EF91CF91BF91AF9106
:101E80009F918F917F916F915F914F913F912F9192
:101E90000F900FBE0F901F901895AC01A0E0B0E01E
:101EA0009D01A817B90748F4E1E3F5E08191280FF7
:101EB000311D1196A417B507C8F33F70FD01EF5C03
:101EC000FA4FC90156E0969587955A95E1F7835CDC
:101ED00080831196FD01EF5CFA4F2F733070822FD3
:101EE000835C8083AE5CBA4F8DE08C9310920F01BF
:101EF000809131058093C6000895A0E0B0E0E3E84A
:101F0000FFE00C94EF722C859D850E85BB2483E247
:101F1000809331059F59909332052093330533E028
:101F2000E32EF12C002309F49EC0CF84D888BE0193
:101F30006D5E7F4FA989BA890150109709F493C04B
:101F40001097B9F0F601EB0DF11DB3949081119744
:101F500091F4002349F1FB016E5F7F4FDB01C080EC
:101F6000D1806E5F7F4F0D90BC91A02DBB2401509E
:101F700002C090E019C01097B9F0F601EB0DF11D09
:101F8000B3944081119791F4002341F1FB016E5FFE
:101F90007F4FDB01C080D1806E5F7F4F0D90BC9181
:101FA000A02DBB24015002C040E018C01097B1F032
:101FB000F601EB0DF11DB3941081119781F400230C
:101FC00071F0FB013296DB01CD90DC90BF016E5FBA
:101FD0007F4FA081B181BB24015001C010E0F70107
:101FE000EF5CFA4F892F86958695835C80830894F1
:101FF000E11CF11CF701EF5CFA4F892F99278370E0
:10200000907024E0880F991F2A95E1F755279A01CF
:1020100094E0369527959A95E1F7822B835C80832F
:102020000894E11CF11CF701EF5CFA4F4F705070FF
:10203000440F551F440F551F812F992726E0969571
:1020400087952A95E1F7842B835C80830894E11CB3
:10205000F11CF701EF5CFA4F1F73135C10830894B7
:10206000E11CF11C6ACFC7010E944D0FE9E00C94FE
:102070000B73A3E07A2F4091E4014650442309F406
:1020800058C0E72FFF27E157FB4F80818D537F5FBB
:10209000E72FFF27E157FB4F20812D537F5FE72F6D
:1020A000FF27E157FB4F30813D537F5FE72FFF272D
:1020B000E157FB4F60816D537F5F9927880F991F10
:1020C000880F991F522F52955F70582B822F992796
:1020D0008F709070F4E0880F991FFA95E1F7232F25
:1020E00026952695282B832F992783709070E6E0FC
:1020F000880F991FEA95E1F7682B41504F3FC9F0CF
:10210000EA2FFF27E157FB4F5083AF5F41504F3F0E
:1021100081F0EA2FFF27E157FB4F2083AF5F41504B
:102120004F3F39F0EA2FFF27E157FB4F6083AF5F46
:10213000A5CF82E994E09093E3018093E201A3505C
:10214000A093E1010895A2E0B0E0E9EAF0E10C9487
:10215000F5728091E701882309F45DC30E9439106C
:1021600080919004823609F01FC2809191049927D2
:102170008037910509F4ACC081379105A4F4863607
:10218000910509F470C18736910524F48B349105CB
:10219000F1F00AC28D36910509F468C08E369105BA
:1021A00009F453C001C28337910509F4EDC08437A7
:1021B00091052CF48137910509F491C0F5C184375C
:1021C000910511F18937910509F48AC1EDC1E091BA
:1021D000E201F091E3018081918190930203809369
:1021E00001032091FF0230910003821B930B845E58
:1021F0009D4F68E671E00E949672845B90409093D8
:10220000FE028093FD02D0C18091E401A091E20121
:10221000B091E301853140F080E1EAE6F4E00D9011
:1022200001928A95E1F70DC08D919D910D90BC9121
:10223000A02D80936A0490936B04A0936C04B093D8
:102240006D0480EF8093DF0146C080910F018823E9
:10225000E1F38DE490E09F938F9381E094E09F936E
:102260008F9381E08F938F938EE42AC080910F012A
:102270008823E1F3A091E201B091E3011C911130B8
:1022800091F461E074E08DE4FB010D9001928A9578
:10229000E1F723E23EE04DE450E088EE93E00E9457
:1022A000E570198301C0198281E090E09F938F93BC
:1022B000CE0101969F938F9381E08F938F938DE44E
:1022C0008F930E947D0F8DB79EB707968DBF6CC10F
:1022D00081E08093EA018FEF80930D0165C1E09169
:1022E000E201F091E30180818F3F39F40E94710790
:1022F000E091E201F091E3018083E091E201F0914D
:10230000E3018081882311F481E003C0863010F05E
:1023100085E08083E091E201F091E3014CE663EC1B
:1023200076E080810E94FC0680910F018823E1F312
:10233000E091E201F091E3018081898382E58A8363
:102340008CE690E09F938F9383EC96E09F938F931E
:1023500021E030E03F932F93CE0102969F938F931D
:102360003F932F93CE01820F931F9F938F9383E010
:102370008F9381E08F9381E58F930E947D0FADB79E
:10238000BEB71F96ADBF10C12091E2013091E301AD
:10239000F90180818150853008F04CC081818235FF
:1023A00009F048C063EC76E08CE62E5F3F4FDB011E
:1023B000F901982F01900D929A95E1F72250304043
:1023C000482FD9018C910E942E07809100079927F0
:1023D000AA27BB27BC01CD0124EC39E040E050E046
:1023E0000E945772DC01CB018093990190939A016E
:1023F000A0939B01B0939C01809101079927AA2784
:10240000BB27BC01CD010E945772DC01CB01809338
:10241000950190939601A0939701B0939801E09154
:10242000E201F091E30180810E9419070E94710787
:10243000898301C0198280910F018823E1F381E033
:1024400090E09F938F93CE0101969F938F9381E0AD
:102450008F938F9383E58F930E947D0FEDB7FEB727
:102460003796EDBF2EC0E091E201F091E301E081EB
:102470008E2F8150853018F48E2F0E941907E0911D
:10248000E201F091E301808189834CE663EC76E020
:102490000E94FC0680910F018823E1F381E090E027
:1024A0009F938F93CE0101969F938F9381E08F939B
:1024B0008F9386E48F930E947D0F8DB79EB707960A
:1024C0008DBF8091E502882329F46EE670E0898152
:1024D0000E947E3280E00E94BB070E94E46964C0D3
:1024E000E091E201F091E3018081992787FD9095C9
:1024F00090936F0680936E068181992787FD909552
:1025000090937106809370068281992787FD90953C
:1025100090937306809372068381992787FD909527
:1025200090937506809374068481992787FD909512
:1025300090937706809376068581992787FD9095FD
:1025400090937906809378068681992787FD9095E8
:1025500090937B0680937A068781992787FD9095D3
:1025600090937D0680937C068085992787FD9095C2
:1025700090937F0680937E068185992787FD9095AD
:1025800090938106809380068285992787FD909598
:1025900090938306809382068385992787FD909583
:1025A00090938506809384068091910499278436C0
:1025B000910509F4C5C085369105ACF481369105C5
:1025C00009F479C0823691052CF48B34910509F415
:1025D00055C019C18236910509F47AC08336910538
:1025E00009F489C010C18C36910509F4F7C08D3605
:1025F00091054CF48736910509F402C1883691059E
:1026000009F4BCC000C18437910529F086379105D3
:1026100009F4F2C0F8C08091E401A091E201B09108
:10262000E301853140F080E1EAE6F4E00D900192AB
:102630008A95E1F70DC08D919D910D90BC91A02DD3
:1026400080936A0490936B04A0936C04B0936D0420
:1026500080910F018823E1F31F9280910C018F93E9
:1026600084E58F930E947D0F8AEF8093DF018FEFC7
:1026700080930D010F900F900F90C5C0E091E20183
:10268000F091E30180819181909302038093010393
:102690002091FF0230910003821B930B845E9D4FBB
:1026A00068E671E00E949672845B90409093FE020F
:1026B0008093FD02A8C0E091E201F091E3018081E6
:1026C00080930E01803298F08FE180930E010FC04D
:1026D000A091E201B091E3018BE0E2E8F4E00D901B
:1026E00001928A95E1F780918B04809313068FEF16
:1026F00080930D0188C08091DB019091DC01892BD2
:1027000089F4E091E201F091E301E081EE2351F0E0
:102710008AE0E89FC00111240E94E11790935D04B4
:1027200080935C04E091E201F091E30190818AE002
:10273000989FC00111249093DC018093DB0115C0A8
:102740008FEF80930D01E091E201F091E301908120
:102750008AE0989FC00111249093DE018093DD01EF
:10276000892B19F081E08093EC0180EA9FE00E94C0
:10277000E1179093D8018093D70145C08FEF8093E4
:102780000D01E091E201F091E301908197FD08C015
:1027900082E08093E9011092DA011092D9011AC007
:1027A000909580914202892B8093420291818AE028
:1027B000989FC00111249093DA018093D90184E09D
:1027C0008093E90180EA9FE00E94E1179093D8018D
:1027D0008093D70181E08093ED0115C08FEF809346
:1027E0000D01E091E201F091E301808180934302C9
:1027F00081E08093EE0107C081E08093EB0103C08C
:1028000081E08093EF011092E7011092E3011092B2
:10281000E2011092E101E3E0CE5F0C941173982F76
:102820008091C00085FFFCCF9093C60008950F9360
:102830001F9388E18093C1008091C00082608093E3
:10284000C0008091C10080688093C1008091C10068
:1028500080648093C10000E010E00093C5008AE22C
:1028600090E08093C4008091DD019091DE010E9490
:10287000E11790935F0480935E048CED90E00E94DA
:10288000E11790938E0480938D04109260048EE47F
:102890008093610483E0809364048BE080936204FE
:1028A000109263041093E3010093E2011092E1019E
:1028B0001F910F910895A0E1B0E0E1E6F4E10C94DE
:1028C000F27280910F01882309F48CC28091D701A4
:1028D0009091D8010E94EA17882361F01092DA01E2
:1028E0001092D9011092DE011092DD011092DC01EC
:1028F0001092DB018091D9019091DA01892B41F08E
:1029000080912F05909130050E94EA17882329F4C1
:102910008091ED01882309F460C080910F01882324
:1029200009F45BC08091E90108E211E08430A8F06D
:102930000E94CB2180E590E09F938F931F930F938C
:1029400081E08F938F9388E48F930E947D0F2DB742
:102950003EB7295F3F4F2DBF34C01092440284ED33
:1029600094E09F938F9380EC91E29F938F93E091FB
:10297000FF03F0910004099584E190E09F938F9309
:102980001F930F9381E090E09F938F9389EE91E0E6
:102990009F938F9382E08F9381E08F9388E48F934E
:1029A0000E947D0F8091E901982F8F5F8093E9014C
:1029B0002DB73EB7215F3F4F2DBF943010F01092DE
:1029C000E9018091D9019091DA010E94E117909379
:1029D000300580932F051092ED018091EE01882340
:1029E00051F180910F01882331F10E94CB2180E5C4
:1029F00090E09F938F9388E291E09F938F9321E0E3
:102A000030E03F932F9387E291E09F938F933F9322
:102A10002F9383E492E09F938F9383E08F9381E0E1
:102A20008F938CE48F930E947D0F1092EE018DB7EF
:102A30009EB70F968DBF8091EB018823D1F08091D6
:102A40000F018823B1F08AE090E09F938F9380E696
:102A500094E09F938F9381E08F938F9386E58F937C
:102A60000E947D0F1092EB012DB73EB7295F3F4FBB
:102A70002DBF8091EF018823D9F080910F01882329
:102A8000B9F08BE090E09F938F9382E894E09F935E
:102A90008F9381E08F9380910C018F9387E48F93C4
:102AA0000E947D0F1092EF018DB79EB707968DBFE4
:102AB00080918D0490918E040E94EA17882309F476
:102AC00061C080910F01882309F45CC08091DE060B
:102AD0009927880F991F880F991F7C010027F7FC01
:102AE0000095102F80913B0390913C03A0913D03F2
:102AF000B0913E03BC01CD01A80197010E94CB72A9
:102B000030937B0420937A048091330390913403B3
:102B1000A0913503B0913603BC01CD01A801970106
:102B20000E94CB7230937D0420937C048091D2026A
:102B300080937E048091D10280937F0488E090E0AE
:102B40009F938F938AE794E09F938F9381E08F9375
:102B500083E08F9387E78F930E947D0F809180049D
:102B60002DB73EB7295F3F4F2DBF853018F086E067
:102B70008093800483E690E00E94E11790938E0496
:102B800080938D048091DD019091DE01892B41F0CD
:102B900080915E0490915F040E94EA17882321F4DB
:102BA0008091EC01882329F180910F01882309F19C
:102BB00082E490E09F938F9381ED95E09F938F93B4
:102BC00081E08F938F9384E48F930E947D0F109206
:102BD000EC018DB79EB707968DBF8091DD01909176
:102BE000DE01009731F00E94E11790935F0480931B
:102BF0005E048091DB019091DC01892B09F485C092
:102C000080915C0490915D040E94EA17882309F486
:102C10007CC080910F01882309F477C08091DE0683
:102C20009927880F991F880F991F7C010027F7FCAF
:102C30000095102F80913B0390913C03A0913D03A0
:102C4000B0913E03BC01CD01A80197010E94CB7257
:102C500030934F0420934E048091330390913403BA
:102C6000A0913503B0913603BC01CD01A8019701B5
:102C70000E94CB72309351042093500420918A0714
:102C800030918B0740918C0750918D07DA01C90173
:102C900003E0880F991FAA1FBB1F0A95D1F7820F67
:102CA000931FA41FB51F820F931FA41FB51F209150
:102CB000790130917A0140917B0150917C01BC01F6
:102CC000CD010E94CB7230935304209352048EE0C6
:102CD00090E09F938F938EE494E09F938F9381E095
:102CE0008F938F9383E48F930E947D0F8091DB01FC
:102CF0009091DC010E94E11790935D0480935C0445
:102D00002DB73EB7295F3F4F2DBF80910E018F3FFA
:102D100071F1992714E0880F991F1A95E1F78C52E9
:102D20009D4F40E150E0BC01CE0101960E94AA7087
:102D300080E190E09F938F93CE0101969F938F93B4
:102D400081E090E09F938F938EE091E09F938F932B
:102D500082E08F9381E08F9381E48F930E947D0FB7
:102D60008FEF80930E018DB79EB70B968DBF80912C
:102D700013068823D1F080910F018823B1F081E000
:102D800090E09F938F9383E196E09F938F9381E0F0
:102D90008F938F9382E48F930E947D0F109213067E
:102DA0002DB73EB7295F3F4F2DBF8091EA018823A1
:102DB000C9F080910F018823A9F084E390E09F93EC
:102DC0008F9384E596E09F938F9381E08F938F9309
:102DD00080E58F930E947D0F1092EA018DB79EB718
:102DE00007968DBFE6E0C05F0C940E731F920F92A2
:102DF0000FB60F9211242F933F935F936F937F939E
:102E00008F939F93AF93BF93EF93FF938091FD01B7
:102E1000882329F08091FD0181508093FD018091EC
:102E2000E203882319F081508093E2038091050228
:102E30008150809305028F3FB9F489E080930502A9
:102E4000809112018F5F817080931201882319F4A1
:102E500081E0809302028091030290910402019626
:102E600090930402809303028091FE019091FF01F0
:102E7000892BC9F08091FE019091FF0101979093F9
:102E8000FF018093FE018091FE019091FF0120914E
:102E900010013091110182239323892B11F021E03D
:102EA00009C020E007C020E08FEF9FEF9093110151
:102EB0008093100180910201222331F08A3011F4B5
:102EC0005A9A07C0479A05C08A3011F45A9801C02F
:102ED00047988091D403882309F063C08091CF067E
:102EE00083FF5FC086B19927FC01E071F07084FF19
:102EF0000AC0809100029091010201969093010214
:102F0000809300024EC08091000290910102892BB3
:102F100009F443C080910002909101028A569140C9
:102F2000E0F5809100029091010269E270E00E9458
:102F300082728091000290910102860F971F9093F8
:102F400001028093000280910002909101020B9790
:102F500050F080910002909101020A979093020331
:102F60008093010304C0F0930203E0930103809176
:102F70000103909102032091FF0230910003821B14
:102F8000930B845E9D4F68E671E00E949672845BAD
:102F900090409093FE028093FD02109201021092E5
:102FA0000002FF91EF91BF91AF919F918F917F911F
:102FB0006F915F913F912F910F900FBE0F901F90D7
:102FC00018952091030230910402280F391FC9017E
:102FD000019608952091030230910402821B930B05
:102FE000892F99278695807490700895CF93DF93E9
:102FF0000E94E117EC01CE010E94EA178823D9F361
:10300000DF91CF910895CF93DF930E94E117EC01F8
:1030100009C080911701882329F0909317018FEC44
:1030200080937A00CE010E94EA17982F882389F3B3
:10303000DF91CF9108959FB7F8945F983E9A469A92
:103040008091B0008F708093B0008091B000836059
:103050008093B0008091B1008B738093B100809118
:10306000B1008B608093B1001092B2008FEF80931B
:10307000B3008091B00080688093B00080917000B0
:103080008A7F8093700080917000826080937000CE
:103090009FBF08958AE090E00E94E11790930D028F
:1030A00080930C0282E085BD83EA84BD17BC88E76B
:1030B00088BD86E086BD80916E00816080936E0041
:1030C00008951F920F920FB60F9211242F933F93E2
:1030D0004F935F936F937F938F939F93AF93BF9320
:1030E000CF93DF93EF93FF938091020190910602BB
:1030F000843108F011C1992309F066C38091B000B2
:1031000086FFECC08091B0008F7B8093B00089EA8D
:1031100093E09093080280930702809113019091AD
:1031200014019C01220F331F280F391F8091850144
:103130009927880F991F880F991F280F391F37FF6C
:1031400002C02D5F3F4FC90195958795959587954D
:1031500090931401809313019093FB018093FA01E3
:10316000809121076091EF0620913B0330913C0351
:1031700040913D0350913E0380FF2CC07727882764
:103180009927EA01D90157FF04C0A158BF4FCF4F7B
:10319000DF4FE7E0D595C795B795A795EA95D1F7A5
:1031A0009D01AE010E9457729B01AC0197FF04C0C4
:1031B000215C3F4F4F4F5F4F66E0559547953795E0
:1031C00027956A95D1F78091FA019091FB01820FC2
:1031D000931F2BC0772788279927EA01D90157FF2A
:1031E00004C0A158BF4FCF4FDF4F27E0D595C795FB
:1031F000B795A7952A95D1F79D01AE010E94577208
:103200009B01AC0197FF04C0215C3F4F4F4F5F4FC4
:10321000F6E05595479537952795FA95D1F7809122
:10322000FA019091FB01821B930B9093FB01809319
:10323000FA018091F006282F3327220F331F220F27
:10324000331F8091FA019091FB01821793077CF064
:103250008091F106282F3327220F331F220F331FAF
:103260008091FA019091FB012817390724F43093DB
:10327000FB012093FA01209107023091080280910E
:10328000FA019091FB01280F391F205032403093F2
:103290000802209307028091FA019091FB0197FDAB
:1032A000039695958795959587959093FB018093C7
:1032B000FA0145E02D3D340718F08CED95E005C08E
:1032C0002757314030F487E791E0909308028093CC
:1032D0000702809107029091080243C28091B000DA
:1032E00080648093B0008091F606282F33278DEDFF
:1032F00096E0289FA001299F500D389F500D112462
:10330000CA012091090230910A02821B930B90930B
:1033100008028093070255C2992309F055C2809193
:10332000B00086FF23C28091B0008F7B8093B000F5
:10333000E0910B02EE23F1F48091F606282F33275B
:103340008DED96E0289FA001299F500D389F500DCC
:103350001124CA012091090230910A02821B930BA9
:10336000909308028093070210920A0210920902B9
:10337000469A27C289EA93E0909308028093070255
:103380008E2F99278330910509F4A4C184309105CB
:103390003CF48130910561F0029709F4D2C0AAC1D2
:1033A0008430910509F499C1059709F4A0C1A2C11F
:1033B00080911301909114019C01220F331F280F5B
:1033C000391F809185019927880F991F880F991FB0
:1033D000280F391F37FF02C02D5F3F4FC901959558
:1033E00087959595879590931401809313019093F9
:1033F000FB018093FA01809121076091EF062091F3
:103400003B0330913C0340913D0350913E0380FFCC
:103410002CC0772788279927EA01D90157FF04C0D4
:10342000A158BF4FCF4FDF4F27E0D595C795B79530
:10343000A7952A95D1F79D01AE010E9457729B0175
:10344000AC0197FF04C0215C3F4F4F4F5F4FA6E098
:103450005595479537952795AA95D1F78091FA010B
:103460009091FB01820F931F27C077278827992708
:1034700057FF04C021583F4F4F4F5F4FF7E055951E
:10348000479537952795FA95D1F70E9457729B017A
:10349000AC0197FF04C0215C3F4F4F4F5F4FE6E008
:1034A0005595479537952795EA95D1F78091FA017B
:1034B0009091FB01821B930B9093FB018093FA0187
:1034C0008091F006282F3327220F331F220F331F3E
:1034D0008091FA019091FB01821793077CF0809113
:1034E000F106282F3327220F331F220F331F80911D
:1034F000FA019091FB012817390724F43093FB015E
:103500002093FA0180910702909108022091FA011C
:103510003091FB01820F931F8050924090930802DC
:10352000809307028091FA019091FB0197FD039629
:1035300095958795959587959093FB018093FA01D2
:10354000ECC080911501909116019C01220F331F50
:10355000280F391F809184019927880F991F880FA0
:10356000991F280F391F37FF02C02D5F3F4FC90138
:10357000959587959595879590931601809315015C
:103580009093F9018093F801809121076091F306EF
:10359000A0913303B0913403C0913503D091360329
:1035A00081FF2AC07727882799279D01AE01D7FF81
:1035B00004C021583F4F4F4F5F4FA7E055954795A7
:1035C00037952795AA95D1F70E9457729B01AC01B8
:1035D00097FF04C0215C3F4F4F4F5F4FF6E055957A
:1035E000479537952795FA95D1F78091F8019091F5
:1035F000F901820F931F29C07727882799279D01FA
:10360000AE01D7FF04C021583F4F4F4F5F4FE7E057
:103610005595479537952795EA95D1F70E945772AA
:103620009B01AC0197FF04C0215C3F4F4F4F5F4FA0
:1036300076E055954795379527957A95D1F78091FE
:10364000F8019091F901821B930B9093F9018093FB
:10365000F8018091F406282F3327220F331F220F01
:10366000331F8091F8019091F901821793077CF044
:103670008091F506282F3327220F331F220F331F87
:103680008091F8019091F9012817390724F43093BB
:10369000F9012093F801809107029091080220918E
:1036A000F8013091F901820F931F8050924090935E
:1036B0000802809307028091F8019091F90197FD2B
:1036C000039695958795959587959093F9018093A5
:1036D000F80123C08091560702C08091C206992745
:1036E000880F991F880F991F87559E4F12C0809190
:1036F0006007F5CFFF27EE0FFF1FEC5AF94F20812F
:103700003181220F331F8091070290910802820FAE
:10371000931F909308028093070280910702909173
:10372000080255E08D3D950718F08CED95E005C039
:103730008757914030F487E791E090930802809397
:10374000070220910702309108022C5B3040309331
:103750000802209307028091090290910A02820FC9
:10376000931F90930A02809309022BC08091B000AE
:1037700080648093B0008CEB90E09093080280937B
:1037800007028091090290910A0284549F4F9093FE
:103790000A02809309028091FC01882331F0809114
:1037A000EF02853B10F0469801C0469A80910B02CB
:1037B0008F5F80930B029091F606981710F4109289
:1037C0000B0281E0809306022091070230910802EB
:1037D00041E02F37340730F08FEF8093B3002F5F35
:1037E00030400FC02F3F3105C9F0C0F0A9014F5F35
:1037F00050404F37510550F480E88093B300205873
:103800003040309308022093070212C08FEF80935C
:10381000B30050930802409307020AC08091070248
:103820008093B300109208021092070210920602D1
:10383000FF91EF91DF91CF91BF91AF919F918F91C8
:103840007F916F915F914F913F912F910F900FBE9C
:103850000F901F90189510927C008FEC80937A0047
:1038600008950F931F93CF93DF938FB399278C0104
:103870000270107081FDF9CF83E090E092BD81BDB0
:10388000F89A80B5C82FDD27C531D10508F02A97F1
:10389000C7BD1092150284E690E00E940318809143
:1038A0001B0190911C018052934008F4E801CA3F2B
:1038B000D105F8F4C7BD82E390E00E94031889EEB9
:1038C00094E09F938F938FE094E19F938F93E09187
:1038D000FF03F0910004099580911B0190911C0158
:1038E0000F900F900F900F908052934010F0219600
:1038F000DECF2C2FF999FECF1FBA83E090E092BD66
:1039000081BD20BD0FB6F894FA9AF99A0FBEC09304
:1039100020068CE291E00E940318DF91CF911F9165
:103920000F910895EF92FF921F93CF93C0E0C09341
:103930001002C0930F02C0930E0280ED97E00E9428
:10394000E1177C011CE8C33019F41B3008F019E0C2
:10395000C0E080912502909126028C5F934024F470
:1039600080911A0181500AC080912502909126020F
:103970008750944034F080911A018F5F80931A0130
:1039800001C0C1E080912302909124028C5F93409A
:1039900024F48091190181500AC0809123029091F2
:1039A00024028750944034F0809119018F5F8093F6
:1039B000190101C0CF5F80912102909122028C5F9A
:1039C000934024F48091180181500AC08091210213
:1039D0009091220287509440C4F0809118018F5F2B
:1039E0008093180113C08BEE94E09F938F938FE028
:1039F00094E19F938F93E091FF03F0910004099568
:103A00000F900F900F900F904DC0CF5F88E0809384
:103A10004A020E94FA2B80911A018A3030F481E028
:103A2000809310028AE080931A0180911A01863FE8
:103A300030F081E08093100285EF80931A0180912D
:103A400019018A3030F481E080930F028AE080937C
:103A5000190180911901863F30F081E080930F02B7
:103A600085EF80931901809118018A3030F481E04C
:103A700080930E028AE08093180180911801863F9E
:103A800030F081E080930E0285EF809318018091E1
:103A90004A02882339F0C7010E94EA17882309F0F7
:103AA000A2CFF5CF109217018FEC80937A0080910E
:103AB00017018823E1F31A3020F48AE090E00E9495
:103AC0000318115009F03FCF86E490E00E940318DC
:103AD000CF911F91FF90EF9008951F920F920FB614
:103AE0000F921124AF92BF92CF92DF92EF92FF928A
:103AF0000F931F932F933F934F935F936F937F93F6
:103B00008F939F93AF93BF93EF93FF9380912E0278
:103B1000282F3327442755278F5F80932E02F901E2
:103B20002231310508F0FAC3E25CFF4F0C941D739B
:103B3000809178009091790046C0809178009091B2
:103B400079009AC180917800909179009093300229
:103B500080932F02C5C18091470390914803209123
:103B6000780030917900821B930B90931506809317
:103B70001406809114069091150690933A02809352
:103B80003902CCC18091780090917900209149034D
:103B900030914A03821B930B90931F0680931E065D
:103BA00080911E0690911F0690933C0280933B02E9
:103BB000B7C3809133029091340220917800309104
:103BC0007900820F931F909334028093330281E037
:103BD000A8C38091310290913202209178003091F7
:103BE0007900820F931F909332028093310284E018
:103BF00098C380912501909126019C01220F331FCB
:103C0000280F391F809178009091790063E070E06F
:103C10000E948272260F371F369527953695279575
:103C2000309326012093250185E07BC380917800A5
:103C300090917900AA2797FDA095BA2FBC01CD01DC
:103C40000E94A3717B018C018091410390914203FA
:103C5000A0914303B09144039C01AD01C801B70199
:103C60000E940771DC01CB01BC01CD010E94707183
:103C7000DC01CB0190931C0280931B0280911B02FC
:103C800090911C0202970CF446C0809141039091E0
:103C90004203A0914303B091440320E030E84BE39A
:103CA00054E4BC01CD010E946C7188230CF088C0E3
:103CB0008091410390914203A0914303B09144034A
:103CC0002AE037ED43EA5CE3BC01CD010E940871B4
:103CD000DC01CB018093410390934203A093430303
:103CE000B09344038091BF029091C002845F9140E1
:103CF00008F066C08091410390914203A091430374
:103D0000B09144032DEC3CEC4CEC5DE3BC01CD01E7
:103D10000E9408714BC080911B0290911C028F5F22
:103D20009F4F0CF04DC08091410390914203A091B0
:103D30004303B091440320E030E849E054E4BC017F
:103D4000CD010E9453721816DCF5809141039091C9
:103D50004203A0914303B09144032AE037ED43EAC4
:103D60005CE3BC01CD010E940771DC01CB018093B3
:103D7000410390934203A0934303B0934403809183
:103D8000BF029091C002845F9140D0F480914103C2
:103D900090914203A0914303B09144032DEC3CEC7D
:103DA0004CEC5DE3BC01CD010E940771DC01CB014D
:103DB0008093410390934203A0934303B093440341
:103DC00081E080931A02809178009091790090931D
:103DD00017068093160680911B0290911C029C018D
:103DE000442737FD4095542F80910303909104039D
:103DF000A0910503B0910603820F931FA41FB51F66
:103E00008093030390930403A0930503B0930603E8
:103E10002091030330910403409105035091060360
:103E200057FF04C021503C4F4F4F5F4F0AE055955C
:103E30004795379527950A95D1F78091030390917F
:103E40000403A0910503B0910603821B930BA40BFE
:103E5000B50B8093030390930403A0930503B093E1
:103E600006032EC180913102909132022091780098
:103E700030917900820F931F909332028093310228
:103E800010922D0250C2809102018A3071F480910B
:103E900078009091790020912F0230913002820FAA
:103EA000931F01969695879517C040912F025091C8
:103EB0003002843159F42091780030917900240F38
:103EC000351F8FEF97E0821B930B06C0809178001F
:103ED00090917900840F951F909322028093210284
:103EE00086E01FC28091470390914803209178009B
:103EF00030917900821B930B9093150680931406E2
:103F000080911406909115062091390230913A0261
:103F1000820F931F9093200280931F0287E001C2BB
:103F200080917800909179002091490330914A0363
:103F3000821B930B90931F0680931E0680911E0692
:103F400090911F0620913B0230913C02820F931FFB
:103F500090931E0280931D02E3C1209133023091A1
:103F600034028091780090917900280F391F3093A6
:103F7000340220933302809102018A3019F4220F17
:103F8000331F04C0220F331F220F331F309334021C
:103F9000209333022091330230913402C90137FD5E
:103FA0000796A3E095958795AA95E1F79093260249
:103FB000809325028091350290913602820F931FE3
:103FC00097FD0196959587959093360280933502DB
:103FD0002091530330915403821B930B909324013F
:103FE0008093230120912B0230912C028091230198
:103FF00090912401280F391F37FF02C02F5F3F4FD8
:104000003595279530932C0220932B02E0CD2091FB
:104010003102309132028091780090917900280F1E
:10402000391F3093320220933102809102018A308D
:1040300019F4220F331F04C0220F331F220F331F26
:1040400030933202209331022091310230913202BA
:10405000C90137FD079663E0959587956A95E1F765
:10406000909324028093230280913702909138022A
:10407000820F931F97FD019695958795909338022F
:10408000809337022091510330915203821B930B8E
:1040900090932201809321012091290230912A02DC
:1040A0008091210190912201280F391F37FF02C012
:1040B0002F5F3F4F3595279530932A022093290291
:1040C00083E02FC110922E0281E08093170180912E
:1040D00011029091120201969093120280931102A4
:1040E000809178009091790090931C0180931B013E
:1040F00080911B0190911C01AA27BB27A0903D0233
:10410000B0903E02C0903F02D0904002A80EB91E6F
:10411000CA1EDB1EA0923D02B0923E02C0923F0238
:10412000D0924002809141028F5F809341028231A0
:1041300008F4F6C080911D0190911E01A0911F010D
:10414000B09120017C018D0123E0EE0CFF1C001FCB
:10415000111F2A95D1F7E81AF90A0A0B1B0BEA0C72
:10416000FB1C0C1D1D1D80911502992787FD909544
:10417000A92FB92FBC01CD0126EC34E240E050E07C
:104180000E945772DC01CB01E81AF90A0A0B1B0BDB
:10419000D801C7010496A11DB11DB7FF05C0D80104
:1041A000C7010B96A11DB11D13E0B595A795979575
:1041B00087951A95D1F780931D0190931E01A093C6
:1041C0001F01B093200180911806909119067C017F
:1041D0000027F7FC0095102F80911D0190911E0182
:1041E000A0911F01B0912001E81AF90A0A0B1B0BDC
:1041F000E092E102F092E2020093E3021093E40203
:104200002091160230911702409118025091190224
:1042100057FF04C0215F3F4F4F4F5F4FF4E055956C
:10422000479537952795FA95D1F780911602909189
:104230001702A0911802B0911902821B930BA40BD4
:10424000B50B8093160290931702A0931802B093B7
:1042500019028091160290911702A0911802B09154
:1042600019028E0D9F1DA01FB11F809316029093FF
:104270001702A0931802B093190280911302909133
:104280001402AC01E4E0440F551FEA95E1F7481B26
:10429000590B8091160290911702A0911802B091CB
:1042A0001902B7FF03C00F96A11DB11D74E0B595AB
:1042B000A795979587957A95D1F72091E10230914E
:1042C000E202281B390B63E0220F331F6A95E1F7E6
:1042D000240F351F37FF02C0215F3F4F44E0359563
:1042E00027954A95E1F73093140220931302D601E3
:1042F000C501D7FE03C00196A11DB11DB595A795B7
:104300009795879580933D0290933E02A0933F023C
:10431000B093400289E08093410202C010922E02C5
:1043200082E080932D0280912D0280937C00809109
:104330002E02882319F08FEC80937A00FF91EF9181
:10434000BF91AF919F918F917F916F915F914F91AD
:104350003F912F911F910F91FF90EF90DF90CF90A1
:10436000BF90AF900F900FBE0F901F90189590E2E6
:10437000E8E2F1E08FE49193815087FFFCCF08954C
:1043800090914402E8E2F1E0E90FF11D80839F5F24
:10439000909344020895EF92FF920F931F93CF934F
:1043A000DF932091420220FF0AC0809143028823BC
:1043B00011F0815002C0809127018093430221FFB8
:1043C0000CC09091430280912701981719F4109224
:1043D000430203C09F5F90934302822F992780FF7F
:1043E00004C081FF02C0109243020E94B721809155
:1043F0004302282F3327C0ECEC2EC1E2FC2EC091E3
:10440000FF03D09100048A3098F481E18093440244
:104410003F932F9382E295E09F938F93FF92EF92C9
:10442000FE0109952DB73EB72A5F3F4F2DBF11C042
:1044300080E1809344023F932F9387E295E09F931E
:104440008F93FF92EF92FE0109958DB79EB7069666
:104450008DBF20914302822F9927AA27BB27FC01F9
:10446000419710F00C94E42BE05BFF4FB0ECEB2E87
:10447000B1E2FB2EC091FF03D09100040C941D7398
:10448000109244028CE295E09F938F93FF92EF92FB
:10449000FE01099584E1809344020F900F900F90E4
:1044A0000F9084E690E09F938F938EE490E09F932B
:1044B0008F931F921F92809102016AE00E94767290
:1044C000892F99279F938F93809102010E94767282
:1044D00099279F938F938CE395E09F938F93FF92FF
:1044E000EF92E091FF03F0910004099588E2809338
:1044F00044022DB73EB7225F3F4F2DBF82E094E0CC
:104500009F938F930E94710799279F938F9381E5C3
:1045100095E09F938F93FF92EF92E091FF03F091CC
:104520000004099580919F019091A0012DB73EB79D
:10453000285F3F4F2DBF069730F48CE380934402F1
:104540008FE595E0CDC090914702992311F40C942A
:10455000ED2B8CE380934402892F99279F938F93AF
:104560008CE695E09F938F9380EC91E29F938F93DD
:1045700077C08091CF06A0ECEA2EA1E2FA2EC0917E
:10458000FF03D091000480FF74C010924402809118
:10459000E1029091E202A091E302B091E402BC0139
:1045A000CD0125E030E040E050E00E94CB723F9327
:1045B0002F9381E895E09F938F93FF92EF92FE01F6
:1045C000099584E1809344022DB73EB72A5F3F4F9F
:1045D0002DBF8091DD029091DE02A091DF02B091AB
:1045E000E002BC01CD0125E030E040E050E00E9457
:1045F000CB723F932F938EE895E09F938F93FF921A
:10460000EF92E091FF03F0910004099588E2809316
:1046100044028DB79EB706968DBF80911B01909185
:104620001C019F938F938BE995E09F938F93FF924B
:10463000EF92E091FF03F091000409958CE38093E1
:1046400044022DB73EB72A5F3F4F2DBF87B599274C
:104650009F938F9388EA95E09F938F93FF92EF92B9
:10466000E091FF03F091000409958DB79EB706967F
:1046700039C71092440285EB95E09F938F93FF9288
:10468000EF92FE01099584E1809344020F900F9010
:104690000F900F9084EC95E09F938F93FF92EF9291
:1046A000E091FF03F0910004099588E280934402B1
:1046B0000F900F900F900F908DEC95E09F938F933C
:1046C000FF92EF92E091FF03F091000409958CE3D3
:1046D000809344020F900F900F900F908CED95E017
:1046E0009F938F93FF92EF92EFC71092440285EE53
:1046F00095E09F938F9300EC11E2FF92EF92FE0101
:10470000099584E1809344020F900F900F900F90D1
:1047100080913B0390913C03A0913D03B0913E03F7
:10472000B7FF04C081509C4FAF4FBF4FFAE0B59523
:10473000A79597958795FA95D1F7BF93AF939F93D8
:104740008F9382EF95E09F938F931F930F93E09148
:10475000FF03F0910004099588E2809344022DB78D
:104760003EB7285F3F4F2DBF8091330390913403B4
:10477000A0913503B0913603B7FF04C081509C4F20
:10478000AF4FBF4FEAE0B595A79597958795EA9506
:10479000D1F7BF93AF939F938F9381E096E09F9360
:1047A0008F931F930F93E091FF03F09100040995FD
:1047B0008CE3809344028DB79EB708968DBF80919D
:1047C0000103909102039F938F9380E196E09F9362
:1047D0008F931F930F93EEC310924402809158065B
:1047E000909159069F938F9380915606909157060A
:1047F0009F938F938FE196E09F938F93FF92EF9219
:10480000FE01099584E1809344028DB79EB7089616
:104810008DBF80915C0690915D069F938F938091F0
:104820005A0690915B069F938F938FE296E09F9339
:104830008F93FF92EF92E091FF03F09100040995AE
:1048400088E2809344022DB73EB7285F3F4F2DBFCB
:1048500080916006909161069F938F9380915E0690
:1048600090915F069F938F938FE396E09F938F9332
:10487000FF92EF92E091FF03F091000409958CE321
:10488000809344028DB79EB708968DBF80916406D1
:10489000909165069F938F93809162069091630635
:1048A0009F938F938FE496E076C510924402809197
:1048B000C406E82FFF27EE0FFF1FEC5AF94F808147
:1048C00091819F938F938091C306E82FFF27EE0F6E
:1048D000FF1FEC5AF94F808191819F938F938FE551
:1048E00096E09F938F93FF92EF92FE01099584E1EA
:1048F000809344028DB79EB708968DBF8091C606FF
:10490000E82FFF27EE0FFF1FEC5AF94F80819181AE
:104910009F938F938091C506E82FFF27EE0FFF1F0F
:10492000EC5AF94F8081918188589F4F9F938F93C4
:104930008FE696E09F938F93FF92EF92E091FF03B3
:10494000F0910004099588E2809344022DB73EB7A8
:10495000285F3F4F2DBF8091C806E82FFF27EE0F3D
:10496000FF1FEC5AF94F8081918182599F4F9F938D
:104970008F938091C706E82FFF27EE0FFF1FEC5A99
:10498000F94F8081918182599F4F9F938F938FE739
:1049900096E09F938F93FF92EF92E091FF03F09147
:1049A000000409958CE3809344028DB79EB7089666
:1049B0008DBF8091CA06E82FFF27EE0FFF1FEC5A2C
:1049C000F94F8081918182599F4F9F938F9380915E
:1049D000C906E82FFF27EE0FFF1FEC5AF94F808121
:1049E000918182599F4F9F938F938FE896E0D3C414
:1049F000109244028FE996E09F938F9300EC11E2AE
:104A0000FF92EF92FE010995809102010F900F90A5
:104A10000F900F908A3009F0A1C084E18093440286
:104A200080915303909154039C0197FF02C0295F2A
:104A30003F4F287F821B930B9F938F93809153034B
:104A40009091540397FD079673E0959587957A9515
:104A5000E1F79F938F93209153033091540337FFD5
:104A600002C0295F3F4F63E0359527956A95E1F7CE
:104A70008091250290912602821B930B9F938F9326
:104A80008DEA96E09F938F931F930F93E091FF031E
:104A9000F0910004099588E2809344028DB79EB797
:104AA0000A968DBF80915103909152039C0197FF0C
:104AB00002C0295F3F4F287F821B930B9F938F93E8
:104AC000809151039091520397FD079653E095957D
:104AD00087955A95E1F79F938F93209151033091D9
:104AE000520337FF02C0295F3F4F43E035952795BA
:104AF0004A95E1F78091230290912402821B930B47
:104B00009F938F938EEB96E09F938F931F930F93BA
:104B1000E091FF03F091000409958CE38093440237
:104B20002DB73EB7265F3F4F2DBF80914F03909129
:104B300050039F938F9380914F0390915003209146
:104B4000210230912202821B930B9F938F938FEC53
:104B500096E09F938F931F930F93B6C38B3019F0FA
:104B6000843109F0ADC084E1809344028091530305
:104B7000909154039C0197FF02C0215F3F4F207F1B
:104B8000821B930B97FD0196959587959F938F9325
:104B9000809153039091540397FD0F9624E09595CF
:104BA00087952A95E1F79F938F9320915303309136
:104BB000540337FF02C0295F3F4F83E035952795A7
:104BC0008A95E1F78091250290912602821B930B32
:104BD0009F938F938DED96E09F938F931F930F93E9
:104BE000E091FF03F0910004099588E2809344026C
:104BF0002DB73EB7265F3F4F2DBF80915103909157
:104C000052039C0197FF02C0215F3F4F207F821B10
:104C1000930B97FD0196959587959F938F93809120
:104C200051039091520397FD0F96B4E095958795A7
:104C3000BA95E1F79F938F932091510330915203DE
:104C400037FF02C0295F3F4FA3E035952795AA950E
:104C5000E1F78091230290912402821B930B9F9392
:104C60008F938FEE96E09F938F931F930F93E09116
:104C7000FF03F091000409958CE3809344028DB703
:104C80009EB70A968DBF80914F039091500397FD78
:104C90000196959587959F938F9380914F0390915F
:104CA00050032091210230912202821B930B9F938B
:104CB0008F9381E097E09F938F931F930F936FC320
:104CC0008D3009F08AC584E18093440280911A01F5
:104CD00099279F938F93809153039091540397FD4D
:104CE0000F96E4E095958795EA95E1F79F938F936A
:104CF000209153033091540337FF02C0295F3F4F87
:104D000073E0359527957A95E1F78091250290918A
:104D10002602821B930B9F938F9380E197E09F93D2
:104D20008F931F930F93E091FF03F0910004099577
:104D300088E2809344028DB79EB70A968DBF80911A
:104D4000190199279F938F9380915103909152035A
:104D500097FD0F9664E0959587956A95E1F79F9387
:104D60008F93209151033091520337FF02C0295F86
:104D70003F4F53E0359527955A95E1F780912302EF
:104D800090912402821B930B9F938F9384E297E070
:104D90009F938F931F930F93E091FF03F091000473
:104DA00009958CE3809344022DB73EB7265F3F4FB1
:104DB0002DBF8091180199279F938F9380914F0366
:104DC0009091500397FD0196959587959F938F93AA
:104DD00080914F0390915003209121023091220243
:104DE000821B930B9F938F9388E397E09F938F93FE
:104DF0001F930F93E091FF03F091000409958DB785
:104E00009EB70A966FC3109244028CE497E09F937A
:104E10008F93FF92EF92FE01099584E18093440203
:104E20000F900F900F900F908091490390914A033B
:104E30009F938F9380911D0290911E029F938F9359
:104E400089E597E09F938F93FF92EF92E091FF03A4
:104E5000F0910004099588E2809344022DB73EB793
:104E6000285F3F4F2DBF80914703909148039F9348
:104E70008F9380911F02909120029F938F9388E6D9
:104E800097E09F938F93FF92EF92E091FF03F09151
:104E9000000409958CE3809344028DB79EB7089671
:104EA0008DBF8091410390914203A0914303B09143
:104EB0004403BC01CD010E947071DC01CB019F93C2
:104EC0008F9380914B0790914C079F938F9387E727
:104ED00097E061C2109244028091250190912601D1
:104EE0006AE070E00E9496729F938F9380912501F3
:104EF000909126016AE070E00E9496727F936F9312
:104F000086E897E09F938F93FF92EF92FE010995B9
:104F100084E1809344028DB79EB708968DBF80913F
:104F20000008909101086AE070E00E9482729F93ED
:104F30008F9380910008909101086AE070E00E94D0
:104F400082727F936F938AE997E09F938F93FF928A
:104F5000EF92E091FF03F0910004099588E28093BD
:104F600044022DB73EB7285F3F4F2DBF8091020806
:104F7000909103089F938F938EEA97E09F938F936E
:104F8000FF92EF92E091FF03F091000409958CE30A
:104F9000809344028DB79EB706968DBF809104081A
:104FA000909105089F938F938EEB97E09F938F933B
:104FB000FF92EF92E091FF03F091000409952DB765
:104FC0003EB72A5F3F4FF4C11092440280ED97E054
:104FD0009F938F93FF92EF92FE01099584E1809356
:104FE00044020F900F900F900F9080915406909173
:104FF00055069F938F9389ED97E09F938F93FF9230
:10500000EF92E091FF03F0910004099588E280930C
:1050100044028DB79EB706968DBF8091EF02992707
:105020009F938F9389EE97E09F938F93FF92EF92D8
:10503000E091FF03F091000409958CE38093440212
:105040002DB73EB72A5F3F4F2DBF8091530699275A
:1050500001979F938F9389EF97E0FECA10924402C5
:1050600089E098E09F938F93FF92EF92FE0109955C
:1050700084E1809344020F900F900F900F908091E5
:10508000FD029091FE029F938F9381E198E09F93A0
:105090008F93FF92EF92E091FF03F0910004099546
:1050A00088E2809344022DB73EB72A5F3F4F2DBF61
:1050B00080910103909102039F938F938FE198E079
:1050C0009F938F93FF92EF92E091FF03F091000482
:1050D00009958CE3809344028DB79EB706968DBFE9
:1050E0008091FF02909100039F938F938DE298E04F
:1050F0005DCF109244028091F00299279F938F9385
:105100008BE398E09F938F93FF92EF92FE010995B6
:1051100084E1809344028DB79EB706968DBF80913F
:10512000F10299279F938F9387E498E09F938F9341
:10513000FF92EF92E091FF03F0910004099588E25D
:10514000809344022DB73EB72A5F3F4F2DBF809119
:10515000F20299279F938F9383E598E09F938F9313
:10516000FF92EF92E091FF03F091000409958CE328
:10517000809344028DB79EB706968DBF8091F3024F
:1051800099279F938F938FE598E010CF1092440258
:105190008091F40299279F938F938BE698E09F93D9
:1051A0008F93FF92EF92FE01099584E18093440270
:1051B0008DB79EB706968DBF8091F50299279F9374
:1051C0008F9387E798E09F938F93FF92EF92E09100
:1051D000FF03F0910004099588E2809344022DB703
:1051E0003EB72A5F3F4F2DBF8091F60299279F93CC
:1051F0008F9383E898E09F938F93FF92EF92E091D3
:10520000FF03F091000409958CE3809344028DB76D
:105210009EB706968DBF8091F70299279F938F9333
:105220008FE898E0C3CE109244028BE998E09F93F8
:105230008F93FF92EF92FE01099584E180934402DF
:105240000F900F900F900F908091850199279F9359
:105250008F9383EA98E09F938F93FF92EF92E09170
:10526000FF03F0910004099588E2809344028DB712
:105270009EB706968DBF8091FA019091FB019F9396
:105280008F9381EB98E09F938F93FF92EF92E09141
:10529000FF03F091000409958CE3809344022DB73D
:1052A0003EB72A5F3F4F2DBF8091F10699279F930C
:1052B0008F938091F00699279F938F938FEB98E0BF
:1052C0009F938F93FF92EF92E091FF03F091000480
:1052D00009958DB79EB7089605C1109244028DECD2
:1052E00098E09F938F93FF92EF92FE01099584E1DE
:1052F000809344020F900F900F900F90809186043E
:10530000992787FD90959F938F9380918504992786
:1053100087FD90959F938F938DED98E09F938F934A
:10532000FF92EF92E091FF03F0910004099588E26B
:10533000809344022DB73EB7285F3F4F2DBF809129
:105340008704992787FD90959F938F938091880478
:1053500099279F938F938DEE98E09F938F93FF9261
:10536000EF92E091FF03F091000409958CE38093A4
:1053700044028DB79EB708968DBF80918C04992703
:105380009F938F9380918904992787FD90959F9390
:105390008F938DEF98E09F938F93FF92EF92E09120
:1053A000FF03F091000409952DB73EB7285F3F4FEA
:1053B0002DBF13C2109244028DE099E09F938F930A
:1053C000FF92EF92FE01099584E1809344020F90D1
:1053D0000F900F900F908091300699278F779070E3
:1053E0009F938F9380912C0699278F7790709F932E
:1053F0008F938091280699278F7790709F938F9332
:105400008091240699278F7790709F938F938DE1D9
:1054100099E09F938F93FF92EF92E091FF03F091B9
:105420000004099588E2809344028DB79EB70C96DC
:105430008DBF8091400699278F7790709F938F93AF
:1054400080913C0699278F7790709F938F938091DE
:10545000380699278F7790709F938F9380913406A9
:1054600099278F7790709F938F938EE299E09F9307
:105470008F93FF92EF92E091FF03F0910004099562
:105480008CE3809344022DB73EB7245F3F4F2DBF7E
:105490008091500699278F7790709F938F9380917A
:1054A0004C0699278F7790709F938F938091480631
:1054B00099278F7790709F938F93809144069927B7
:1054C0008F7790709F938F938FE399E09F938F9343
:1054D000FF92EF92E091FF03F091000409958DB7E0
:1054E0009EB70C968DBF79C11092440280E599E079
:1054F0009F938F9300EC11E2FF92EF92FE010995CA
:1055000084E1809344020F900F900F900F90809150
:105510003006881F8827881F97E0899FC0011124C3
:105520008D969F938F9380912C06881F8827881FC4
:1055300096E0899FC00111248D969F938F9380914F
:105540002806881F8827881F95E0899FC00111249D
:105550008D969F938F9380912406881F8827881F9C
:105560009927880F991F880F991F8D969F938F9366
:105570008FE599E09F938F93FF92EF92E091FF0365
:10558000F0910004099588E2809344022DB73EB75C
:10559000245F3F4F2DBF80914006881F8827881FBA
:1055A0009BE0899FC00111248D969F938F938091DA
:1055B0003C06881F8827881F9AE0899FC001112414
:1055C0008D969F938F9380913806881F8827881F18
:1055D00099E0899FC00111248D969F938F938091AC
:1055E0003406881F8827881F992723E0880F991F72
:1055F0002A95E1F78D969F938F9383E799E09F9388
:105600008F93FF92EF92E091FF03F09100040995D0
:105610008CE3809344028DB79EB70C968DBF80912A
:105620004406881F8827881F9CE0899FC001112499
:105630008D969F938F9387E899E09F938F93FF9226
:10564000EF92E091FF03F0910004099580914806E4
:105650002DB73EB72A5F3F4F2DBF87FF12C080E4B2
:105660008093440288E999E09F938F93FF92EF9291
:10567000E091FF03F091000409950F900F900F90B7
:105680000F9080914C0687FF12C084E480934402FF
:105690008BE999E09F938F931F930F93E091FF0302
:1056A000F091000409950F900F900F900F9080914A
:1056B000500687FF92C088E4809344028EE999E007
:1056C0009F938F931F930F93E091FF03F09100043A
:1056D00009950F900F900F900F907FC01092440289
:1056E00081EA99E09F938F93FF92EF92FE010995D3
:1056F00084E1809344020F900F900F900F9080915F
:10570000D2019091D3019F938F938FEA99E09F9359
:105710008F93FF92EF92E091FF03F09100040995BF
:1057200088E2809344028DB79EB706968DBF809124
:10573000D4019091D5019F938F938CEB99E09F9327
:105740008F93FF92EF92E091FF03F091000409958F
:1057500089E4809344022DB73EB72A5F3F4F2DBFA7
:1057600089EC99E09F938F93FF92EF92E091FF0372
:10577000F09100040995809142020F900F900F90D4
:105780000F9083FF2AC01092D5011092D401F9998D
:10579000FECF1FBA8EE090E092BD81BD10BC0FB667
:1057A000F894FA9AF99A0FBE2091D401F999FECF94
:1057B0001FBA8FE090E092BD81BD20BD0FB6F89476
:1057C000FA9AF99A0FBE09C080912701281719F497
:1057D0002150209327011092430210924202E6E0EA
:1057E000CDB7DEB70C940E731092B9008AE28093A5
:1057F000B800089585EA8093BC00089584E98093F9
:10580000BC0008951092B9008093BB0085E8809396
:10581000BC0008950E94FE2B10924A028091BB00AA
:105820001092490280E88093BC001092BD00109253
:10583000BA001092BB001092B9001092B8000E94FA
:10584000F42B0E94FA2B80E00E94022C0895809392
:10585000BB0085E88093BC00089585EC8093BC0074
:10586000089585E88093BC0008951F920F920FB6AB
:105870000F9211242F933F934F935F936F937F93D6
:105880008F939F93AF93BF93EF93FF9380914A02BF
:10589000282F3327442755278F5F80934A02F90129
:1058A0002731310508F0F2C0EF59FF4F0C941D73FA
:1058B00020914902E22FFF27EE0FFF1FEE0FFF1F7F
:1058C000EF5FFB4F85851816A4F02C3090F4922FD3
:1058D0009F5FE92FFF27EE0FFF1FEE0FFF1FEF5F08
:1058E000FB4F858518161CF0292F9C3080F3909370
:1058F0004902809149028C3051F41092490283E0B0
:1059000080934A0280914802880F8D5AB4C0880F54
:105910008E5AB1C080914902E82FFF27EE0FFF1F7A
:10592000EE0FFF1FED5DF94F8F5F8093490280817D
:10593000A2C08091B9008033E1F480914B028823AA
:1059400021F48091490280934B0280914902E82F13
:10595000FF27EE0FFF1FEE0FFF1FE05EF94F2081C4
:10596000822F99278F7790708F37910514F42F5FCE
:1059700020830E94FE2B8AE090E09093A001809308
:105980009F0110924A026CC08091B9009091480228
:105990008034C1F0E92FFF27EE0FFF1FEE0FFF1F2E
:1059A000ED5DF94F81818F778183892F8F5F8093A0
:1059B00048028C3010F0109248020E94FE2B109288
:1059C0004A020DC0E92FFF27EE0FFF1FEE0FFF1F4A
:1059D000ED5DF94F8181806881830E942D2C80913B
:1059E0004B028093470210924B0252C080914802B2
:1059F000E82FFF27EE0FFF1FEE0FFF1FED5DF94FA2
:105A00008091BB0082830E94312C42C09091480259
:105A1000E92FFF27EE0FFF1FEE0FFF1FED5DF94F80
:105A20008091BB008383892F8F5F809348028C30E5
:105A300010F0109248020E94FE2B28C080E11BC08B
:105A400080911A0118C082E116C08091190113C01B
:105A50000E94FE2B8AE090E09093A00180939F012A
:105A60000E94FA2B15C088E906C084E104C0809129
:105A7000180101C080E80E94022C0AC00E94FE2B7F
:105A80008AE090E09093A00180939F0110924A02D7
:105A90008091BC0080688093BC00FF91EF91BF9122
:105AA000AF919F918F917F916F915F914F913F91B6
:105AB0002F910F900FBE0F901F90189589E1A8E8C5
:105AC000B6E0E4E5F6E011821082329611961C925F
:105AD0001E921296815087FFF6CF109250031092BB
:105AE0004F031092520310925103109254031092DC
:105AF000530308951F920F920FB60F9211240F9324
:105B00001F932F933F934F935F936F937F938F9345
:105B10009F93AF93BF93CF93DF93EF93FF938091C6
:105B2000220782FDC8C04091860050918700809175
:105B30004D0290914E02481B590B80918600909126
:105B4000870090934E0280934D02CA018D54944079
:105B5000A0914F02B0915002835F9A4178F48091F6
:105B60004F0280935306149714F01092780181E04D
:105B700090E09093500280934F02FCC1AD30B1058C
:105B80000CF0F8C1CA018B5F9040845B914008F033
:105B900074C0425D5140FD01EA0FFB1FEC5AF94F02
:105BA00080819181FA01E81BF90BCF01F7FF03C057
:105BB000909581959F4F06975CF48091EF02883C09
:105BC00020F48091EF02865F01C088EC8093EF02A1
:105BD000FD01EA0FFB1FEC5AF94F808191819C0176
:105BE000220F331F280F391F240F351F37FF02C024
:105BF0002D5F3F4FE901D595C795D595C795CA014A
:105C000001968C179D0714F4219706C0415050400F
:105C1000C417D5070CF421968091EF02833CE0F085
:105C20008D010A0F1B1FF801EC5AF94F80819181F9
:105C30009E01281B390BC90163E070E00E94967237
:105C4000CB01880F991F860F971F0857194FD8014E
:105C500011969C938E9307C0AA0FBB1FA857B94FEC
:105C600011961C921E92E0914F02F0915002EE0F9D
:105C7000FF1FEC5AF94FD183C08380914F0290915E
:105C8000500201969093500280934F02059711F4B1
:105C90005D9A01C05D9880914F02909150028630CC
:105CA000910511F45C9A01C05C98079711F45B9A16
:105CB00061C15B985FC140918600509187008091DF
:105CC000510290915202481B590B8091860090918D
:105CD00087009093520280935102CA018D549440E0
:105CE0006091BB02835F9A4108F07AC060934C02D6
:105CF00080914C02843008F453C0909153068091F7
:105D00004C02981709F04CC05091BC025B3008F46B
:105D10003FC0109278011092BB0240E05F31C0F0AA
:105D2000E42FFF27EE0FFF1F9F0129573D4FDF0193
:105D3000AC5AB94F8D919C91D9018D939C93DF0101
:105D4000A857B94F8D919C91EF55FD4F918380835A
:105D5000E42FFF27EE0FFF1F9F012C5A394FDF0161
:105D6000AD5ABD4F8D919C91D90111969C938E9304
:105D7000DF01A359BD4F8D919C91E857F94F918355
:105D80008083842F8F5F482F8D3040F28093BB0239
:105D90008091BC028F3FB9F08F5F8093BC0213C02B
:105DA0008091BC02853620F08AE08093BC0202C05C
:105DB0001092BC02809102018A3011F0843111F4FA
:105DC000289A01C0289881E08093BB028091E50267
:105DD000882309F0CFC080914C0280935306CAC03B
:105DE0006D3008F09FC0CA018B5F9040845B91408A
:105DF00008F07EC0425D5140E62FFF27EE0FFF1FE7
:105E0000ED5AFD4F80819181FA01E81BF90BCF011A
:105E100005960B97B0F48091BC028A3120F08091F6
:105E2000EF02865F05C08B3028F08091EF028E5F15
:105E30008093EF028091EF02893C18F088EC809308
:105E4000EF02E62FFF27EE0FFF1FED5AFD4F808177
:105E500091819C01220F331F280F391F240F351FFA
:105E600037FF02C02D5F3F4FE901D595C795D59506
:105E7000C795CA0101968C179D0714F4219706C097
:105E800041505040C417D5070CF421968091EF0281
:105E90008E3BD8F0E62FFF27EE0FFF1FDF01AD5A34
:105EA000BD4F8D919C919E01281B390BC90163E068
:105EB00070E00E949672CB01880F991F860F971F82
:105EC000E359FD4F9183808308C0E62FFF27EE0F33
:105ED000FF1FE359FD4F118210828091BB02E82F12
:105EE000FF27EE0FFF1FED5AFD4FD183C08309C07E
:105EF000809102018A3011F0843111F4289A01C096
:105F000028988091BB02853011F45D9A05C05D9898
:105F1000863011F45C9A05C05C98873011F45B9A66
:105F200001C05B988091BB02843120F48F5F809325
:105F3000BB0220C08431F1F4809102018A3011F05B
:105F4000843111F4289A01C028988EE18093BB0215
:105F50002CE0C8E8D6E0A7E8B2E0E4E5F6E08D91F1
:105F60009D919183808332961982188222962150C6
:105F700027FFF5CFFF91EF91DF91CF91BF91AF91C7
:105F80009F918F917F916F915F914F913F912F9151
:105F90001F910F910F900FBE0F901F90189581E0E9
:105FA0008093C50682E08093C40683E08093C30695
:105FB00084E08093C60685E08093C70686E08093E0
:105FC000C80687E08093C90688E08093CA0689E006
:105FD0008093CB068AE08093CC068BE08093CD063D
:105FE0008CE08093CE0608951F938AE68093CF06B7
:105FF00061E0609322075EE15093D0068FEF8093BB
:10600000D2068AE08093D3065093D1065093D506EA
:1060100085E08093D60680E48093D7061092D80658
:1060200084E18093D4068EE08093D906F0E1F0936A
:10603000DA061CE01093DB06A8E0A093DC0686EEEF
:106040008093DD065093DE0680E88093DF0640E50E
:106050004093E00696E99093E10683E08093E206A0
:106060004093E3069093E40681E28093E50683E2A1
:106070008093E6065093E70670E27093E90610926B
:10608000EA061092EB061092EC061092ED061092C2
:10609000050710920607109207071092080724E6DA
:1060A0002093EE0638E23093EF06609321071092BA
:1060B000F00697EF9093F106E6E0E093F6068DE7A1
:1060C0008093F7068093F8068093F9062093F206F2
:1060D0003093F3061092F4069093F50682E38093D2
:1060E000FA069AE59093FB068093FC06109220072F
:1060F0009093FD064093FE066093FF0685E580932E
:10610000000780930107F093020770930307209321
:1061100004078FE58093090783EF80930B078AEAD2
:1061200080930D0780930E078FE080930A0780937A
:106130000C078EEF80930F072093100790931107A1
:1061400090931207909313078BE480931407809326
:1061500015078093160710921707E0931807A0936E
:10616000190790931A0750931B0720931C0720933D
:106170001D0784E080931E076093E806A1EAB1E062
:10618000E3E2F7E00D9001921A95E1F71F9108956F
:106190008AE68093CF06E1E0E09322076EE1609308
:1061A000D0068FEF8093D2069AE09093D306609347
:1061B000D1066093D50685E08093D60680E480936F
:1061C000D7061092D8068FE08093D4069093D90614
:1061D00080E18093DA0676E07093DB06F8E0F093D6
:1061E000DC0686EE8093DD066093DE0680E8809311
:1061F000DF062AE52093E00698E79093E10683E026
:106200008093E2062093E3069093E40681E2809374
:10621000E50683E28093E6066093E70650E250933A
:10622000E9061092EA061092EB061092EC06109224
:10623000ED061092050710920607109207071092BC
:10624000080744E64093EE0638E23093EF06E09309
:1062500021071092F00697EF9093F1067093F606DF
:106260008DE78093F7068093F8068093F9064093B4
:10627000F2063093F3061092F4069093F50682E34B
:106280008093FA062093FB068093FC061092200769
:106290002093FD0680E58093FE068CE38093FF0645
:1062A00085E5809300078093010750930207509380
:1062B00003079BE4909304078FE58093090783EF1E
:1062C00080930B078AEA80930D0780930E0784E181
:1062D00080930A0780930C078EEF80930F074093FB
:1062E0001007209311072093120720931307909310
:1062F0001407909315079093160710921707709341
:106300001807F093190720931A0760931B0740930F
:106310001C0740931D0784E080931E07E093E80666
:106320008CE0A8EAB1E0E3E2F7E00D9001928A95F3
:10633000E1F708958AE68093CF0671E07093220713
:106340004EE14093D0068FEF8093D2068AE080938F
:10635000D3064093D1064093D50685E08093D606B8
:1063600080E48093D7061092D8068FE08093D406FD
:1063700068E06093D90620E12093DA0656E0509356
:10638000DB066093DC0686EE8093DD064093DE0636
:1063900080E88093DF0634E63093E00698E7909338
:1063A000E10683E08093E2063093E3069093E406EF
:1063B00081E28093E50683E28093E60684E18093A0
:1063C000E7062093E9061092EA061092EB06109277
:1063D000EC061092ED061092050710920607109237
:1063E0000707109208073093EE0628E22093EF0685
:1063F000709321071092F00697EF9093F106509357
:10640000F6068DE78093F7068093F8068093F906E9
:106410003093F2062093F3061092F4069093F5065B
:1064200092E39093FA062AE52093FB069093FC06EC
:10643000109220072093FD0680E58093FE0686E4F7
:106440008093FF0685E5809300078093010780E233
:106450008093020780930307909304078FE580934E
:10646000090783EF80930B078AEA80930D078093D7
:106470000E0740930A0740930C078EEF80930F0797
:1064800030931007209311072093120720931307CE
:106490008BE480931407809315078093160710925E
:1064A0001707509318076093190720931A07409312
:1064B0001B0730931C0730931D0784E080931E0751
:1064C0007093E8068CE0A0EBB1E0E3E2F7E00D901A
:1064D00001928A95E1F708956817790754F4680FD7
:1064E000791F77FF02C06F5F7F4FCB01959587952E
:1064F0000895681B790B861B970B08951F93CF9304
:10650000DF93182FEB018091E5028823A1F411504D
:106510001F3F89F0D093FF01C093FE018091FE01DF
:106520009091FF01892BD1F7CE018C0F9D1F0E9406
:10653000F617115078F7DF91CF911F910895A3E1DD
:10654000B0E0E5EAF2E30C94E67280914F0390919B
:1065500050032091210230912202821B930B9093D1
:1065600084078093830780912B0290912C0297FDE2
:1065700007969C0153E0359527955A95E1F730939E
:106580004107209340078091290290912A0297FDAC
:10659000079643E0959587954A95E1F790933207E2
:1065A0008093310730934E0720934D079093440713
:1065B0008093430780917E0790917F07AA2797FDDC
:1065C000A095BA2F7C018D01EE0CFF1C001F111F3E
:1065D000E80EF91E0A1F1B1F80911D0290911E02DA
:1065E0009C01442737FD4095542FDA01C901F2E0A0
:1065F000880F991FAA1FBB1FFA95D1F7820F931F0F
:10660000A41FB51F820F931FA41FB51FE80EF91E0C
:106610000A1F1B1F17FF08C023E030E040E050E0D6
:10662000E20EF31E041F151FE2E015950795F7947F
:10663000E794EA95D1F7F0927F07E0927E07809188
:106640008E0790918F07AA2797FDA095BA2F7C01FE
:106650008D01EE0CFF1C001F111FE80EF91E0A1F12
:106660001B1F80911F02909120029C01442737FD3F
:106670004095542FDA01C90162E0880F991FAA1FC3
:10668000BB1F6A95D1F7820F931FA41FB51F820FFE
:10669000931FA41FB51FE80EF91E0A1F1B1F17FF2B
:1066A00008C083E090E0A0E0B0E0E80EF91E0A1F09
:1066B0001B1F82E015950795F794E7948A95D1F70B
:1066C000F0928F07E0928E0780914B0790914C07D4
:1066D000AA2797FDA095BA2F9C01AD01220F331F69
:1066E000441F551F280F391F4A1F5B1F80911B0233
:1066F00090911C02AA2797FDA095BA2F280F391F49
:106700004A1F5B1F57FF04C02D5F3F4F4F4F5F4F26
:10671000F2E05595479537952795FA95D1F730933F
:106720004C0720934B0720911D0230911E02C90196
:10673000880F991F880F991F820F931F820F931F35
:106740009C01442737FD4095542F80912B03909155
:106750002C03A0912D03B0912E03820F931FA41F31
:10676000B51F80932B0390932C03A0932D03B0931C
:106770002E0320911F0230912002C901880F991F1A
:10678000880F991F820F931F820F931F9C0144272C
:1067900037FD4095542F8091270390912803A091B5
:1067A0002903B0912A03820F931FA41FB51F809362
:1067B000270390932803A0932903B0932A03809181
:1067C00057079091580720911D0230911E02820FA9
:1067D000931F909358078093570780918607909155
:1067E000870720911F0230912002820F931F909300
:1067F0008707809386078091450390914603019611
:106800009093460380934503809123039091240342
:10681000A0912503B0912603BC01CD010E94A37174
:106820005B016C018091160690911706AA2797FDCF
:10683000A095BA2FBC01CD010E94A3717B018C01F0
:106840008091410390914203A0914303B09144038E
:106850009C01AD01C801B7010E940771DC01CB01A9
:106860009C01AD01C601B5010E940871DC01CB019C
:10687000BC01CD010E947071DC01CB018093230328
:1068800090932403A0932503B09326038FEC809369
:106890007A00109217012091130330911403409154
:1068A00015035091160329873A874B875C87295433
:1068B0003B46414050402CF028E43BE641E050E0AC
:1068C0000DC089859A85AB85BC85885B9449AE4FA0
:1068D000BF4F4CF428EB34E94EEF5FEF2D833E833E
:1068E0004F83588708C089859A85AB85BC858D8381
:1068F0009E83AF83B88720911B0330911C03409186
:106900001D0350911E032D873E874F87588B2954B6
:106910003B46414050402CF028E43BE641E050E04B
:106920000DC08D859E85AF85B889885B9449AE4F33
:10693000BF4F4CF428EB34E94EEF5FEF29833A83E5
:106940004B835C8308C08D859E85AF85B88989831C
:106950009A83AB83BC83A0918307B0918407BA8BE1
:10696000A98BFD01CF01AA2797FDA095BA2FA09072
:106970000B03B0900C03C0900D03D0900E03A80E33
:10698000B91ECA1EDB1EA0920B03B0920C03C0926C
:106990000D03D0920E03E0908A07F0908B070091D0
:1069A0008C0710918D07E80EF91E0A1F1B1FE0923D
:1069B0008A07F0928B0700938C0710938D07F09154
:1069C000D802FB8BFF2309F098C18091D70288235E
:1069D00009F093C18091CF0686FF8FC18091310766
:1069E00090913207AA2797FDA095BA2FBC01CD013F
:1069F00029813A814B815C810E9457729B01AC01D5
:106A000097FF04C02150384F4F4F5F4F6BE05595B3
:106A10004795379527956A95D1F780918101682E22
:106A2000772488249924CA01B901A40193010E9402
:106A30005772DC01CB0180935F0390936003A093B6
:106A40006103B0936203B7FF04C08150904FAF4F12
:106A5000BF4F1C012D013CE0559447943794279477
:106A60003A95D1F720925F03309260034092610320
:106A7000509262038091400790914107AA2797FDA9
:106A8000A095BA2FBC01CD012D813E814F81588543
:106A90000E94577297FF04C06150784F8F4F9F4FED
:106AA0002BE095958795779567952A95D1F7A40161
:106AB00093010E945772DC01CB0180936303909392
:106AC0006403A0936503B0936603B7FF04C08150CD
:106AD000904FAF4FBF4F9C01AD018CE0559547954E
:106AE000379527958A95D1F72093630330936403F4
:106AF000409365035093660380915F039091600318
:106B00009093BD068093BC068091630390916403CB
:106B10009093C1068093C006221933094409550990
:106B2000209363033093640340936503509366039B
:106B3000E20EF31E041F151FE0928A07F0928B07E6
:106B400000938C0710938D07809180018823B1F406
:106B500057FF04C02F5F3F4F4F4F5F4F55954795ED
:106B600037952795A21AB30AC40AD50AA0920B0337
:106B7000B0920C03C0920D03D0920E0329893A897A
:106B800079010027F7FC0095102F80916303909105
:106B90006403A0916503B0916603E80EF91E0A1F15
:106BA0001B1FC801B70129813A814B815C810E947A
:106BB00057729B01AC0197FF04C02150384F4F4FD3
:106BC0005F4FBBE05595479537952795BA95D1F717
:106BD00080918201A82EBB24CC24DD24CA01B901F6
:106BE000A60195010E945772DC01CB0180935703E7
:106BF00090935803A0935903B0935A03B7FF04C06E
:106C00008150904FAF4FBF4F3C014D01ACE0959488
:106C1000879477946794AA95D1F7609257037092FE
:106C200058038092590390925A03C801B7012D81ED
:106C30003E814F8158850E94577297FF04C0615072
:106C4000784F8F4F9F4FFBE0959587957795679588
:106C5000FA95D1F7A60195010E945772DC01CB018C
:106C600080935B0390935C03A0935D03B0935E03FA
:106C7000B7FF04C08150904FAF4FBF4FAC01BD0173
:106C8000ECE07595679557954795EA95D1F7409350
:106C90005B0350935C0360935D0370935E032989EB
:106CA0003A8937FF03C0309521953F4F2134310594
:106CB000E4F1D401C30197FE07C0B095A09590956B
:106CC00081959F4FAF4FBF4F81389105A105B10509
:106CD00084F4DB01CA0177FF07C0B095A0959095B9
:106CE00081959F4FAF4FBF4F81389105A105B105E9
:106CF000E4F081E08093FB0218C01092C10610926C
:106D0000C0061092BD061092BC0610925B03109252
:106D10005C0310925D0310925E0310925703109271
:106D200058031092590310925A0380915B0390917B
:106D30005C03A0915D03B0915E03BC01CD0124E62C
:106D400030E040E050E00E94CB72E0905703F090BA
:106D50005803E21AF30AF0923F07E0923E0780914F
:106D6000570390915803A0915903B0915A03BC0165
:106D7000CD0124E630E040E050E00E94CB72DA0121
:106D8000C90120915B0330915C038C01021B130B42
:106D900010933407009333078091790190917A0121
:106DA000A0917B01B0917C01BC01CD0128E631E0CE
:106DB00040E050E00E94577220918A0730918B0783
:106DC00040918C0750918D072617370748075907C0
:106DD00064F0261B370B480B590B20938A0730931E
:106DE0008B0740938C0750938D0720918A07309131
:106DF0008B0740918C0750918D0757FF0CC0260FD1
:106E0000371F481F591F20938A0730938B074093E1
:106E10008C0750938D0760913107709132076E0D8A
:106E20007F1D9B01442737FD4095542F80910F0310
:106E300090911003A0911103B0911203820F931F40
:106E4000A41FB51F80930F0390931003A093110309
:106E5000B09312038091DB029091DC02681B790BE6
:106E6000CB01AA2797FDA095BA2F29853A854B8596
:106E70005C85820F931FA41FB51F8093130390930B
:106E80001403A0931503B0931603C0909501D090FE
:106E90009601E0909701F0909801C816D906EA068D
:106EA000FB06C4F488EA91E6A0E0B0E08C199D09E5
:106EB000AE09BF098093130390931403A0931503A5
:106EC000B093160380930F0390931003A0931103C4
:106ED000B093120322273327A9012C193D094E092B
:106EE0005F098091130390911403A0911503B09151
:106EF000160382179307A407B507B4F4D701C60198
:106F0000885A9146A040B040809313039093140395
:106F1000A0931503B093160380930F03909310036F
:106F2000A0931103B0931203609140077091410741
:106F3000600F711F9B01442737FD4095542F8091AE
:106F4000170390911803A0911903B0911A03820FAF
:106F5000931FA41FB51F8093170390931803A0934A
:106F60001903B0931A038091D9029091DA02681B39
:106F7000790BCB01AA2797FDA095BA2F2D853E85C9
:106F80004F855889820F931FA41FB51F80931B0341
:106F900090931C03A0931D03B0931E03E0909901EE
:106FA000F0909A0100919B0110919C01E816F9065E
:106FB0000A071B07C4F488EA91E6A0E0B0E08E1946
:106FC0009F09A00BB10B80931B0390931C03A0930C
:106FD0001D03B0931E038093170390931803A0938F
:106FE0001903B0931A0322273327A9012E193F0949
:106FF000400B510B80911B0390911C03A0911D032A
:10700000B0911E0382179307A407B507B4F4D80103
:10701000C701885A9146A040B04080931B039093CB
:107020001C03A0931D03B0931E038093170390933A
:107030001803A0931903B0931A0380910B03909146
:107040000C03A0910D03B0910E0380931F03909346
:107050002003A0932103B093220380911B039091FE
:107060001C03A0911D03B0911E0380933B039093DA
:107070003C03A0933D03B0933E0380911303909192
:107080001403A0911503B0911603809333039093DA
:107090003403A0933503B093360380911703909186
:1070A0001803A0911903B0911A03809337039093AA
:1070B0003803A0933903B0933A0380910F03909162
:1070C0001003A0911103B091120380932F039093AA
:1070D0003003A0933103B093320380912301909148
:1070E000240197FD079633E0959587953A95E1F74A
:1070F0009093410780934007809121019091220154
:1071000097FD079623E0959587952A95E1F790934B
:1071100032078093310780912502909126020F97C4
:1071200034F488E19CEF909341078093400780916D
:10713000250290912602079734F480E398EF90930C
:10714000410780934007209102012A30A9F48091E1
:10715000250290912602835F934034F088EE93E0FD
:1071600090934107809340078091250290912602D9
:107170008A5F9340DCF014C0809125029091260232
:10718000815D974034F088EE93E0909341078093BF
:1071900040078091250290912602805E974034F04E
:1071A00080ED97E090934107809340078091230200
:1071B000909124020F9734F488E19CEF909332076A
:1071C000809331078091230290912402079734F431
:1071D00080E398EF90933207809331072A30A9F427
:1071E0008091230290912402835F934034F088EED3
:1071F00093E090933207809331078091230290911E
:1072000024028A5F9340DCF014C0809123029091A5
:107210002402815D974034F088EE93E0909332072A
:10722000809331078091230290912402805E9740E1
:1072300034F080ED97E09093320780933107E0912E
:107240008C01EE2309F4B7C0409123015091240131
:107250008091670390916803481B590B50936E030C
:1072600040936D032091230130912401280F391F91
:1072700037FF02C02F5F3F4F359527953093680346
:1072800020936703413851051CF080E890E005C069
:1072900040585F4F34F480E89FEF90936E038093E3
:1072A0006D038E2F9927A0916D03B0916E03A89F57
:1072B000A001A99F500DB89F500D112457FF02C087
:1072C000415F5F4F84E0559547958A95E1F780913E
:1072D000400790914107840F951F90934107809339
:1072E0004007609121017091220180916903909182
:1072F0006A03681B790B70936C0360936B03409176
:10730000210150912201480F591F57FF02C04F5FC2
:107310005F4F5595479550936A03409369036138D1
:1073200071051CF080E890E005C060587F4F34F490
:1073300080E89FEF90936C0380936B032E2F33278D
:1073400080916B0390916C03829FB001839F700DBD
:10735000929F700D1124AB0177FF02C0415F5F4F18
:1073600014E0559547951A95E1F780913107909172
:107370003207840F951F9093320780933107A29FA5
:10738000C001A39F900DB29F900D11249C0180918C
:10739000230190912401820F931F909324018093E5
:1073A00023018091210190912201860F971F9093D4
:1073B000220180932101009143071091440780919D
:1073C000BC069091BD06101611065CF59C0197FF56
:1073D00004C022273327281B390BC901AA2797FD90
:1073E000A095BA2F20918001332744275527BC014F
:1073F000CD010E9457729B01AC0197FF04C0215C34
:107400003F4F4F4F5F4FF6E055954795379527957E
:10741000FA95D1F780913E0790913F07820F931F15
:1074200027C097FF03C0909581959F4FAA2797FD8E
:10743000A095BA2F20918001332744275527BC01FE
:10744000CD010E9457729B01AC0197FF04C0215CE3
:107450003F4F4F4F5F4FE6E055954795379527953E
:10746000EA95D1F780913E0790913F07821B930BDD
:1074700090933F0780933E07E0904D07F0904E07B2
:107480008091C0069091C1061E141F045CF59C01FA
:1074900097FF04C022273327281B390BC901AA27CD
:1074A00097FDA095BA2F20918001332744275527B7
:1074B000BC01CD010E9457729B01AC0197FF04C033
:1074C000215C3F4F4F4F5F4F76E05595479537957D
:1074D00027957A95D1F78091330790913407820FE1
:1074E000931F27C097FF03C0909581959F4FAA27B0
:1074F00097FDA095BA2F2091800133274427552767
:10750000BC01CD010E9457729B01AC0197FF04C0E2
:10751000215C3F4F4F4F5F4F66E05595479537953C
:1075200027956A95D1F78091330790913407821B94
:10753000930B90933407809333078091CF0687FF96
:1075400044C09B89992309F040C08091D7028823C9
:10755000E1F5A1E0EA16A1E0FA064CF080914007BF
:10756000909141078E0D9F1D805091400DC0B0E05D
:10757000EB16BFEFFB0664F4809140079091410742
:107580008E0D9F1D80509F4F909341078093400721
:10759000E1E001301E074CF08091310790913207F5
:1075A000800F911F805091400CC0FFEF00301F07EB
:1075B00064F48091310790913207800F911F8050C1
:1075C0009F4F9093320780933107A0EFB2E067ECB2
:1075D00076E057E0FB018191BF01E82FFF27EE0F16
:1075E000FF1FEC5AF94F0190F081E02DE259FF4F57
:1075F000EF3FF10521F01CF0EFEFF0E004C0F7FFE2
:1076000002C0E0E0F0E04C91242F3327E217F307AB
:10761000B1F0CF01821B930B97FD079633E0959550
:1076200087953A95E1F7242F280F2C93822F9927DD
:10763000E817F90714F4215001C02F5F2C93515023
:10764000119657FFC7CFE2E1CD5E0C940273CF9342
:10765000DF93809102018D3011F40E94921C1092F0
:107660007A008091250290912602909341078093A1
:1076700040078091230290912402909332078093D7
:107680003107809121029091220290938407809388
:10769000830780911D0290911E029C01442737FDB3
:1076A0004095542FDA01C90172E0880F991FAA1F73
:1076B000BB1F7A95D1F7820F931FA41FB51F820FAE
:1076C000931FA41FB51F90937F0780937E0780911F
:1076D0001F02909120029C01442737FD4095542FB2
:1076E000DA01C90162E0880F991FAA1FBB1F6A95C2
:1076F000D1F7820F931FA41FB51F820F931FA41FE2
:10770000B51F90938F0780938E0780911B029091F5
:107710001C0290934C0780934B078FEC80937A0068
:10772000A0EFB2E0C7ECD6E097E08991E82FFF2701
:10773000EE0FFF1FEC5AF94F0190F081E02DE25956
:10774000FF4F1E161F061CF0E0E0F0E005C0EF3F03
:10775000F10514F0EFEFF0E08C91282F3327E217BA
:10776000F30714F4815004C02E173F0714F48F5F01
:107770008C939150119697FFD8CF8091000799274D
:10778000AA27BB27BC01CD0124EC39E040E050E042
:107790000E945772DC01CB018093990190939A016A
:1077A000A0939B01B0939C01809101079927AA2780
:1077B000BB27BC01CD010E945772DC01CB01809335
:1077C000950190939601A0939701B0939801DF9152
:1077D000CF910895A0E0B0E0E0EFFBE30C94EA72F3
:1077E000C0E0D0E07E016E01469AD0934A03C09378
:1077F0004903D0934803C093470380E090E0A0E0A2
:10780000B0E08093410390934203A0934303B0936D
:107810004403D0935403C0935303D0935203C093B3
:107820005103D0935003C0934F03D0935F07C0938D
:107830005E071092820110928101109215020E943F
:10784000273B84E690E00E9403180E94273B80912A
:10785000CF0680FF10C080911B0190911C01875BB7
:10786000934038F480911B0190911C018E5E9240F0
:1078700010F40E94311C1FE18AE090E00E9403187E
:107880008091210290912202C80FD91F8091250278
:1078900090912602E80EF91E809123029091240215
:1078A000C80ED91E115017FFE7CFA701405F5F4FE9
:1078B00056954795569547955093540340935303D7
:1078C0009601205F3F4F3695279536952795309343
:1078D000520320935103CE01409615E0969587956B
:1078E0001A95E1F79093500380934F0390935F07AD
:1078F00080935E0730934E0320934D0350934C03C7
:1079000040934B03F999FECF84E090E092BD81BD96
:10791000F89A80B5853058F180918E0790918F0745
:1079200097FF03C0909581959F4F6CE070E00E9497
:107930009672709348036093470380917E079091FD
:107940007F0797FF03C0909581959F4F6CE070E093
:107950000E94967270934A036093490380911606C1
:1079600090911706AA2797FDA095BA2F4CC0F999B8
:10797000FECF84E090E092BD81BDF89A80B5992752
:10798000382F2227F999FECF85E090E092BD81BD86
:10799000F89A80B5280F311D30934A03209349038C
:1079A000F999FECF86E090E092BD81BDF89A80B54E
:1079B0009927382F2227F999FECF87E090E092BDD2
:1079C00081BDF89A80B5280F311D3093480320936C
:1079D0004703F999FECF88E090E092BD81BDF89A07
:1079E00080B59927382F2227F999FECF89E090E0BA
:1079F00092BD81BDF89A80B5280F311DC901AA2713
:107A000097FDA095BA2FBC01CD010E94A371DC01A6
:107A1000CB018093410390934203A0934303B0931F
:107A200044031092410710924007109232071092BF
:107A30003107109284071092830784E690E00E9439
:107A4000031880911D0290911E02AA2797FDA09510
:107A5000BA2F9C01AD01F2E0220F331F441F551FC6
:107A6000FA95D1F7280F391F4A1F5B1F280F391FBE
:107A70004A1F5B1F30937F0720937E0780911F0270
:107A800090912002AA2797FDA095BA2F7C018D0125
:107A9000E2E0EE0CFF1C001F111FEA95D1F7E80E83
:107AA000F91E0A1F1B1FE80EF91E0A1F1B1FF0926A
:107AB0008F07E0928E078091DE06682E7724882457
:107AC0009924C9019C01442737FD4095542FC401D6
:107AD000B3010E9457725B016C0160933B0370938A
:107AE0003C0380933D0390933E039701442737FD69
:107AF0004095542FC401B3010E945772DC01CB01A1
:107B00008093330390933403A0933503B0933603EB
:107B1000A0921703B0921803C0921903D0921A03CF
:107B200080930F0390931003A0931103B09312035B
:107B300010920B0310920C0310920D0310920E037F
:107B400080911D0190911E01A0911F01B091200113
:107B50009093190680931806109214021092130243
:107B6000109203031092040310920503109206036F
:107B70008091010390910203909300038093FF0290
:107B80000E943D5D82E390E09093FF018093FE01AF
:107B9000809100079927AA27BB27BC01CD0124ECBF
:107BA00039E040E050E00E945772DC01CB0188567A
:107BB000954CAF4FBF4F8093990190939A01A0933A
:107BC0009B01B0939C01809101079927AA27BB27AD
:107BD000BC01CD010E945772DC01CB018856954C47
:107BE000AF4FBF4F8093950190939601A09397015B
:107BF000B093980110927E0110927D018091010353
:107C000090910203AA2797FDA095BA2F20917901A0
:107C100030917A0140917B0150917C01BC01CD01F2
:107C20000E945772DC01CB0180938A0790938B07E7
:107C3000A0938C07B0938D071092FA021092F9026C
:107C400081E0809301010E945F618091BE028460A7
:107C50008093BE028FEF8093FB071092FC0780E2B7
:107C60008093FD07C0EFD2E0A7ECB6E017E08D915E
:107C7000E82FFF27EE0FFF1FEC5AF94F808191810B
:107C800082598993115017FFF2CF84E68093EF0257
:107C90008091FC01882311F0469A579AEEE0CDB707
:107CA000DEB70C9406738091E5028823F9F4809185
:107CB000BE028C7F8093BE02A3E2B6E0EAE6F4E067
:107CC0009BE08091DF01882309F4808381918C936C
:107CD0001496915097FFF5CF8091DF01882359F0DA
:107CE0008091DF0181508093DF0105C08091BE0249
:107CF00081608093BE028091230699279093EC05C2
:107D00008093EB058091270699279093EE05809349
:107D1000ED0580912B0699279093F0058093EF0550
:107D200080912F0699279093F2058093F105109288
:107D30004A02109249020E94FA2B08958091D106BE
:107D4000883F38F0EFEFF0E0E81BF109E051FD4F1C
:107D500080818093920180919201882329F084365A
:107D600018F084E6809392018091D306883F38F022
:107D7000EFEFF0E0E81BF109E051FD4F80818093C7
:107D8000900180919001882329F0843618F084E6D0
:107D9000809390018091E006883F38F0EFEFF0E0AB
:107DA000E81BF109E051FD4F808180938B018091A8
:107DB0008B018B3010F48AE002C08F3F11F4809366
:107DC0008B0180910A07883F38F0EFEFF0E0E81B65
:107DD000F109E051FD4F8081809359078091590747
:107DE000823010F481E002C08F3F11F48093590774
:107DF00080910C07883F38F0EFEFF0E0E81BF109C5
:107E0000E051FD4F8081809381078091810782300E
:107E100010F481E002C08F3F11F4809381078091BC
:107E2000F706883F38F0EFEFF0E0E81BF109E0518A
:107E3000FD4F8081809356078091F806883F38F087
:107E4000EFEFF0E0E81BF109E051FD4F80818093F6
:107E5000C2068091F906883F38F0EFEFF0E0E81BAA
:107E6000F109E051FD4F8081809360079091D20627
:107E7000983F18F49093910109C0EFEFF0E0E91BEF
:107E8000F109E051FD4F808180939101983F18F4F2
:107E90009093910109C0EFEFF0E0E91BF109E05187
:107EA000FD4F8081809391018091D506883F38F005
:107EB000EFEFF0E0E81BF109E051FD4F8081809386
:107EC0008F018091D706883F38F0EFEFF0E0E81B94
:107ED000F109E051FD4F808180938D018091DF0693
:107EE000883F38F0EFEFF0E0E81BF109E051FD4F7B
:107EF000808180938E018091E106883F38F0EFEF1A
:107F0000F0E0E81BF109E051FD4F808180938A0188
:107F10008091E206883F38F0EFEFF0E0E81BF109CE
:107F2000E051FD4F808180938C018091E306883F72
:107F300038F0EFEFF0E0E81BF109E051FD4F8081F0
:107F4000809389018091E406883F38F0EFEFF0E0FC
:107F5000E81BF109E051FD4F8081809388018091F9
:107F6000E906883F38F0EFEFF0E0E81BF109E05157
:107F7000FD4F8081809386018091EA06883F38F02A
:107F8000EFEFF0E0E81BF109E051FD4F80818093B5
:107F9000D2028091EB06883F38F0EFEFF0E0E81B6B
:107FA000F109E051FD4F80818093D1028091EC0670
:107FB000883F38F0EFEFF0E0E81BF109E051FD4FAA
:107FC00080818093D0028091ED06883F38F0EFEFFA
:107FD000F0E0E81BF109E051FD4F80818093CF0272
:107FE00080910507883F38F0EFEFF0E0E81BF109DA
:107FF000E051FD4F80818093CE0280910607883F3B
:1080000038F0EFEFF0E0E81BF109E051FD4F80811F
:108010008093CD0280910707883F38F0EFEFF0E0C2
:10802000E81BF109E051FD4F80818093CC028091E3
:108030000807883F38F0EFEFF0E0E81BF109E05166
:10804000FD4F80818093CB028091EE06883F38F00F
:10805000EFEFF0E0E81BF109E051FD4F80818093E4
:1080600085018091F206883F38F0EFEFF0E0E81BE1
:10807000F109E051FD4F8081809384018091FA06DF
:10808000883F38F0EFEFF0E0E81BF109E051FD4FD9
:108090008081809383018091FD06883F38F0EFEF67
:1080A000F0E0E81BF109E051FD4F808180938201EF
:1080B0008091FE06883F38F0EFEFF0E0E81BF10911
:1080C000E051FD4F8081809381018091FF06883FC0
:1080D00038F0EFEFF0E0E81BF109E051FD4F80814F
:1080E0008093800180910407883F38F0EFEFF0E043
:1080F000E81BF109E051FD4F808180937F01809161
:108100001F07883F38F0EFEFF0E0E81BF109E0517E
:10811000FD4F80818093910780918601282F33271E
:108120002F5F3F4F8CE398E2B9010E9496727093E3
:108130009401609393018091DD0680938207809182
:10814000DC06809345070895A4E1B0E0EAEAF0E494
:108150000C94E6728091BD0281508093BD02882309
:1081600019F485E08093BD020E949F323091020194
:108170003C3010F4299A01C02998E090E602F09072
:10818000E702FA82E9828091450799270A96E81664
:10819000F90614F49A8389838091EF02843608F0FB
:1081A0005CC080918B0390918C03009731F0019714
:1081B00090938C0380938B0307C01092E50280910B
:1081C000BE028F7E8093BE023A3011F0343111F43A
:1081D000289A01C028988091BF029091C002895EC0
:1081E0009340C0F18091E606282F33273A832983F4
:1081F0008091BE0280618093BE028091C306A82F49
:10820000BB27AA0FBB1FFD01E857F94F118210824F
:108210008091C406282F3327220F331FC9018857A6
:10822000994FFC0111821082AC5AB94F11961C92E1
:108230001E922C5A394FD90111961C921E92809190
:10824000C606E82FFF27EE0FFF1FEC5AF94F1182E9
:10825000108221C31092E5021EC38091EF028D3877
:1082600008F419C38091BE028F7E8093BE02909164
:10827000E70682E3989FC001112490938C038093BA
:108280008B03E981FA81B9978CF08091E50288230C
:1082900069F08091BF029091C002FFEF8F3F9F076E
:1082A00029F001969093C0028093BF028091BF0293
:1082B0009091C0028F3F910509F038F510926F033D
:1082C0001092700310927103109272031092730354
:1082D0001092740310927503109276038A3F9105F1
:1082E000C9F481E080939103109277031092780390
:1082F0001092790310927A0310920B0310920C03E0
:1083000010920D0310920E0305C08091BE02826090
:108310008093BE028091C506E82FFF27EE0FFF1F56
:10832000EC5AF94F80819181813591050CF4DFC1C0
:108330002091E502222309F0DAC18091C606E82FD8
:10834000FF27EE0FFF1FEC5AF94F808191818C348B
:1083500091050CF404C180918D038F5F80938D0390
:10836000893C08F4C4C13C3010F4299801C0299A12
:108370001092E50210928D031092C0021092BF027B
:108380003091C306E32FFF27EE0FFF1FEC5AF94F82
:108390008081918187349105B4F48091C406E82FDF
:1083A000FF27EE0FFF1FEC5AF94F8081918101905A
:1083B000F081E02DF7FF03C0F095E195FF4FE73422
:1083C000F1050CF478C041E02091C406A22FBB2730
:1083D000AA0FBB1FAC5AB94F8D919C91119787344E
:1083E000910544F0E32FFF27EE0FFF1FEC5AF94FE2
:1083F000808191818D919C918734910574F0809159
:10840000C306E82FFF27EE0FFF1FEC5AF94F8081BC
:108410009181873491050CF042E0E22FFF27EE0FA7
:10842000FF1FEC5AF94F808191818634910574F4D5
:108430008091C306E82FFF27EE0FFF1FEC5AF94F7C
:1084400080819181873491050CF043E0E22FFF2772
:10845000EE0FFF1FEC5AF94F808191818A5B9F4F8D
:1084600074F48091C306E82FFF27EE0FFF1FEC5A2C
:10847000F94F80819181873491050CF044E0E22F1F
:10848000FF27EE0FFF1FEC5AF94F808191818A5B25
:108490009F4F74F48091C306E82FFF27EE0FFF1F54
:1084A000EC5AF94F80819181863491050CF445E0B6
:1084B000842F0E9419078091C406E82FFF27EE0F32
:1084C000FF1FEC5AF94F808191810190F081E02DDE
:1084D000F7FF03C0F095E195FF4F7E97BCF48091C4
:1084E000C306E82FFF27EE0FFF1FEC5AF94F8081DC
:1084F00091818A5B9F4F54F481E08093800488EEE1
:1085000093E09093FF018093FE01F1C00E947107F8
:108510004CE663EC76E00E94FC0680E00E94BB071C
:108520000E94E4698091CF0680FF10C080911B01FA
:1085300090911C01875B934038F480911B019091CE
:108540001C018E5E924010F40E94311C1092FC01BE
:108550000E94EA3B81E08093FC01579ABFC0808172
:108560009181855B9F4F0CF0C0C080918D038F5F20
:1085700080938D03893C08F4BAC03C3010F42998EC
:1085800001C0299A8FB399279C012270307081FD18
:10859000F9CF1FBA84E090E092BD81BD8FEF80BD1E
:1085A0000FB6F894FA9AF99A0FBE1092E50210925B
:1085B0008D033093C0022093BF020E94EA3B2091BA
:1085C000490330914A03C90137FF02C081509F4FD0
:1085D000892F990F990B482FF999FECF1FBA84E084
:1085E00090E092BD81BD40BD0FB6F894FA9AF99A19
:1085F0000FBEF999FECF1FBA85E090E092BD81BD14
:1086000020BD0FB6F894FA9AF99A0FBE209147034D
:1086100030914803C90137FF02C081509F4F892F15
:10862000990F990B482FF999FECF1FBA86E090E079
:1086300092BD81BD40BD0FB6F894FA9AF99A0FBE6B
:10864000F999FECF1FBA87E090E092BD81BD20BDB1
:108650000FB6F894FA9AF99A0FBE8091410390915F
:108660004203A0914303B0914403BC01CD010E9499
:108670007071DC01CB019C0197FF02C021503F4F7C
:10868000832F992787FD9A95282FF999FECF1FBA36
:1086900088E090E092BD81BD20BD0FB6F894FA9AB3
:1086A000F99A0FBE8091410390914203A091430338
:1086B000B0914403BC01CD010E947071DC01CB017B
:1086C000282FF999FECF1FBA89E090E092BD81BDB5
:1086D00020BD0FB6F894FA9AF99A0FBE0E9471075E
:1086E00068E770E00E947E3202C020938D03809183
:1086F000C506E82FFF27EE0FFF1FEC5AF94F8081C8
:1087000091818B5A9F4F0CF0C6C02091E502E091F9
:10871000C606222309F0A3C0FF27EE0FFF1FEC5A65
:10872000F94F80819181855B9F4F0CF095C08091BE
:108730008E038F5F80938E03893C08F4ACC0209336
:108740008E0381E090E09093C0028093BF0281E0AD
:108750008093E502109277031092780310927903C8
:1087600010927A0310920B0310920C0310920D03D7
:1087700010920E031092070310920803109209033F
:1087800010920A038091DE06E82EFF2400271127AD
:1087900080917E0790917F079C01442737FD40958B
:1087A000542FC801B7010E945772DC01CB0180939E
:1087B0001B0390931C03A0931D03B0931E03809191
:1087C0008E0790918F079C01442737FD4095542FC9
:1087D000C801B7010E945772DC01CB0180931303DB
:1087E00090931403A0931503B093160380913B0359
:1087F00090913C03A0913D03B0913E0380931703F9
:1088000090931803A0931903B0931A038091330334
:1088100090913403A0913503B091360380930F03F8
:1088200090931003A0931103B093120310926F035F
:1088300010927003109271031092720310927303DE
:108840001092740310927503109276038091BE0209
:1088500088608093BE021FC020938E031CC0FF2738
:10886000EE0FFF1FEC5AF94F808191818C349105F6
:1088700084F080918F038F5F80938F03893C58F041
:108880001092E50210928F031092C0021092BF0264
:1088900002C010928F0380917801815080937801FB
:1088A000809178018F3F21F08091BE0284FFD5C274
:1088B0000E949E3E80919A0390919B03AC01440FCD
:1088C000551F480F591F0091C306A02FBB27AA0FA1
:1088D000BB1FFD01EC5AF94FF090D906CF2CDD24D7
:1088E000808191818C9DF0018D9DF00D9C9DF00DFE
:1088F00011244E0F5F1F57FF02C04D5F5F4F55950C
:10890000479555954795A857B94F8091DA06682F36
:1089100077278D919C91869F9001879F300D969F20
:10892000300D1124420F531F50939B0340939A0321
:108930008091D1039091D2032091CD033091CE0349
:10894000820F931F481B590B5093ED024093EC028A
:1089500080919C0390919D03AC01440F551F480FDB
:10896000591F1091C406A12FBB27AA0FBB1FFD01E1
:10897000EC5AF94F808191818C9DF0018D9DF00D15
:108980009C9DF00D11244E0F5F1F57FF02C04D5FDD
:108990005F4F5595479555954795A857B94F8D9178
:1089A0009C91869F9001879F300D969F300D1124DA
:1089B000420F531F50939D0340939C038091CF031C
:1089C0009091D0032091CB033091CC03820F931F61
:1089D000481B590B5093EB024093EA028091C60664
:1089E000E82FFF27EE0FFF1FEC5AF94F808191818E
:1089F000909581959F4F9093E9028093E802833090
:108A0000910514F0029705C03FEF8E3F930734F4B1
:108A100002969093E9028093E80204C01092E90262
:108A20001092E8028091C506E82FFF27EE0FFF1F86
:108A3000EC5AF94FC080D18048E750E0C40ED51EF3
:108A4000D092E702C092E60280918B019927AA2773
:108A500097FDA095BA2FBC01CD010E94A371DC0146
:108A6000CB0120E030E040E251E4BC01CD010E94A6
:108A70000871DC01CB01BC01CD010E947571DC01E4
:108A8000CB018093880780918A0180936107809150
:108A900089019927AA2797FDA095BA2FBC01CD017E
:108AA0000E94A371DC01CB0120E030E040E251E400
:108AB000BC01CD010E940871DC01CB01BC01CD01DC
:108AC0000E947571DC01CB01809338078091880189
:108AD00080934F0780918C0480FF61C08091910743
:108AE000813808F45CC080918504992787FD9095B2
:108AF0004F2D5527849F9001859F300D949F300DF9
:108B000011248091EC029091ED02820F931F9093BB
:108B1000ED028093EC0280918604992787FD909561
:108B2000849F9001859F300D949F300D112480917A
:108B3000EA029091EB02820F931F9093EB028093D5
:108B4000EA0280918704282F332727FD30958091F2
:108B5000E8029091E902820F931F9093E9028093BB
:108B6000E80280918904282F332727FD30958091D2
:108B7000D4069927289FB001299F700D389F700D4A
:108B8000112470937E0160937D0180918804992760
:108B90008C159D0524F49093E7028093E602809162
:108BA000E6029091E70297FF04C01092E70210924C
:108BB000E6028091CF0682FF02C0109261074091C9
:108BC000EC025091ED02CA0157FD03969C013595C8
:108BD00027953595279537FF03C0309521953F4F51
:108BE0008091C3029091C40282179307B4F4CA0122
:108BF00057FF03C0909581959F4F97FD03969595DC
:108C00008795959587959093C4028093C302853686
:108C1000910544F084E690E001C001979093C4026E
:108C20008093C3024091EA025091EB02CA0157FDC2
:108C300003969C01359527953595279537FF03C0F9
:108C4000309521953F4F8091C1029091C2028217C9
:108C50009307B4F4CA0157FF03C0909581959F4FC5
:108C600097FD039695958795959587959093C20264
:108C70008093C1028536910544F084E690E001C0FE
:108C800001979093C2028093C1028091BE0284FF3B
:108C900008C01092C4021092C3021092C202109235
:108CA000C102E12FFF27EE0FFF1FEC5AF94F409151
:108CB000FB06242F3327808191812817390744F43C
:108CC0008091200782FF04C081E08093D60213C008
:108CD000E12FFF27EE0FFF1FEC5AF94F842F992742
:108CE0002091FC06821B91092081318128173907C8
:108CF00014F41092D6024091C406E42FFF27EE0F21
:108D0000FF1FEC5AF94F5091FB06852F9927222718
:108D10003327281B390B808191818217930744F4F4
:108D20008091200783FF04C081E08093D50216C0A4
:108D30008091D502882391F0E42FFF27EE0FFF1FCB
:108D4000EC5AF94F8091FC069927851B91092081E7
:108D500031818217930714F41092D502E02FFF2778
:108D6000EE0FFF1FEC5AF94F4091FB06242F3327DB
:108D7000808191812817390744F48091200780FF72
:108D800004C081E08093D30217C08091D30288236E
:108D900099F0E02FFF27EE0FFF1FEC5AF94F842FB9
:108DA00099272091FC06821B910920813181281787
:108DB000390714F41092D3024091C306E42FFF2721
:108DC000EE0FFF1FEC5AF94F5091FB06852F9927A4
:108DD00022273327281B390B808191818217930723
:108DE00044F48091200781FF04C081E08093D40285
:108DF00016C08091D402882391F0E42FFF27EE0F54
:108E0000FF1FEC5AF94F8091FC069927851B9109A9
:108E1000208131818217930714F41092D40280913B
:108E2000D602882319F48091D502811181E08093C4
:108E3000D7028091D302882321F48091D402882321
:108E400051F081E08093D8021092D7021092D6029E
:108E50001092D50202C08093D8028091D702882355
:108E600021F48091D802882369F08091FA0699272D
:108E7000A981BA818A179B0714F49A83898381E0B8
:108E80008093FB028091BE0284FF1AC01092E90217
:108E90001092E8021092ED021092EC021092EB0296
:108EA0001092EA029AE59093880788E78093610719
:108EB0009093380780934F071092D7021092D802F0
:108EC0008091520790915307A0915407B091550794
:108ED00020913B0330913C0340913D0350913E0370
:108EE000820F931FA41FB51F8093520790935307BF
:108EF000A0935407B093550780915A0790915B0750
:108F0000A0915C07B0915D0720903303309034034B
:108F10004090350350903603820D931DA41DB51D5E
:108F200080935A0790935B07A0935C07B0935D070B
:108F30008091470790914807A0914907B0914A074F
:108F4000E0903703F09038030091390310913A0311
:108F5000EB82FC820D831E838E0D9F1DA01FB11F0F
:108F60008093470790934807A0934907B0934A0717
:108F70008091390790913A07A0913B07B0913C0747
:108F8000E0902F03F09030030091310310913203F1
:108F9000EF82F88609871A878E0D9F1DA01FB11FCB
:108FA0008093390790933A07A0933B07B0933C070F
:108FB000F090D802FB86FF2029F48091D702882305
:108FC00009F460C010922B0310922C0310922D0311
:108FD00010922E0310922703109228031092290357
:108FE00010922A03109252071092530710925407BE
:108FF0001092550710925A0710925B0710925C0767
:1090000010925D0710924707109248071092490787
:1090100010924A071092390710923A0710923B07B4
:1090200010923C0780911B0390911C03A0911D039B
:10903000B0911E038093170390931803A093190314
:10904000B0931A038091130390911403A091150318
:10905000B091160380930F0390931003A093110314
:10906000B093120310921202109211021092DA02BF
:109070001092D9021092DC021092DB020B850023C1
:1090800009F0F2C18091D702882309F0EDC18091E7
:10909000160690911706815092402CF48091E502BB
:1090A000882309F4E1C19090FB07A090DE0660914F
:1090B0007E0770917F077C8B6B8B80918E079091E0
:1090C0008F079A8B898B9FEF991609F4D9C0BB241F
:1090D000CC24DD24CA01B901A60195010E94CB72FE
:1090E00079018A01EB89FC89CF01AA2797FDA09518
:1090F000BA2FE81AF90A0A0B1B0BC201B101A6012B
:1091000095010E94CB7259016A0129893A89C901E6
:10911000AA2797FDA095BA2FA81AB90ACA0ADB0A8E
:10912000292C332427FC3094432C532CC801B7013D
:10913000A20191010E94577297FF04C061507E4FB7
:109140008F4F9F4F3B014C0109E095948794779492
:1091500067940A95D1F7C601B501A20191010E9459
:10916000577297FF04C061507E4F8F4F9F4F5B0136
:109170006C0119E0D594C794B794A7941A95D1F7C8
:109180008091C3029091C402813491053CF4809196
:10919000C1029091C20281349105D4F0D401C3017F
:1091A00097FE03C00196A11DB11D3C014D01959490
:1091B000879477946794D601C501D7FE03C00196C2
:1091C000A11DB11D5C016D01D594C794B794A794FE
:1091D0008091C606E82FFF27EE0FFF1FEC5AF94FCC
:1091E000808191810190F081E02DF7FF03C0F0951F
:1091F000E195FF4F7A97A4F0C401B30123E030E07A
:1092000040E050E00E94CB7239014A01C601B5012D
:1092100023E030E040E050E00E94CB7259016A0147
:109220008091FD07282F332727FD3095432F532F9B
:10923000261537054805590514F439014A019927BF
:1092400087FD9095909581959F4FAA2797FDA095B2
:10925000BA2F681679068A069B0614F43C014D0164
:109260002A153B054C055D0514F459016A01A81641
:10927000B906CA06DB060CF0CFC05C016D01CCC09C
:10928000EA2CFF2400271127CA01B901A801970180
:109290000E94CB7239014A014B895C89CA01AA2715
:1092A00097FDA095BA2F681A790A8A0A9B0AC2010B
:1092B000B101A80197010E94CB7259016A01698925
:1092C0007A89CB01AA2797FDA095BA2FA81AB90AC7
:1092D000CA0ADB0AD401C30197FE03C00F96A11D81
:1092E000B11D3C014D01F4E0959487947794679407
:1092F000FA95D1F7D601C501D7FE03C00F96A11D7F
:10930000B11D5C016D01E4E0D594C794B794A794B6
:10931000EA95D1F78091C3029091C40281349105FE
:109320003CF48091C1029091C20281349105A4F075
:10933000C401B30123E030E040E050E00E94CB7272
:1093400039014A01C601B50123E030E040E050E0B8
:109350000E94CB7259016A018091C606E82FFF274F
:10936000EE0FFF1FEC5AF94F808191810190F0813F
:10937000E02DF7FF03C0F095E195FF4F7A97A4F039
:10938000C401B30123E030E040E050E00E94CB7222
:1093900039014A01C601B50123E030E040E050E068
:1093A0000E94CB7259016A0171E26716710481044F
:1093B00091042CF070E2672E712C812C912C80EEA0
:1093C00068168FEF78068FEF88068FEF980644F4C3
:1093D00060EE662E6FEF762E6FEF862E6FEF962E75
:1093E00091E2A916B104C104D1042CF050E2A52EDB
:1093F000B12CC12CD12CA0EEAA16AFEFBA06AFEF5C
:10940000CA06AFEFDA0644F440EEA42E4FEFB42EB6
:109410004FEFC42E4FEFD42E80911B0390911C036D
:10942000A0911D03B0911E0386199709A809B909D7
:1094300080931B0390931C03A0931D03B0931E0302
:109440008091130390911403A0911503B09116031A
:109450008A199B09AC09BD098093130390931403E7
:10946000A0931503B09316038091110290911202FC
:109470008F3F910509F008F4DEC5BB85BB2309F0D9
:1094800068C58091D702882309F063C58091FB02EB
:10949000882309F05EC5E0910307EC87EE2309F409
:1094A00058C58091520790915307A0915407B091ED
:1094B0005507B7FF04C081509F4FAF4FBF4FE92EF4
:1094C000FA2E0B2F112707FD1A95E0925207F09202
:1094D0005307009354071093550780915A079091B2
:1094E0005B07A0915C07B0915D07B7FF04C0815096
:1094F0009F4FAF4FBF4F892F9A2FAB2FBB27A7FD91
:10950000BA958D879E87AF87B88B80935A079093C3
:109510005B07A0935C07B0935D078091DE06A82EE1
:10952000BB24CC24DD2420912B0330912C034091CB
:109530002D0350912E03C601B5010E94577297FF6B
:1095400004C061507F4F8F4F9F4F672E782E892E1A
:10955000992487FC9A9460922B0370922C0380923A
:109560002D0390922E0320912703309128034091E0
:10957000290350912A03C601B5010E94577297FF33
:1095800004C061507F4F8F4F9F4F272E382E492E9A
:10959000552447FC5A942092270330922803409286
:1095A000290350922A038091230390912403A091D0
:1095B0002503B0912603B7FF04C081509F4FAF4FE2
:1095C000BF4F892F9A2FAB2FBB27A7FDBA9580934A
:1095D000230390932403A0932503B0932603D8017B
:1095E000C70186199709A809B90980938303909345
:1095F0008403A0938503B093860320910207E22E93
:10960000FF2400271127BC01CD01A80197010E946A
:10961000CB7259016A0120939203309393034093D4
:109620009403509395038D859E85AF85B8898219E3
:109630009309A409B5098093870390938803A093A5
:109640008903B0938A03BC01CD01A80197010E9450
:10965000CB722093960330939703409398035093D3
:109660009903D601C501D7FE04C081509F4FAF4F6B
:10967000BF4F892F9A2FAB2FBB27A7FDBA95909389
:10968000DA028093D90257FF04C021503F4F4F4F59
:109690005F4FBB2757FDBA95A52F942F832F90932B
:1096A000DC028093DB028091C3029091C40281347A
:1096B0009105DCF48091C1029091C2028134910540
:1096C000A4F48091C606E82FFF27EE0FFF1FEC5A87
:1096D000F94F808191810190F081E02DF7FF03C067
:1096E000F095E195FF4F7A97E4F08091FB078F3F6B
:1096F000C1F48091D9029091DA0297FD0196959577
:1097000087959093DA028093D9028091DB02909141
:10971000DC0297FD0196959587959093DC028093E6
:10972000DB028091470790914807A0914907B091CB
:109730004A07B7FF04C081509F4FAF4FBF4F892FDB
:109740009A2FAB2FBB27A7FDBA958093470790931D
:109750004807A0934907B0934A0780913907909131
:109760003A07A0913B07B0913C07B7FF04C0815076
:109770009F4FAF4FBF4F892F9A2FAB2FBB27A7FD0E
:10978000BA958093390790933A07A0933B07B0931B
:109790003C0780913B0390913C03A0913D03B09125
:1097A0003E032B813C814D815E81281B390B4A0B86
:1097B0005B0B20937B0330937C0340937D0350939A
:1097C0007E038091330390913403A0913503B091CF
:1097D0003603EF80F88409851A85E81AF90A0A0B1E
:1097E0001B0BE0927F03F0928003009381031093A0
:1097F0008203209383033093840340938503509323
:109800008603E0928703F092880300938903109304
:109810008A038091170390911803A0911903B091C6
:109820001A03821B930BA40BB50B80931703909321
:109830001803A0931903B0931A0380910F0390911A
:109840001003A0911103B09112038E199F09A00B70
:10985000B10B80930F0390931003A0931103B09367
:109860001203FC85FF2371F12091F9023091FA0275
:109870002138310594F080914F0390915003019667
:109880009093500380934F0380915E0790915F0700
:10989000019690935F0780935E0720583F4F94F4A2
:1098A00080914F03909150030197909350038093C0
:1098B0004F0380915E0790915F07019790935F0738
:1098C00080935E071092FA021092F90281E090E014
:1098D00090939F0380939E03E0908303F090840312
:1098E0000091850310918603D801C70117FF07C0B7
:1098F00088279927DC018E199F09A00BB10B815095
:109900009240A040B04034F084E090E090939F03F8
:1099100080939E038091A4039091A503A091A60338
:10992000B091A703209152073091530740915407FB
:1099300050915507821B930BA40BB50B815E914B85
:10994000AF4FBF4F8F539C49A040B04028F080914B
:10995000FC0789310CF4FFC041E0E41640E1F40655
:1099600040E0040740E014070CF473C08091A003AA
:10997000882309F46AC0D801C70117FF07C08827E8
:109980009927DC018E199F09A00BB10B9C01AD0139
:10999000B7FF04C021503E4F4F4F5F4FF9E0559540
:1099A000479537952795FA95D1F780919E03909129
:1099B0009F03820F931F90939F0380939E03D80170
:1099C000C70117FF03C00796A11DB11DE3E0B595C0
:1099D000A79597958795EA95D1F7809392039093F1
:1099E0009303A0939403B093950389589341A040A7
:1099F000B04064F088E893E1A0E0B0E08093920387
:109A000090939303A0939403B093950320919203B2
:109A100030919303409194035091950357FF04C0F4
:109A200021503F4F4F4F5F4F232F342F452F552746
:109A300047FD5A958091D9029091DA02820F931FC7
:109A40009093DA028093D90206C081E08093A0034C
:109A500002C01092A00360E0E61660EFF6066FEF1A
:109A600006076FEF16070CF073C08091A1038823DF
:109A700009F46AC0D801C70117FF07C088279927D2
:109A8000DC018E199F09A00BB10B9C01AD01B7FF42
:109A900004C021503E4F4F4F5F4F69E055954795A9
:109AA000379527956A95D1F780919E0390919F03F2
:109AB000820F931F90939F0380939E03D801C70149
:109AC00017FF03C00796A11DB11D23E0B595A7950B
:109AD000979587952A95D1F7809392039093930356
:109AE000A0939403B093950388579C4EAF4FBF4FFC
:109AF00064F488E79CEEAFEFBFEF809392039093FE
:109B00009303A0939403B093950320919203309113
:109B10009303409194035091950357FF04C0215043
:109B20003F4F4F4F5F4F232F342F452F552747FD72
:109B30005A958091D9029091DA02820F931F9093E7
:109B4000DA028093D90211C081E08093A1030DC095
:109B50001092A1030AC010929F0310929E0388EEF8
:109B600093E090939E0180939D018C85282F33274D
:109B700080919E0390919F032817390724F4309316
:109B80009F0320939E031091FC07112379F0212F4E
:109B9000332727FD309580919E0390919F032817CE
:109BA000390724F430939F0320939E03409183034D
:109BB000509184036091850370918603413851056B
:109BC0006105710574F080915303909154032091C5
:109BD0009E0330919F03820F931F909354038093B1
:109BE000530340585F4F6F4F7F4F74F4809153037E
:109BF0009091540320919E0330919F03821B930BFD
:109C0000909354038093530381E090E090939F03DB
:109C100080939E03C0908703D0908803E0908903CF
:109C2000F0908A03D701C601F7FE07C0882799275D
:109C3000DC018C199D09AE09BF0981509240A040FA
:109C4000B04034F084E090E090939F0380939E03B3
:109C50001092960310929703109298031092990312
:109C60008091A8039091A903A091AA03B091AB039E
:109C700020915A0730915B0740915C0750915D0736
:109C8000821B930BA40BB50B815E914BAF4FBF4F63
:109C90008F539C49A040B04018F019310CF4FFC01C
:109CA00001E0C01600E1D00600E0E00600E0F006AA
:109CB0000CF473C08091A203882309F46AC0D70111
:109CC000C601F7FE07C088279927DC018C199D097A
:109CD000AE09BF099C01AD01B7FF04C021503E4F42
:109CE0004F4F5F4F09E055954795379527950A9552
:109CF000D1F780919E0390919F03820F931F9093C1
:109D00009F0380939E03D701C601F7FE03C0079609
:109D1000A11DB11D13E0B595A795979587951A9547
:109D2000D1F78093960390939703A0939803B093F1
:109D3000990389589341A040B04064F088E893E1CA
:109D4000A0E0B0E08093960390939703A0939803CC
:109D5000B093990320919603309197034091980313
:109D60005091990357FF04C021503F4F4F4F5F4F11
:109D7000232F342F452F552747FD5A958091DB021D
:109D80009091DC02820F931F9093DC028093DB02A0
:109D900006C081E08093A20302C01092A20320E0DB
:109DA000C21620EFD2062FEFE2062FEFF2060CF0DC
:109DB00073C08091A303882309F46AC0D701C60148
:109DC000F7FE07C088279927DC018C199D09AE0989
:109DD000BF099C01AD01B7FF04C021503E4F4F4F5A
:109DE0005F4FE9E05595479537952795EA95D1F767
:109DF00080919E0390919F03820F931F90939F03E6
:109E000080939E03D701C601F7FE03C00796A11DEC
:109E1000B11D73E0B595A795979587957A95D1F77C
:109E20008093960390939703A0939803B09399031C
:109E300088579C4EAF4FBF4F64F488E79CEEAFEF5E
:109E4000BFEF8093960390939703A0939803B093EA
:109E50009903209196033091970340919803509174
:109E6000990357FF04C021503F4F4F4F5F4F232F9F
:109E7000342F452F552747FD5A958091DB0290914D
:109E8000DC02820F931F9093DC028093DB0211C0EF
:109E900081E08093A3030DC01092A3030AC0109227
:109EA0009F0310929E0388EE93E090939E0180930F
:109EB0009D014C85242F332780919E0390919F0311
:109EC0002817390724F430939F0320939E03809131
:109ED000FC07882379F0282F332727FD30958091C0
:109EE0009E0390919F032817390724F430939F0312
:109EF00020939E03409187035091880360918903CA
:109F000070918A03413851056105710574F08091A3
:109F100051039091520320919E0330919F03820F31
:109F2000931F909352038093510340585F4F6F4F9C
:109F30007F4FCCF4809151039091520320919E0366
:109F400030919F03821B930B909352038093510394
:109F50000AC01092DC021092DB021092DA02109218
:109F6000D9021092FB0280916107882341F410927C
:109F7000DC021092DB021092DA021092D902809178
:109F8000520790915307A0915407B09155078093C1
:109F9000A4039093A503A093A603B093A703809175
:109FA0005A0790915B07A0915C07B0915D07809381
:109FB000A8039093A903A093AA03B093AB031092B4
:109FC0002B0310922C0310922D0310922E0310924B
:109FD0002703109228031092290310922A0310924B
:109FE000230310922403109225031092260310924B
:109FF000520710925307109254071092550710926F
:10A000005A0710925B0710925C0710925D0710923E
:10A010004707109248071092490710924A0710927A
:10A02000390710923A0710923B0710923C071092A2
:10A03000120210921102E090E802F090E902C701CA
:10A04000F7FE04C0882799278E199F0940976CF066
:10A0500088EE93E090939E0180939D018091CF06BE
:10A0600084FD03C081E0809391031091DB06A12E53
:10A07000BB24CC24DD24B701882777FD8095982F59
:10A080009701F7FE04C0222733272E193F094427E2
:10A0900037FD4095542F0E9457729B01AC01C601B9
:10A0A000B5010E94577297FF04C061507E4F8F4FD9
:10A0B0009F4F59E095958795779567955A95D1F774
:10A0C0009B01812F99278E9DD0018F9DB00D9E9D64
:10A0D000B00D1124CD01B7FD039695958795959503
:10A0E0008795280F391F442737FD4095542F20931B
:10A0F0007703309378034093790350937A038091E8
:10A100000B0390910C03A0910D03B0910E03821BE1
:10A11000930BA40BB50B80930B0390930C03A093AC
:10A120000D03B0930E038155934CA040B04064F0F2
:10A1300080E593ECA0E0B0E080930B0390930C03D8
:10A14000A0930D03B0930E0380910B0390910C0329
:10A15000A0910D03B0910E03805B9C43AF4FBF4FA6
:10A1600064F480EB9CE3AFEFBFEF80930B0390931D
:10A170000C03A0930D03B0930E0340900103509085
:10A1800002034114510409F488C18091CF0683FF72
:10A1900084C180913B0390913C03A0913D03B09119
:10A1A0003E03B7FF04C081509E4FAF4FBF4F09E041
:10A1B000B595A795979587950A95D1F76C0197FF67
:10A1C00004C0D094C194D108D3948091330390916A
:10A1D0003403A0913503B0913603B7FF04C081501A
:10A1E0009E4FAF4FBF4F19E0B595A79597958795AF
:10A1F0001A95D1F7BC0197FF03C0709561957F4F09
:10A20000C616D7060CF46B01B601D7FE02C0695F13
:10A210007F4F3B01B3E075946794BA95E1F70894DA
:10A22000611C711CACE1EA2EA2E0FA2E4E0C5F1C00
:10A2300072010027F7FC0095102F24EE3DEF420E2F
:10A24000531E80918A0790918B07A0918C07B09143
:10A250008D078090790190907A01A0907B01B09059
:10A260007C01BC01CD01A50194010E94CB72E21AD0
:10A27000F30A040B150BC801B70128E631E040E0F2
:10A2800050E00E94CB72DC01CB018C01045B1040DA
:10A29000809183079091840797FF03C090958195E3
:10A2A0009F4F8138910514F000E010E0E0909D018F
:10A2B000F0909E01E114F10489F539E1C316D1044F
:10A2C0006CF58091F9029091FA02800F911F9093A2
:10A2D000FA028093F902809191038823F9F0C20178
:10A2E000AA2797FDA095BA2FBC01CD01A501940125
:10A2F0000E945772DC01CB0180938A0790938B07F1
:10A30000A0938C07B0938D07BC01CD010E94CB7246
:10A31000309300032093FF0210929103C801F3E0F1
:10A32000880F991FFA95E1F7B3010E949672CB014D
:10A33000AA2797FDA095BA2F20918A0730918B0705
:10A3400040918C0750918D07280F391F4A1F5B1FC2
:10A3500020938A0730938B0740938C0750938D0787
:10A3600010918E01612F7727C69EC001C79E900D68
:10A37000D69E900D112497FD4F966C01E5E0D59483
:10A38000C794EA95E1F76C197D096B0177FD7FC0F1
:10A39000E114F10409F073C0E090C302F090C4022C
:10A3A0008091C1029091C202E80EF91EF7FE04C02E
:10A3B00067E070E0E60EF71E63E0F594E7946A95B7
:10A3C000E1F780E490E0E80EF91ECA01B901A501A9
:10A3D00094010E94CB72DA01C9012091FF023091F1
:10A3E0000003442737FD4095542F821B930BA40B89
:10A3F000B50B845E9D4FAF4FBF4FBC01CD0128E62A
:10A4000031E040E050E00E94CB72DC01CB01845B84
:10A4100090408C9DD0018D9DB00D9C9DB00D112460
:10A42000CD01B7010E94967283E0189F600111244C
:10A43000C616D70614F4B60108C0882799278C19C8
:10A440009D09681779070CF4BC019B01442737FD6F
:10A450004095542F80910B0390910C03A0910D0314
:10A46000B0910E03820F931FA41FB51F80930B039F
:10A4700090930C03A0930D03B0930E030EC00894A9
:10A48000E108F108F0929E01E0929D0106C084EF80
:10A4900091E090939E0180939D0180919003815063
:10A4A000809390038F3F09F0DCC088E18093900394
:10A4B0008091DE069927880F991F880F991F7C01CC
:10A4C0000027F7FC0095102F80913B0390913C03EF
:10A4D000A0913D03B0913E03BC01CD01A8019701BD
:10A4E0000E94CB723093D4052093D305809133031F
:10A4F00090913403A0913503B0913603BC01CD0196
:10A50000A80197010E94CB723093D6052093D50500
:10A5100080917E0790917F0797FD0396959587958B
:10A52000959587959093D8058093D70580918E0750
:10A5300090918F0797FD03969595879595958795AB
:10A540009093DA058093D9058091830790918407D1
:10A550009093DC058093DB058091E1029091E2020B
:10A56000A091E302B091E402BC01CD0125E030E00E
:10A5700040E050E00E94CB723093DE052093DD0571
:10A5800080911606909117069093E0058093DF0561
:10A590005092E4054092E3058091250190912601B7
:10A5A0009093E6058093E5058091EF0299279093BB
:10A5B000E8058093E70580918A0790918B07A09129
:10A5C0008C07B0918D072091790130917A014091EB
:10A5D0007B0150917C01BC01CD010E94CB72309374
:10A5E000EA052093E905809113029091140290935B
:10A5F000F8058093F7058091800499279093FA05D8
:10A600008093F9058091FA019091FB019093FC05EC
:10A610008093FB05809100089091010890930006BB
:10A620008093FF058091040890910508909302069D
:10A63000809301068091FE07992790930E068093E0
:10A640000D068091D1039091D203909310068093D0
:10A650000F068091CF039091D003909312068093C0
:10A6600011068091FB02882381F0109273031092EF
:10A670007403109275031092760310926F03109278
:10A6800070031092710310927203F090D802FF20B1
:10A69000F1F480916107282F3327442755278091B3
:10A6A0003B0390913C03A0913D03B0913E03BC015C
:10A6B000CD010E945772DC01CB01BC01CD0128EF16
:10A6C0003AE240E050E00E94CB72490102C0882487
:10A6D0009924E090D702EE20F1F480916107282FB1
:10A6E0003327442755278091330390913403A09159
:10A6F0003503B0913603BC01CD010E945772DC01D5
:10A70000CB01BC01CD0128EF3AE240E050E00E94CD
:10A71000CB72390102C0662477248091330790916F
:10A720003407893C91051CF088EC90E005C0885303
:10A730009F4F34F488E39FEF90933407809333075F
:10A7400080913E0790913F07893C91051CF088EC71
:10A7500090E005C088539F4F34F488E39FEF9093B7
:10A760003F0780933E078091400790914107AA27B9
:10A7700097FDA095BA2F20918807A22EBB24CC2448
:10A78000DD24BC01CD01A60195010E9457729B01F9
:10A79000AC018091330790913407AA2797FDA095CB
:10A7A000BA2F17E0880F991FAA1FBB1F1A95D1F760
:10A7B000280F391F4A1F5B1F57FF04C0215C3F4F02
:10A7C0004F4F5F4FA6E05595479537952795AA952A
:10A7D000D1F78401020F131F109341070093400724
:10A7E0008091310790913207AA2797FDA095BA2F43
:10A7F000BC01CD01A60195010E9457729B01AC01DD
:10A8000080913E0790913F07AA2797FDA095BA2F08
:10A81000F7E0880F991FAA1FBB1FFA95D1F7280FE1
:10A82000391F4A1F5B1F57FF04C0215C3F4F4F4F2A
:10A830005F4FE6E05595479537952795EA95D1F70F
:10A840002301420E531E50923207409231078091ED
:10A85000830790918407880F991FAA2797FDA095D9
:10A86000BA2F20913807332744275527BC01CD0143
:10A870000E9457725B016C0197FF08C02FE330E024
:10A8800040E050E0A20EB31EC41ED51E76E0D59463
:10A89000C794B794A7947A95D1F780914F07282F42
:10A8A00033274427552780911F0390912003A091BF
:10A8B0002103B0912203BC01CD010E945772DC013B
:10A8C000CB01BC01CD0120EF35E540E050E00E9416
:10A8D000CB72B501620F731F709384076093830777
:10A8E0000150104434F080E090E49093410780934D
:10A8F000400780914007909141078050904C34F47C
:10A9000080E090EC909341078093400751E045161A
:10A9100050E4550634F080E090E490933207809341
:10A92000310780913107909132078050904C34F478
:10A9300080E090EC9093320780933107615070442F
:10A9400034F080E090E490938407809383078091B3
:10A950008307909184078050904C34F480E090EC11
:10A96000909384078093830780910001482F552797
:10A9700080912501909126014817590794F4209160
:10A9800025013091260109811A81049FC001059F8C
:10A99000900D149F900D1124B9010E9482727A8348
:10A9A000698329813A81220F331F220F331F3A8393
:10A9B00029834091CF0640FFA0C5EE2009F09DC538
:10A9C000FF2009F09AC58091B0039091B103909354
:10A9D000FE058093FD0580911302909114029093DF
:10A9E000F8058093F7052091550330915603211502
:10A9F000310509F03FC080911B0190911C018959DC
:10AA0000934058F087B5853F20F48091150281501E
:10AA100011C081E08093B9034EC080911B019091D9
:10AA20001C018436910508F587B58B30D0F08091F4
:10AA300015028F5F809315029AE08902900111241C
:10AA400080912006821B87BD8CE291E09093FF01EC
:10AA50008093FE018EE591E0909356038093550319
:10AA60002AC081E08093B80326C0F092B803F09228
:10AA7000B90321C08091E1029091E202A091E3022A
:10AA8000B091E40254E0880F991FAA1FBB1F5A958A
:10AA9000D1F78093160290931702A0931802B093F7
:10AAA0001902109214021092130221503040309378
:10AAB0005603209355032091910141FF24C0223376
:10AAC000D8F48091BE0181508093BE018F3FD9F5AB
:10AAD0001092FC028091E1029091E202A091E302C7
:10AAE000B091E4028093DD029093DE02A093DF0236
:10AAF000B093E00281E004C081E08093FC0288EC26
:10AB00008093BE0120C080917D0190917E01820FD3
:10AB1000911D2091D4063327829FA001839F500D61
:10AB2000929F500D1124CA01AA2797FDA095BA2F14
:10AB30008093DD029093DE02A093DF02B093E002E7
:10AB400081E08093FC0280913B0390913C03A091B3
:10AB50003D03B0913E03E0907901F0907A010091BD
:10AB60007B0110917C01BC01CD01A80197010E94DD
:10AB7000CB7259016A018091330390913403A09103
:10AB80003503B0913603BC01CD01A80197010E94A5
:10AB9000CB72B901C5010E9480707C01CC971CF07A
:10ABA0004CE3E42EF12CC7010E940D657C018091DD
:10ABB000FC02882309F42DC38091BE0299279C01D1
:10ABC0002071307084FD25C36091220760FD04C0B0
:10ABD0008091CF0681FD07C0C980DA803093AD0334
:10ABE0002093AC0356C18091BE0281FF2EC14091DB
:10ABF000BA015091BB01CA010F962091E602309133
:10AC0000E7028217930784F58091B803882361F5E2
:10AC10008091BA0381FF13C08D7F8093BA03809126
:10AC2000E1029091E202A091E302B091E4028093EC
:10AC3000DD029093DE02A093DF02B093E0028091E8
:10AC4000BA0381608093BA03241B350B2F50304028
:10AC500037FF03C0309521953F4F8091AC03909111
:10AC6000AD03820F931F34C0CA010F97281739070D
:10AC7000A4F58091B903882381F58091BA0380FF00
:10AC800013C08E7F8093BA038091E1029091E2021B
:10AC9000A091E302B091E4028093DD029093DE0282
:10ACA000A093DF02B093E0028091BA0382608093A8
:10ACB000BA03241B350B215F3F4F37FF03C030958C
:10ACC00021953F4F8091AC039091AD03821B930B74
:10ACD0009093AD038093AC0327C02091BA03822FD9
:10ACE000992783709070892BF9F02C7F2093BA03F9
:10ACF0001092AD031092AC038091E1029091E202B8
:10AD0000A091E302B091E4028093DD029093DE0211
:10AD1000A093DF02B093E00261FF06C084EF91E0F0
:10AD20009093FF018093FE012091AC033091AD031D
:10AD3000C90137FF04C088279927821B930B8150D4
:10AD400092400CF46BC08091D4069927289FD001C3
:10AD5000299FB00D389FB00D1124CD0160E075E042
:10AD60000E9496729B01442737FD4095542F809195
:10AD7000DD029091DE02A091DF02B091E002820F2D
:10AD8000931FA41FB51F8093DD029093DE02A09352
:10AD9000DF02B093E0021092AD031092AC038091F9
:10ADA000220781FF06C08BE490E09093FF0180931F
:10ADB000FE018091D806882389F54091B003509117
:10ADC000B10357FF02C04D5F5F4F559547955595AD
:10ADD000479580912501909126012091000133270C
:10ADE000489FF001499FF00D589FF00D1124CF01AD
:10ADF000B9010E9496727093BB016093BA016634E8
:10AE000071051CF486E490E005C06739710534F0E3
:10AE100086E990E09093BB018093BA01809155033D
:10AE200090915603892B89F18091E1029091E20281
:10AE3000A091E302B091E4028093DD029093DE02E0
:10AE4000A093DF02B093E00220C08091E1029091D4
:10AE5000E202A091E302B091E40280599140A04047
:10AE6000B0408093DD029093DE02A093DF02B093A6
:10AE7000E0028091D806882311F0992702C088E764
:10AE800090E09093BB018093BA01C090B003D09042
:10AE9000B1032090E1023090E2024090E302509032
:10AEA000E4022091DD023091DE024091DF025091F8
:10AEB000E002221533054405550524F08091220750
:10AEC00080FDE9C1D201C101821B930BA40BB50B1C
:10AED00080937B0390937C03A0937D03B0937E03C8
:10AEE0008130F3E89F07FFEFAF07FFEFBF072CF4B8
:10AEF00080E093E8AFEFBFEF09C080509D47A040CE
:10AF0000B04064F080E09DE7A0E0B0E080937B0378
:10AF100090937C03A0937D03B0937E0300917B0309
:10AF200010917C03809190019927089F9001099FBF
:10AF3000300D189F300D1124C90137FD0F9624E004
:10AF4000959587952A95E1F7C81AD90A2091130299
:10AF50003091140237FF02C0295F3F4FB3E03595AF
:10AF60002795BA95E1F72930310514F028E030E053
:10AF7000229FA001239F500D329F500D11241216C5
:10AF8000130674F4CA0157FD039695958795959518
:10AF900087952091130230911402280F391F0DC09C
:10AFA000CA0157FD039695958795959587952091AC
:10AFB000130230911402281B390B809192019927BA
:10AFC000AA27BB27442737FD4095542FBC01CD014C
:10AFD0000E94577297FF04C061587F4F8F4F9F4F59
:10AFE000E7E09595879577956795EA95D1F79B0169
:10AFF0004FEF623874071CF421E83FEF05C06F3F44
:10B00000710514F02FEF30E0C21AD30A2090030329
:10B0100030900403409005035090060357FE08C08B
:10B020006FE770E080E090E0260E371E481E591E44
:10B0300057E055944794379427945A95D1F78091C7
:10B040008F01282F332744275527C201B1010E94C1
:10B05000577297FF04C0615E7F4F8F4F9F4F45E04F
:10B0600095958795779567954A95D1F79B017FEFE1
:10B07000223837071CF421E83FEF05C02F3F310588
:10B0800014F02FEF30E0C21AD30A0B561F4F0B52A9
:10B090001140E0F48091AC039091AD03892BB1F4A1
:10B0A0008091B0039091B103181619067CF4809139
:10B0B000B2039091B3038C159D053CF48091BC01C3
:10B0C0009091BD01C816D9060CF06C018091550312
:10B0D00090915603892B21F0C090B003D090B1031A
:10B0E00080918D019927AA27BB272091FF0733273D
:10B0F00027FD3095432F532FBC01CD010E9457727D
:10B1000097FF04C061587F4F8F4F9F4F37E0959551
:10B110008795779567953A95D1F79B019FEF2238F0
:10B1200039071CF421E83FEF05C02F3F310514F02B
:10B130002FEF30E0C21AD30AC601AA2797FDA095C7
:10B14000BA2F2DE0880F991FAA1FBB1F2A95D1F790
:10B150009701442737FD4095542FBC01CD010E9433
:10B16000CB7220937F0330938003409381035093ED
:10B170008203C0907F03D09080038091AE039091B2
:10B18000AF039C01220F331F280F391F2C0D3D1DCB
:10B1900037FF02C02D5F3F4FA90155954795559543
:10B1A00047955093AF034093AE038091D006282F6C
:10B1B0003327220F331F220F331F241735076CF458
:10B1C00080918207282F3327220F331F220F331F2E
:10B1D000205530404217530724F03093AF0320939B
:10B1E000AE038091220780FF0DC08091AE03909145
:10B1F000AF03A981BA81A817B90724F4B093AF03AC
:10B20000A093AE03E091AE03F091AF03FA83E9831C
:10B2100042C08091D806882301F56091B0037091F7
:10B22000B10377FF02C06D5F7F4F75956795759588
:10B230006795409125015091260180910001282FAA
:10B240003327649FC001659F900D749F900D11245A
:10B25000B9010E949672CB0101C099279093BB015E
:10B260008093BA018091BA019091BB018634910517
:10B270001CF486E490E005C08739910534F086E936
:10B2800090E09093BB018093BA0109811A811093D9
:10B29000AF030093AE038091BE0281FF2EC1809167
:10B2A000BE0284FD2AC18091B4039091B503A091A0
:10B2B000B603B091B7030097A105B105B1F4298198
:10B2C0003A81C901AA2797FDA095BA2FECE0880F13
:10B2D000991FAA1FBB1FEA95D1F78093B4039093DF
:10B2E000B503A093B603B093B70380911302909176
:10B2F0001402809113029091140297FF03C090955D
:10B3000081959F4F843691050CF0F7C049815A8191
:10B31000CA01AA2797FDA095BA2F9701442737FDA8
:10B320004095542FBC01CD010E945772DC01CB0126
:10B3300080937F0390938003A0938103B093820353
:10B34000B7FF04C08150904EAF4FBF4F7C018D01BD
:10B350007DE015950795F794E7947A95D1F7E092FB
:10B360007F03F09280030093810310938203809106
:10B37000BF029091C00257E0803D9507F8F480919C
:10B38000B4039091B503A091B603B091B7039C01AB
:10B39000AD0169E056954795379527956A95D1F7A0
:10B3A000821B930BA40BB50BA801970113E0220F8E
:10B3B000331F441F551F1A95D1F722C06FE0803A02
:10B3C000960758F58091B4039091B503A091B60308
:10B3D000B091B7039C01AD01FAE0569547953795BA
:10B3E0002795FA95D1F7821B930BA40BB50BA801F7
:10B3F0009701E2E0220F331F441F551FEA95D1F752
:10B40000820F931FA41FB51F8093B4039093B503BD
:10B41000A093B603B093B7033CC02091B40330911E
:10B42000B5034091B6035091B70380549F41C0F4D7
:10B43000DA01C9017BE0B695A795979587957A952E
:10B44000D1F7281B390B4A0B5B0BD801C7018E0DB6
:10B450009F1DA01FB11F280F391F4A1F5B1F11C05E
:10B46000DA01C9016CE0B695A795979587956A951D
:10B47000D1F7281B390B4A0B5B0B2E0D3F1D401FCC
:10B48000511F2093B4033093B5034093B6035093F8
:10B49000B7038091B4039091B503A091B603B09126
:10B4A000B7035CE0B695A795979587955A95D1F720
:10B4B0009093B1038093B0034091D606442399F052
:10B4C00055279C01BA010E949672C901861B970BF1
:10B4D0009093B3038093B203260F371F3093BD01BF
:10B4E0002093BC010AC01092B3031092B2038FEFF5
:10B4F00093E09093BD018093BC0130904507232DCC
:10B500003327C901880F991F880F991F8896A98131
:10B51000BA818A179B0714F09A8389834090820727
:10B52000842D9927880F991F880F991F8055904067
:10B53000E981FA818E179F0714F49A838983809199
:10B5400047028823A1F08091BF029091C002029728
:10B55000C09768F4E980FA801E141F0444F481E067
:10B5600090E09093C0028093BF023A8329830981BF
:10B570001A811093E2050093E10580917703909181
:10B580007803A0917903B0917A0312E0880F991F94
:10B59000AA1FBB1F1A95D1F700918307109184074A
:10B5A000081B190B29813A81213A31058CF0C90118
:10B5B00037FD019695958795801791070CF48C01BE
:10B5C000909581959F4F081719076CF48C010BC05B
:10B5D0000135110514F000E510E03FEF003B1307C3
:10B5E00014F400EB1FEF242D3327220F331F220FFB
:10B5F000331FC90149815A81841B950B801791071C
:10B600000CF48C0169817A81621B730B0617170792
:10B610000CF48B0180914007909141076091EC02FE
:10B620007091ED02861B970B909351078093500702
:10B63000D090610720916F033091700340917103A6
:10B6400050917203DD2041F0861A970AC401AA279F
:10B6500097FDA095BA2F04C0AA2797FDA095BA2FF1
:10B66000280F391F4A1F5B1F20936F03309370030D
:10B67000409371035093720380916F039091700314
:10B68000A0917103B091720381509A4FA040B040D5
:10B6900064F080E09AEFA0E0B0E080936F039093B5
:10B6A0007003A0937103B093720380916F03909124
:10B6B0007003A0917103B091720380509640AF4F18
:10B6C000BF4F64F480E096E0AFEFBFEF80936F036D
:10B6D00090937003A0937103B093720380909301D1
:10B6E000909094019401442737FD4095542F809108
:10B6F0006F0390917003A0917103B0917203BC012C
:10B70000CD010E94CB72E0905007F0905107E20EFD
:10B71000F31EB0907F016B2D77278827992798011A
:10B7200017FF04C022273327201B310B37FF02C02D
:10B730002F5F3F4F3595279549815A81240F351F3B
:10B74000442737FD4095542F0E94577297FF04C03D
:10B75000615C7F4F8F4F9F4F56E09595879577950A
:10B7600067955A95D1F79B016E157F050CF47B0107
:10B77000309521953F4FE216F3060CF47901809144
:10B780003107909132076091EA027091EB02861BBB
:10B79000970B9093300780932F072091730330917C
:10B7A00074034091750350917603DD2041F0661AD1
:10B7B000770AC301AA2797FDA095BA2F04C0AA272C
:10B7C00097FDA095BA2F280F391F4A1F5B1F2093A2
:10B7D0007303309374034093750350937603809101
:10B7E000730390917403A0917503B0917603815017
:10B7F0009A4FA040B04064F080E09AEFA0E0B0E043
:10B800008093730390937403A0937503B0937603AE
:10B810008091730390917403A0917503B0917603A6
:10B8200080509640AF4FBF4F64F480E096E0AFEF9A
:10B83000BFEF8093730390937403A0937503B09349
:10B8400076039401442737FD4095542F809173036C
:10B8500090917403A0917503B0917603BC01CD0162
:10B860000E94CB72C0902F07D0903007C20ED31E1B
:10B870006B2D772788279927980117FF04C0222767
:10B880003327201B310B37FF02C02F5F3F4F359509
:10B890002795A981BA812A0F3B1F442737FD409580
:10B8A000542F0E94577297FF04C0615C7F4F8F4FE7
:10B8B0009F4F26E095958795779567952A95D1F7BF
:10B8C0009B016C157D050CF46B01309521953F4F64
:10B8D000C216D3060CF4690183E2682E86E0782E46
:10B8E000B1E0AB2EB4E0BB2EABE05A2EF2E68F2EC9
:10B8F000F7E09F2EF501258512160CF0ABC04981AB
:10B900005A81CA01AA2797FDA095BA2F332727FD90
:10B910003095432F532FBC01CD010E94577297FFE2
:10B9200004C0615C7F4F8F4F9F4FE6E095958795F0
:10B9300077956795EA95D1F77C8B6B8BC701AA2722
:10B9400097FDA095BA2FF5012685332727FD309561
:10B95000432F532FBC01CD010E94577297FF04C0A3
:10B96000615C7F4F8F4F9F4F56E0959587957795F8
:10B9700067955A95D1F72B893C89260F371F3C8B49
:10B980002B8BC601AA2797FDA095BA2FF501278515
:10B99000332727FD3095432F532FBC01CD010E9443
:10B9A000577297FF04C0615C7F4F8F4F9F4F46E0F7
:10B9B00095958795779567954A95D1F72B893C8919
:10B9C000260F371F3C8B2B8BC801AA2797FDA0950C
:10B9D000BA2FF5012089332727FD3095432F532FA8
:10B9E000BC01CD010E945772DC01CB01B7FF03C03F
:10B9F000CF96A11DB11D36E0B595A7959795879572
:10BA00003A95D1F7F401608171812B893C89820FCD
:10BA1000931F0E946C32D4018D939C9397FD0396E3
:10BA200095958795959587959C8B8B8B832D9927DD
:10BA3000EB89FC89E817F9073CF0842D99272B89BD
:10BA40003C898217930714F49C8B8B8BEB89D30171
:10BA5000EC9302C0D3011C925A94E2E0F0E08E0E07
:10BA60009F1E24E030E0A20EB31E620E731E57FE2E
:10BA700041CFE2E1CC5E0C9402738091C7039091B8
:10BA8000C803A091C903B091CA038093BF039093E8
:10BA9000C003A093C103B093C2038091C3039091EC
:10BAA000C403A091C503B091C6038093BB039093D8
:10BAB000BC03A093BD03B093BE0308951092D203BC
:10BAC0001092D1031092D0031092CF03089584B145
:10BAD000806A84B93D9A82E58CBD1DBC459A81E09F
:10BAE000809394078AEA8093A40783E88093A5074C
:10BAF0008AE08093A6071092A8071092A7071092D9
:10BB0000AA071092A9071092FE071092C60708957F
:10BB1000EF92FF920F931F938091DE069927880F73
:10BB2000991F880F991F7C010027F7FC0095102FA3
:10BB300080913B0390913C03A0913D03B0913E0363
:10BB4000BC01CD01A80197010E94CB723093A807D8
:10BB50002093A7078091330390913403A09135037C
:10BB6000B0913603BC01CD01A80197010E94CB72B0
:10BB70003093AA072093A90720918A0730918B0759
:10BB800040918C0750918D07DA01C901E3E0880FDD
:10BB9000991FAA1FBB1FEA95D1F7820F931FA41FFD
:10BBA000B51F820F931FA41FB51F209179013091FB
:10BBB0007A0140917B0150917C01BC01CD010E9432
:10BBC000CB723093B0072093AF07E0914503F0911B
:10BBD00046038091570790915807BF010E949672C3
:10BBE000CB019B01220F331F220F331F280F391F58
:10BBF000280F391F37FF02C02D5F3F4F359527951E
:10BC0000359527953093AC072093AB078091860735
:10BC100090918707BF010E9496729B01220F331FEC
:10BC2000220F331F260F371F260F371F37FF02C083
:10BC30002D5F3F4F35952795359527953093AE0766
:10BC40002093AD07109246031092450310925807B7
:10BC50001092570710928707109286078091A607C7
:10BC600099278D30910509F466C08E3091055CF4FA
:10BC70008B30910509F48EC08C3091050CF00FC10A
:10BC80000A9761F08EC18F30910509F462C18F303F
:10BC900091050CF44EC1409799F183C18091D20275
:10BCA0008093B7078091D1028093B8078091D0022A
:10BCB0008093B9078091CF028093BA078091CE021A
:10BCC0008093BB078091CD028093BC078091CC020A
:10BCD0008093BD078091CB028093BE078091BE0206
:10BCE0008093BF078091BE02837F8093BE02F99943
:10BCF000FECF82E090E092BD81BDF89A80B54FC141
:10BD000080910008909101089093B8078093B7073D
:10BD100080910408909105089093BA078093B90721
:10BD200080912501909126018093BB0780910001AD
:10BD30008093BC0736C180910F078093B70780912D
:10BD400010078093B807809111078093B9078091FD
:10BD500012078093BA07809113078093BB078091E5
:10BD600017078093BC07809118078093BD078091C7
:10BD700019078093BE0780911C078093BF078091AD
:10BD80001A078093C00780911B078093C107809199
:10BD90001D07CCC0F8948091C506E82FFF27EE0F51
:10BDA000FF1FEC5AF94F0190F081E02DE038F105CA
:10BDB0001CF0EFE7F0E006C02FEFE138F20714F4D3
:10BDC000E1E8FFEFE093B7078091C606E82FFF2771
:10BDD000EE0FFF1FEC5AF94F0190F081E02DE03893
:10BDE000F1051CF0EFE7F0E006C06FEFE138F60771
:10BDF00014F4E1E8FFEFE093B8078091C406E82F60
:10BE0000FF27EE0FFF1FEC5AF94F0190F081E02D54
:10BE1000E038F1051CF0EFE7F0E006C08FEFE13805
:10BE2000F80714F4E1E8FFEFE093B9078091C30647
:10BE3000E82FFF27EE0FFF1FEC5AF94F0190F0811A
:10BE4000E02DE038F1051CF0EFE7F0E006C02FEF41
:10BE5000E138F20714F4E1E8FFEF7894E093BA07D1
:10BE60008091F0028093BB078091F1028093BC0720
:10BE70008091F2028093BD078091F3028093BE0708
:10BE80008091F4028093BF078091F5028093C007F0
:10BE90008091F6028093C1078091F70247C080919C
:10BEA0008004863018F01092800485E08093B707F4
:10BEB00080911E078093B8078091DD059091DE0583
:10BEC0009093BA078093B9078091DD029091DE02CA
:10BED000A091DF02B091E002BC01CD0125E030E08D
:10BEE00040E050E00E94CB723093BC072093BB0728
:10BEF000809114078093BD07809115078093BE073A
:10BF0000809116078093BF078091EF028093C0074E
:10BF10008091EE028093C1078091E1059091E20546
:10BF200097FD039695958795959587958093C2077C
:10BF300038C01092B7078EE48093B80783E08093EF
:10BF4000B9078CE08093BA07809102018093BB0708
:10BF500028C08091F6068093B707809121078093CF
:10BF6000B807809185018093B9078091EF0680938F
:10BF7000BA078091F0068093BB078091F106809309
:10BF8000BC07809184018093BD078091F306809364
:10BF9000BE078091F4068093BF078091F5068093D9
:10BFA000C0078091C607882309F4B0C08AEF809348
:10BFB000D4034091C8075091C907CA0181509E4FD0
:10BFC0008F5F9340B0F42091CA073091CB07C9012D
:10BFD00081509E4F8F5F934060F48091CF0685FF24
:10BFE00008C05093D2034093D1033093D0032093E1
:10BFF000CF038091CE079091CF0721E08936920739
:10C0000024F49093020380930103809101039091A3
:10C0100002032091FF0230910003821B930B845E88
:10C020009D4F68E671E00E949672845B9040909309
:10C03000FE028093FD022091D2073091D3078091B8
:10C04000FE019091FF018217930740F480918004D4
:10C05000882321F43093FF012093FE018091C707CC
:10C0600099278836910501F18936910524F48736A0
:10C07000910529F053C08936910559F14FC080913F
:10C08000D4078093FB078091D5078093FD078091AB
:10C09000D6078093FC078091D7078093FE07809195
:10C0A000D8078093FF073AC08091D40780939E07FA
:10C0B0008091D50780939F078091D6078093A00732
:10C0C0008091D7078093A1078091D8078093A2071A
:10C0D00025C08091D407809395078091D5078093E0
:10C0E00096078091D607809397078091D807909103
:10C0F000D90790939907809398078091DA079091D8
:10C10000DB0790939B0780939A0708C01092D20395
:10C110001092D1031092D0031092CF031F910F9170
:10C12000FF90EF90089580919407882309F43BC015
:10C13000459884EA97E090939D0780939C0790919F
:10C14000D303E92FFF27E154FE4F9F5F9093D30362
:10C1500080818093A607993010F01092D30310923B
:10C1600094070E94885D81E08093A307000000008F
:10C1700000000000000000000000000000000000BF
:10C1800000000000000000000000000000000000AF
:10C190000000000000000000000000008091A407E3
:10C1A0008093C3078EBD089530919407332309F01F
:10C1B00085C00DB407FE82C084E08093FD01459ADE
:10C1C0002EB58091D50399278130910589F0823071
:10C1D00091051CF4892B21F03EC00297B9F03BC0B9
:10C1E0003093C5072093D6032138A9F581E008C014
:10C1F000253549F48091D603820F8093D60382E0DF
:10C200008093D50328C03093D50325C08091C507FE
:10C21000E82FFF27EF51F84F20838F5F8093C507EA
:10C220009091D6038A31A0F0291769F48AE1A1EE32
:10C23000B7E0E7ECF7E00D9001928A95E1F781E035
:10C240008093C60702C03093C6071092D50303C07F
:10C25000920F9093D6032091A307203208F028C0B4
:10C2600045980000000000000000000000000000F1
:10C2700000000000000000000000000000000000BE
:10C2800000000000000000000000000000000000AE
:10C290000000E0919C07F0919D07E20FF11D808165
:10C2A0008EBD8091C3079081890F8093C30703C01F
:10C2B00081E0809394072F5F2093A307089587B1AF
:10C2C0008C6087B9429843981092D80380E8809395
:10C2D000C9011092D7038093C80108958091DD03AE
:10C2E00081508093DD038F3F09F0F4C094E0909378
:10C2F000DD038091BE02807BE1F080910D078823F1
:10C3000049F08091E003882311F49093D80381E0F1
:10C310008093E00380910E078823B9F08091E103B8
:10C32000882319F484E08093D70381E08093E103AC
:10C330000CC08093E0038093E10380910907809310
:10C34000DE0380910B078093DF038091E003882355
:10C3500009F040C080912007282F332724FF07C011
:10C360008091E502882319F425FD4DC04EC09091BF
:10C370000A07983F50F0809159078D3D30F0809129
:10C38000DE0388230CF43FC040C0983F48F0809102
:10C3900059078A3028F48091DE038823B4F133C032
:10C3A0008091D80381508093D8038F3F79F5809195
:10C3B000590781508093D8038091C901813011F4CD
:10C3C00080E801C086958093C9018091C901909150
:10C3D000DE0317C08091D80381508093D8038F3F2C
:10C3E000A9F489E08093D8038091C901813011F4C8
:10C3F00080E801C086958093C9018091C901909120
:10C400000D07892311F0429A01C042988091E103FF
:10C41000882309F043C080912007282F332724FF69
:10C4200007C08091E502882319F426FD50C034C06E
:10C4300090910C07983F50F0809181078D3D30F02E
:10C440008091DF0388230CF442C026C0983F48F057
:10C45000809181078A3028F48091DF038823E4F0FB
:10C4600036C08091D70381508093D7038F3F91F5D9
:10C470008091810781508093D7038091C8018130DA
:10C4800011F480E801C086958093C8018091C801AD
:10C490009091DF038923D9F4439808958091D703BD
:10C4A00081508093D7038F3FA9F489E08093D7030D
:10C4B0008091C801813011F480E801C08695809395
:10C4C000C8018091C80190910E07892311F0439A09
:10C4D0000895439808954FB724E130E0F89480918F
:10C4E000C9008F778093C9008091C9008F7B8093AA
:10C4F000C9008091C9008F7D8093C9005A9A5298D3
:10C500005B9A539A832F99278093CD002093CC0078
:10C510008091C80082608093C80080E18093C90048
:10C520008091CA008F778093CA008091CA008F7B68
:10C530008093CA008091CA008F7D8093CA00809149
:10C54000CA008F7E8093CA008091CA00877F809343
:10C55000CA008091C9008B7F8093C9008091CA0076
:10C5600084608093CA008091CA0082608093CA0070
:10C570008091C80087FF03C08091CE00F9CF8091E1
:10C58000C90080688093C9004FBF0895FF920F9340
:10C590001F93CF93DF9380E197E20E94E117EC01B4
:10C5A000FF248091C9008F778093C9008091C900D2
:10C5B0008F7E8093C9005A9881ED99E09F938F9365
:10C5C0000FE014E11F930F93E091FF03F09100043B
:10C5D00009950F900F900F900F9002C04A996CC070
:10C5E000CE010E94EA178823C9F3E091FF03F0917E
:10C5F0000004FF2009F468C087E09AE09F938F93BE
:10C600001F930F930995529A0F900F900F900F90D0
:10C61000CE010E94EA178823D9F383E690E05A9A64
:10C62000019797FFFCCF8FE891E05A98019797FF09
:10C63000FCCF89E090E05A9A019797FFFCCF89E000
:10C6400090E05A98019797FFFCCF8FE891E05A9AB3
:10C65000019797FFFCCF8FE891E05A98019797FFD9
:10C66000FCCF89E090E05A9A019797FFFCCF89E0D0
:10C6700090E05A98019797FFFCCF8FE891E05A9A83
:10C68000019797FFFCCF8FE891E05A98019797FFA9
:10C69000FCCF89E090E05A9A019797FFFCCF89E0A0
:10C6A00090E05A98019797FFFCCF8FE891E05A9A53
:10C6B000019797FFFCCF13C08AE590E00E94E11735
:10C6C000EC0191E0F92E91CF8DE09AE09F938F934A
:10C6D0001F930F9309950F900F900F900F90529802
:10C6E0005A980E946B62E5E0CDB7DEB70C940F73E9
:10C6F000EF92FF920F931F93CF93DF93482F00E0A9
:10C7000010E08091CA01813061F41092CA0184E482
:10C710008093E2031092E4031092E3031092E50386
:10C720002BC18091E203882319F421E030E001C09D
:10C7300098019091E303992371F4232B11F081E088
:10C7400010C084E48093E2039093E4039093E303A6
:10C750009093E503FAC0913069F4232B09F0EBC004
:10C7600082E08093E3038091E4038F5F8093E4038E
:10C7700083E0E9C09230D1F4232B09F0DCC083E0E0
:10C780008093E2034093E5039091E403923039F4FF
:10C790001092E60347FF03C081E08093E60383E045
:10C7A0008093E3039F5F9093E403CFC0933009F03D
:10C7B000C2C0232B09F0BFC09093E20382E08093B4
:10C7C000E3038091E4038F5F8093E4032091E5030A
:10C7D000822F9927782F6627842F9927682B792B0A
:10C7E0008091E806813049F47370CB01805092400B
:10C7F00063E070E00E94967217C0823061F4777037
:10C80000CB018050944066E070E00E9496722695BD
:10C81000269526950BC0737068567140CB0177FD45
:10C820000196BC017595679526952695022F1127CF
:10C830000F7010700F5F1F4F0D30110508F074C09E
:10C840007801E00EF11EF701EC5AF94F80819181D9
:10C850009B01281B390BC90137FF03C090958195B7
:10C860009F4F069794F48091EF02883C30F48091BA
:10C87000EF02865F8093EF0208C088EC8093EF029E
:10C8800080916F008F7D80936F00F701EC5AF94F14
:10C89000808191819C01220F331F280F391F260FA1
:10C8A000371F37FF02C02D5F3F4FE901D595C79570
:10C8B000D595C795CB0101968C179D0714F4219748
:10C8C00006C061507040C617D7070CF421968091BE
:10C8D000EF02843BD0F0F701EC5AF94F808191814F
:10C8E000FE01E81BF90BCF0163E070E00E94967235
:10C8F000CB01880F991F860F971F28E836E0E20EBC
:10C90000F31EF7019183808307C028E836E0E20E2A
:10C91000F31EF70111821082000F111F0C5A194FDC
:10C92000F801D183C08311C00231110570F081E09C
:10C930008093CA010AC081E08093CA011092E40387
:10C940001092E60384E48093E2038091E403803153
:10C9500098F08091E603882331F48091CA018823FE
:10C9600011F4809378011092E4031092E603109280
:10C97000E30384E48093E203E6E0CDB7DEB70C94F2
:10C980000E73CF93FC0197FF05C0CFEFF095E195B3
:10C99000FF4F01C0C1E028E631E0CF01B9010E949C
:10C9A0009672FC018B35910554F08B5590408A3579
:10C9B000910538F484EB90E08E1B9F0BFC0141E065
:10C9C0000DC0CF01855B90408A35910518F4E45B7A
:10C9D000F04003C02E1B3F0BF9014FEFEE0FFF1F7E
:10C9E000E85EF54F259134918C2F992787FD90951E
:10C9F000289FB001299F700D389F700D1124842F3E
:10CA0000992787FD9095689FA001699F500D789F99
:10CA1000500D1124CA01CF9108952AE530E0281B5A
:10CA2000390BC9010E94C1640895CF93DF9380E060
:10CA30000E94796880912501909126016AE070E05A
:10CA40000E9496729F938F93809125019091260169
:10CA50006AE070E00E9496727F936F9386EE9AE090
:10CA60009F938F93CCE6D8E6DF93CF93E091FF03BB
:10CA7000F091000409952DB73EB7285F3F4F2DBFB9
:10CA80008091D403882339F187E00E9479688FED83
:10CA900090E09F938F9380919A0790919B079F932B
:10CAA0008F9380919807909199076AE070E00E94B7
:10CAB00082727F936F938FEE9AE09F938F93DF93B1
:10CAC000CF93E091FF03F091000409958DB79EB7D5
:10CAD0000A968DBF12C087E00E9479688CEF9AE0B9
:10CAE0009F938F93DF93CF93E091FF03F091000426
:10CAF00009950F900F900F900F9080E10E94796838
:10CB00008091D0019091D1016CE370E00E9482721B
:10CB10009F938F938091D0019091D1016CE370E04D
:10CB20000E9482727F936F93809104089091050810
:10CB30009F938F9383E09BE09F938F93DF93CF939B
:10CB4000E091FF03F091000409958091CF062DB785
:10CB50003EB7265F3F4F2DBF80FF24C08BE10E9470
:10CB600079688091E1029091E202A091E302B09194
:10CB7000E402BC01CD0124E630E040E050E00E9438
:10CB8000CB723F932F9381E19BE09F938F93DF9331
:10CB9000CF93E091FF03F091000409958DB79EB704
:10CBA00006968DBFDF91CF910895CF93DF9380E0FC
:10CBB0000E94796886E19BE09F938F93CCE6D8E64C
:10CBC000DF93CF93E091FF03F0910004099580E19A
:10CBD0000E9479680F900F900F900F9080918A07B4
:10CBE00090918B07A0918C07B0918D0720917901CE
:10CBF00030917A0140917B0150917C01BC01CD01C3
:10CC00000E94CB723F932F93809133039091340312
:10CC1000A0913503B0913603B7FF04C081509C4FFB
:10CC2000AF4FBF4F3AE0B595A795979587953A9541
:10CC3000D1F79F938F9380913B0390913C03A091F8
:10CC40003D03B0913E03B7FF04C081509C4FAF4FEE
:10CC5000BF4F2AE0B595A795979587952A95D1F767
:10CC60009F938F9385E29BE09F938F93DF93CF9366
:10CC7000E091FF03F091000409958DB79EB70A96E5
:10CC80008DBFDF91CF9108950F931F9380E00E9495
:10CC900079682AE030E08091000890910108B9019C
:10CCA0000E9482729F938F93809100089091010857
:10CCB000B9010E9482727F936F93809125019091B8
:10CCC0002601B9010E9496729F938F93809125014E
:10CCD00090912601B9010E9496727F936F9381E330
:10CCE0009BE09F938F930CE618E61F930F93E091C0
:10CCF000FF03F0910004099580E10E9479688DB7E7
:10CD00009EB70C968DBF80910408909105089F9363
:10CD10008F9380910208909103089F938F9384E4EE
:10CD20009BE09F938F931F930F93E091FF03F091EC
:10CD3000000409958DB79EB708968DBF1F910F917E
:10CD400008950F931F93CF93DF938091D403CCE684
:10CD5000D8E6882309F490C080E00E947968809129
:10CD6000960799279F938F9380E59BE09F938F93DE
:10CD70008E01DF93CF93E091FF03F09100040995BA
:10CD80008DB79EB706968DBF809197079927823001
:10CD9000910579F0833091051CF4892B21F019C09D
:10CDA000039789F016C087E00E94796889E59BE0C7
:10CDB00005C087E00E9479688FE59BE09F938F9381
:10CDC000DF93CF930FC087E00E94796885E69BE0F0
:10CDD000F5CF87E00E9479688BE69BE09F938F9365
:10CDE0001F930F93E091FF03F091000409950F90BA
:10CDF0000F900F900F908091950781FF14C089E0EC
:10CE00000E94796881E79BE09F938F938CE698E678
:10CE10009F938F93E091FF03F091000409950F9089
:10CE20000F900F900F9080E10E9479688FED90E055
:10CE30009F938F9380919A0790919B079F938F93D5
:10CE400080919807909199076AE070E00E94827241
:10CE50007F936F9387E79BE09F938F938CE698E691
:10CE60009F938F93E091FF03F091000409958DB794
:10CE70009EB70A968DBF12C082E00E94796889E849
:10CE80009BE09F938F93DF93CF93E091FF03F0910B
:10CE9000000409950F900F900F900F90DF91CF91A4
:10CEA0001F910F910895CF93C82F2091E7032093EE
:10CEB000E80399278F329105E1F0803391051CF446
:10CEC0004F9779F027C08F349105D9F08F389105AD
:10CED00009F586E0289FF0011124E253F54F849173
:10CEE00017C086E0289FF0011124E153F54F84918B
:10CEF0000FC086E0289FF0011124E053F54F849184
:10CF000007C086E0289FF0011124EF52F54F84916D
:10CF10008093E7039091E7038091E8039813C0E0C2
:10CF20000E947F689091E70386E0989FF0011124AA
:10CF3000EE52F54F259134918C2FF9010995CF913F
:10CF4000089510920108109200081092050810929E
:10CF5000040810920308109202088AE090E00E94F0
:10CF6000E1179093EA038093E9030895CF93DF9349
:10CF70008091E9039091EA030E94EA17882309F45B
:10CF8000A8C08091E9039091EA030A969093EA037E
:10CF90008093E903E0E0F0E09F0190E0A3E2B6E0D7
:10CFA0004BE0ED01898187FF07C09F5F8A81E80F11
:10CFB000F11D8C91280F311D4150149647FFF1CF80
:10CFC000232B41F52091EF033091F0034091F103C1
:10CFD0005091F203BB27A52F942F832F9093EE033C
:10CFE0008093ED03AA27BB27281B390B4A0B5B0B49
:10CFF000CF01AA27BB27280F391F4A1F5B1F209389
:10D00000EF033093F0034093F1035093F203E5E014
:10D01000F0E013C02091ED033091EE032E173F078F
:10D0200018F4E21BF30B02C0E0E0F0E0892F99272F
:10D03000880F991FE80FF91F3596F0930108E093C8
:10D040000008EF3FF10578F48091250190912601C9
:10D050008E9F90018F9F300D9E9F300D1124C9012E
:10D0600064E670E013C0CF019695879596958795F5
:10D070002091250130912601289FA001299F500D64
:10D08000389F500D1124CA0169E170E00E9482723C
:10D0900070930308609302082091EB033091EC0336
:10D0A0002E0F3F1F3093EC032093EB035EE0213102
:10D0B000350778F0809104089091050801969093C7
:10D0C00005088093040820513E403093EC032093E0
:10D0D000EB03DF91CF9108959091F403933240F4E4
:10D0E000E92FFF27EA5FF74F80839F5F9093F40358
:10D0F0000895833218F48D5F8093F403089590E2CD
:10D10000E9E0F8E08FE19193815087FFFCCF08952B
:10D11000CF93CFB723E031E0F8948091C9008F77A7
:10D120008093C9008091C9008F7B8093C900809152
:10D13000C9008F7D8093C9005A9A52985B9A539A7E
:10D14000832F99278093CD002093CC008091C80035
:10D1500082608093C80088E18093C9008091CA00F2
:10D160008F778093CA008091CA008F7B8093CA001A
:10D170008091CA0080628093CA008091CA00806159
:10D180008093CA008091CA0088608093CA00809111
:10D19000C90084608093C9008091CA008460809334
:10D1A000CA008091CA0082608093CA008091C80042
:10D1B00087FF03C08091CE00F9CF8091C9008068BD
:10D1C0008093C9008091C90080648093C9000E9447
:10D1D0007F68CFBFCF910895282F99278F709070C7
:10D1E000892B31F420958091F303822B8093F303F4
:10D1F00008958091CB01882309F43FC08091BE023D
:10D2000085FF0AC082E98093060883E280930708BD
:10D2100085E58093080802C0109206088091F30308
:10D22000882321F480910608882339F18091CC016C
:10D230008F3021F48091F3030E9453671092CB0149
:10D240008091C80085FFFCCF8091C9008F7E8093BC
:10D25000C9008091C9008E7F8093C9008091060823
:10D26000882311F48EEF01C08EE78093CE00809169
:10D27000F3038093CC011092F30308951F920F9251
:10D280000FB60F9211248F939F93EF93FF9390917A
:10D29000CB019923E1F58091F503882341F4809136
:10D2A0000608882399F483E08093F5030FC0833048
:10D2B00099F480910608882349F09093060880919C
:10D2C000C9008E7F8093C9008EEF1EC08091C90077
:10D2D00081608093C9000EC0833261F48091C900DF
:10D2E0008E7F8093C9008FEF8093CE0081E0809382
:10D2F000CB0114C08091F503E82FFF27EA5FF74FB9
:10D300008F5F8093F50380818093CE0007C01092D9
:10D31000F5038091C90080618093C900FF91EF916E
:10D320009F918F910F900FBE0F901F9018952FB760
:10D3300040E0F894E0E0F0E081E2809357009491BF
:10D34000E2E0F0E0809357003491E4E0F0E0809375
:10D35000570084912FBF9E3199F4363941F48930BA
:10D3600011F441E00DC08A3059F442E009C0373968
:10D3700039F4863011F443E003C0853009F444E009
:10D38000842F992708959FB7F8948091C900877FCB
:10D390008093C9008091C9008F7E8093C9008091DD
:10D3A000C9008F778093C9008091C9008F7B8093DB
:10D3B000C9008091C9008F7D8093C90052985A9A04
:10D3C00053985B9A9FBF0895CF93DF938091F703A3
:10D3D000882309F497C09091E8068091CE019817B0
:10D3E00009F490C08091F603882321F40E94976984
:10D3F0008093F60382E89CE09F938F93CFE0D4E183
:10D40000DF93CF93E091FF03F091000409950F9013
:10D410000F900F900F908091E80699278230910528
:10D4200001F1833091052CF4009761F0019769F0C8
:10D4300024C084309105D9F084309105ACF0059773
:10D44000C9F01BC082E79CE002C080E69CE09F938D
:10D450008F93DF93CF93E091FF03F0910004099540
:10D4600019C087E49CE0F3CF84E29CE0F0CF86E132
:10D470009CE0EDCF8EE09CE0EACF8FE89CE09F93AC
:10D480008F93DF93CF93E091FF03F0910004099510
:10D490001092E8060F900F900F900F908091F60376
:10D4A000843011F08230A9F40E94C3699091E8069B
:10D4B000892F8150833018F40E946B621FC0943012
:10D4C00019F40E9488681AC09530C1F40E948B6BD1
:10D4D00015C08091E806882389F085EA9CE09F9337
:10D4E0008F938FE094E19F938F93E091FF03F091EE
:10D4F000000409950F900F900F900F908091E8060F
:10D500008093CE01DF91CF9108950F931F9381E017
:10D510008093F7034091CD01EEEBFBE020E030E09B
:10D520005FE4849199272F5F3F4F829FB001839FD3
:10D53000700D929F700D112446275150319657FF60
:10D54000F0CF4093CD01E6E9FBE020E030E057E288
:10D55000849199272F5F3F4F829FB001839F700D69
:10D56000929F700D112446275150319657FFF0CFEE
:10D570004093CD018091F603882321F40E9497699E
:10D580008093F6038091CD01833459F088E190E0D7
:10D5900029E20FB6F894A895809360000FBE2093FF
:10D5A000600089E89DE6909300048093FF0380EC7F
:10D5B0009CE09F938F930FE014E11F930F93E091F2
:10D5C000FF03F091000409950F900F900F900F90BA
:10D5D00084E690E09F938F938EE490E09F938F93E7
:10D5E0001F921F92809102016AE00E947672892F39
:10D5F00099279F938F93809102010E9476729927B9
:10D600009F938F9386EE9CE09F938F931F930F932E
:10D61000E091FF03F091000409958EEB9BE09F934E
:10D620008F931F930F93E091FF03F09100040995EE
:10D6300086E99BE09F938F931F930F93E091FF03E5
:10D64000F091000409958DB79EB746968DBF8AE18B
:10D650009DE09F938F931F930F93E091FF03F091B1
:10D660000004099583EC8093810080916F008062B3
:10D6700080936F000F900F900F900F901F910F915C
:10D6800008958091F703882361F08091E806843043
:10D6900011F40E94F9688091CD01833411F0109249
:10D6A000F70308951F920F920FB60F9211242F9334
:10D6B0003F934F935F936F937F938F939F93AF931A
:10D6C000BF93EF93FF932091CE009091E806892FAE
:10D6D0008150833020F4822F0E9478630BC09430F5
:10D6E00021F4822F0E94EC6805C0953019F4822F36
:10D6F0000E94F76CFF91EF91BF91AF919F918F9135
:10D700007F916F915F914F913F912F910F900FBE3D
:10D710000F901F9018954FB720E430E0F894809157
:10D72000C9008F778093C9008091C9008F7B809357
:10D73000C9008091C9008F7D8093C9005A9A529880
:10D740005B9A539A832F99278093CD002093CC0026
:10D750008091C80082608093C80088E18093C900EE
:10D760008091CA008F778093CA008091CA008F7B16
:10D770008093CA008091CA008F7D8093CA008091F7
:10D78000CA008F7E8093CA008091CA00877F8093F1
:10D79000CA008091C9008B7F8093C9008091CA0024
:10D7A00084608093CA008091CA0082608093CA001E
:10D7B0008091C80087FF03C08091CE00F9CF80918F
:10D7C000C90080688093C9004FBF08950F931F93CD
:10D7D000CF93DF93482F4F5F893108F089C0809144
:10D7E0005306841710F440935306CB0183539B4296
:10D7F00068E170E00E949672A42FBB27FD01EA0F3A
:10D80000FB1FEC5AF94F808191819B01281B390B3A
:10D81000C90137FF03C0909581959F4F069794F4F7
:10D820008091EF02883C30F48091EF02865F809314
:10D83000EF0208C088EC8093EF0280916F008F7D2B
:10D8400080936F00FD01EA0FFB1FEC5AF94F8081B6
:10D8500091819C01220F331F280F391F260F371F7C
:10D8600037FF02C02D5F3F4FE901D595C795D5958C
:10D87000C795CB0101968C179D0714F4219706C01C
:10D8800061507040C617D7070CF421968091EF02C3
:10D89000843BD8F08D010A0F1B1FF801EC5AF94F99
:10D8A00080819181FE01E81BF90BCF0163E070E0FC
:10D8B0000E949672CB01880F991F860F971F0857F9
:10D8C000194FF8019183808307C0AA0FBB1FA85787
:10D8D000B94F11961C921E92E42FFF27EE0FFF1FE7
:10D8E000EC5AF94FD183C083443011F4109278017F
:10D8F000DF91CF911F910F910895CF93DF932091E6
:10D900002908822F9927807F9070409709F06CC07A
:10D910002F3109F046C080912A088093F8032091A6
:10D920002C082093FA0380912D088093F903822F0D
:10D9300099279093550680935406222309F054C0EA
:10D940008091C306282F3327220F331FF901E85790
:10D95000F94F118210828091C406A82FBB27AA0F0D
:10D96000BB1FFD01E857F94F118210828091C60656
:10D97000E82FFF27EE0FFF1FCF018857994FEC01CB
:10D98000198218822C5A394FE90119821882AC5A2F
:10D99000B94F11961C921E92EC5AF94F11821082C7
:10D9A00023C0C22FCF70CA30F8F480912A08809328
:10D9B000300880912B0880932F0880912C08809349
:10D9C000320880912D088093310860912F08709162
:10D9D00030088C2F0E94E66B6091310870913208FC
:10D9E0008C2F8F5F0E94E66BDF91CF910895CF93CC
:10D9F000C82F8F3F49F48091FB038F3F29F4109289
:10DA0000FD031092FC0332C02091FD03222339F460
:10DA1000CF3111F485E001C084E08093FE03809152
:10DA2000FE039091FC038217A0F4892F80958093C8
:10DA3000FC038F3F19F48EEF8093FC038091FC036D
:10DA4000C81711F40E947D6C1092FD031092FC0324
:10DA50000BC0E22FFF27E75DF74FC0832F5F2093B6
:10DA6000FD039C0F9093FC03C093FB03CF9108959B
:10DA7000EF92FF920F931F93CF93DF937C018B0163
:10DA8000EA01452B39F0F80181918F01F7010995E1
:10DA90002197C9F7E6E0CDB7DEB70C940E73EF928D
:10DAA000FF920F931F93CF93DF937C018B01EA01C9
:10DAB000452B41F0F8010F5F1F4F8491F701099545
:10DAC0002197C1F7E6E0CDB7DEB70C940E730F9344
:10DAD0001F93CF938C01C62F161634F480E2F80101
:10DAE0000995C1501C16D4F3CF911F910F91089541
:10DAF0000F931F93CF938C01C62F161634F480E337
:10DB0000F8010995C1501C16D4F3CF911F910F91C4
:10DB10000895A5E3B0E0EFE8FDE60C94E6722E96DA
:10DB2000EEADFFAD2E978824992454018091F70320
:10DB3000882321F42C961FAE1EAE2C975EE4452E52
:10DB4000512C4C0E5D1E6F01B60105C0153239F027
:10DB50000894C11CD11CF60114911123B9F7A60138
:10DB6000461B570B31F02C968EAD9FAD2C970E9423
:10DB70004F6D112309F46AC20894C11CD11CFF2403
:10DB8000FDA6FCA64FEFE42EF9A6F6010894C11CF1
:10DB9000D11C1491153721F0812F80628837B1F4A0
:10DBA000F0FE0AC0F20124E030E0420E531E8080F5
:10DBB0009180A280B3800AC0F20142E050E0440E9E
:10DBC000551E808191814C01AA24BB24103221F47E
:10DBD00089A58823D1F61DC0133219F458E0F52A1F
:10DBE000D4CF1A3211F01D3291F41A3259F4F201E5
:10DBF00082E090E0480E591EE081ECA7EE232CF65F
:10DC0000E195ECA790E1F92AAFEDFA22BECF1B32E5
:10DC100011F419A7BACF1E32C1F5F6010894C11C40
:10DC2000D11C14911A3279F4F20122E030E0420E54
:10DC3000531E408151813FEF4F3F530714F44FEF84
:10DC40005FEFE42EA2CF40E050E0812F80538A3076
:10DC5000A0F4CA0133E0880F991F3A95E1F7840FC9
:10DC6000951F480F591F410F511D40535040F60159
:10DC70000894C11CD11C1491E8CF8FEF4F3F580777
:10DC800014F44FEF5FEFE42E85CF103329F4F4FC4A
:10DC90007CCF90E2F92A79CF812F81538930D8F453
:10DCA00040E050E0CA0123E0880F991F2A95E1F770
:10DCB000840F951F480F591F410F511D405350406D
:10DCC000F6010894C11CD11C1491812F80538A3015
:10DCD00048F34CA75FCF183619F4A4E0FA2A55CFC1
:10DCE0001C3619F4B1E0FB2A50CF133661F43E0123
:10DCF0000894611C711CF20122E030E0420E531EB8
:10DD0000808189833CC1143421F0143611F0193616
:10DD100051F5143411F431E0F32AF0FE0AC0F20197
:10DD200044E050E0440E551E80809180A280B38074
:10DD30000CC0F20182E090E0480E591E8081918172
:10DD40004C01AA2497FCA094BA2CB7FE0AC0B09448
:10DD5000A09490948094811C911CA11CB11C8DE214
:10DD600089A70AE06FC01F3411F01F3631F41F3449
:10DD700011F491E0F92A08E064C0103779F4F20157
:10DD8000A2E0B0E04A0E5B1E808191814C01AA2482
:10DD9000BB2400E1B0E4FB2A18E753C01337C1F5F8
:10DDA000F20122E030E0420E531E60807180611467
:10DDB000710489F43E010894611C711C88E2898316
:10DDC0008EE6F301818385E78B838CE68C838D83DC
:10DDD00089E28E831F82E7FC13C08E2D992787FD71
:10DDE0009095AC0160E070E0C3010E94B3700097B1
:10DDF00029F0382E3618E3140CF0C3C03E2CC1C0F5
:10DE0000F30101900020E9F731973E2E3618B9C092
:10DE1000153511F0153731F4153511F4F1E0FF2AFD
:10DE20000AE00FC0183519F0183709F0A0C000E15A
:10DE3000F3FE07C081149104A104B10411F020E4A1
:10DE4000F22A19A6EDA6E7FC02C03FEDF32299E203
:10DE5000692E712C6C0E7D1E81149104A104B104F5
:10DE600021F44DA5442309F47BC0802F9927AA27CC
:10DE7000BB278EA79FA7A8ABB9AB202E332490E079
:10DE8000891690E0990691E0A90690E0B90648F05D
:10DE9000C501B4012EA53FA548A959A90E94A972A0
:10DEA00017C0AFEF8A169104A104B10449F040F005
:10DEB000C401B1010E9482729B014427552708C00A
:10DEC000882D602F0E947672282F332744275527EC
:10DED0002AAB3BAB4CAB5DAB0A3059F48AA9880F37
:10DEE000880F880F9AA9990F890F382D381B832F17
:10DEF00010C0003139F48AA98295807F482D481BD3
:10DF0000842F07C08AA9880F880F880F582D581BA7
:10DF1000852F90E02EA53FA548A959A98216930602
:10DF2000A406B50608F091E08AA89BA8ACA8BDA8F5
:10DF30008A3010F4805D04C0895A183509F48F7D49
:10DF4000D3018E933D01992309F099CF083041F414
:10DF5000F3FE06C0803321F080E3FD0182933F0190
:10DF6000CE010196382E3618F8E23F0E0BC0112371
:10DF700009F46CC03E010894611C711C198381E096
:10DF8000382E19A6032D2DA4231827FC222489A599
:10DF9000882311F00F5F02C0F6FC0E5F020DEF2C1C
:10DFA000FF24C70180739070892B49F48CA5801BD6
:10DFB000682F2C968EAD9FAD2C970E94676D89A51A
:10DFC000882331F041E050E0BE01675D7F4F0AC019
:10DFD000E6FE0EC080E38AA71BA742E050E0BE0128
:10DFE000665D7F4F2C968EAD9FAD2C970E94386D4D
:10DFF000C70180739070809749F48CA5801B682FAF
:10E000002C968EAD9FAD2C970E94786D622D2C962C
:10E010008EAD9FAD2C970E94786D832D992787FD3B
:10E020009095AC01B3012C968EAD9FAD2C970E94BC
:10E03000386DE4FE89CD2CA5201B2CA7622F2C96D1
:10E040008EAD9FAD2C970E94676D7ECDE2E1CB5CDB
:10E050000C940273002422273327442751E0BB2766
:10E06000EE27FF27A0E1660F771F881F991F001C6E
:10E07000221F331F441F660F771F881F991F001C24
:10E08000221F331F441F2AF4050E2B1F3E1F4F1F54
:10E0900004C0051A2B0B3E0B4F0B550FBB1FEE1F79
:10E0A000587F556047FD5250AA95E9F6E695B79519
:10E0B0005795E695B7955795852F9B2F089522275D
:10E0C000332741E0552768E0880F991F221F331F2F
:10E0D000880F991F221F331F1AF4240F351F02C007
:10E0E000241B350B440F551F487F456037FD4250B8
:10E0F0006A9551F75695479556954795842F0895FB
:10E10000AA2797FF04C0809590958A1F9A1F77FFD2
:10E1100004C0609570956A1F7A1F669F9001779F73
:10E12000A001679F300D411D5A1F300D411D5A1F20
:10E13000889FF001999F2E0F3F1F401D511D899F01
:10E14000300D411D5A1F300D411D5A1FCA01B90122
:10E15000112480CFFB01DC0102C005900D924150DB
:10E160005040D8F70895FC014150504030F00190E4
:10E170000616D1F73197CF0108958827992708957A
:10E18000A0E0B0E0E6ECF0E70C94EE726C017B01ED
:10E19000EA01590121978FEFCF3FD80789F0860117
:10E1A0000894C11CD11CC7010894E11CF11CF501A5
:10E1B0000995F80180832197FFEFCF3FDF0779F7BB
:10E1C000EAE0CDB7DEB70C940A73A0E0B0E0EBEE66
:10E1D000F0E70C94F0728C017B01EA016901219750
:10E1E0008FEFCF3FD80771F0F70121917F01C80170
:10E1F0000F5F1F4F622FF60109952197FFEFCF3F69
:10E20000DF0791F7E8E0CDB7DEB70C940C735058F8
:10E21000BB27AA270ED00DC1FED030F003D120F0CD
:10E2200031F49F3F11F41EF4F3C00EF4E095E7FBC8
:10E23000E9C0E92F0FD180F3BA176207730784078B
:10E24000950718F071F49EF527C10EF4E0950B2E9A
:10E25000BA2FA02D0B01B90190010C01CA01A00138
:10E260001124FF27591B99F0593F50F4503E68F193
:10E270001A16F040A22F232F342F4427585FF3CFD4
:10E28000469537952795A795F0405395C9F77EF4A5
:10E290001F16BA0B620B730B840BBAF09150A1F0EE
:10E2A000FF0FBB1F661F771F881FC2F70EC0BA0F74
:10E2B000621F731F841F48F4879577956795B795FC
:10E2C000F7959E3F08F0B3CF9395880F08F09927F4
:10E2D000EE0F97958795089571D008F481E0089521
:10E2E00004D06894B111D9C00895BCD088F09F576C
:10E2F00090F0B92F9927B751A0F0D1F0660F771F92
:10E30000881F991F1AF0BA95C9F712C0B13081F071
:10E31000C3D0B1E00895C0C0672F782F8827B85FB9
:10E3200039F0B93FCCF3869577956795B395D9F7D2
:10E330003EF490958095709561957F4F8F4F9F4FDC
:10E340000895E89409C097FB3EF4909580957095E8
:10E3500061957F4F8F4F9F4F9923A9F0F92F96E931
:10E36000BB279395F695879577956795B795F111A6
:10E37000F8CFFAF4BB0F11F460FF1BC06F5F7F4F43
:10E380008F4F9F4F16C0882311F096E911C0772355
:10E3900021F09EE8872F762F05C0662371F096E85E
:10E3A000862F70E060E02AF09A95660F771F881F2D
:10E3B000DAF7880F9695879597F90895990F0008D1
:10E3C000550FAA0BE0E8FEEF16161706E807F90747
:10E3D000C0F012161306E407F50798F0621B730BE2
:10E3E000840B950B39F40A2661F0232B242B252B63
:10E3F00021F408950A2609F4A140A6958FEF811D06
:10E40000811D089597F99F6780E870E060E00895A6
:10E410009FEF80EC089500240A941616170618063C
:10E420000906089500240A94121613061406050618
:10E430000895092E0394000C11F4882352F0BB0FA9
:10E4400040F4BF2B11F460FF04C06F5F7F4F8F4F0C
:10E450009F4F089557FD9058440F551F59F05F3F47
:10E4600071F04795880F97FB991F61F09F3F79F0F6
:10E4700087950895121613061406551FF2CF469578
:10E48000F1DF08C0161617061806991FF1CF8695FA
:10E490007105610508940895E894BB2766277727DE
:10E4A000CB0197F908958ADF08F48FEF0895629FF2
:10E4B000D001739FF001829FE00DF11D649FE00D7C
:10E4C000F11D929FF00D839FF00D749FF00D659FDD
:10E4D000F00D9927729FB00DE11DF91F639FB00DDC
:10E4E000E11DF91FBD01CF0111240895991B79E0A9
:10E4F00004C0991F961708F0961B881F7A95C9F7D4
:10E5000080950895AA1BBB1B51E107C0AA1FBB1F22
:10E51000A617B70710F0A61BB70B881F991F5A95AF
:10E52000A9F780959095BC01CD01089597FB092E20
:10E5300007260AD077FD04D0E5DF06D000201AF4C4
:10E54000709561957F4F0895F6F7909581959F4F4F
:10E550000895A1E21A2EAA1BBB1BFD010DC0AA1F24
:10E56000BB1FEE1FFF1FA217B307E407F50720F03C
:10E57000A21BB30BE40BF50B661F771F881F991FB7
:10E580001A9469F760957095809590959B01AC0100
:10E59000BD01CF01089597FB092E05260ED057FD2A
:10E5A00004D0D7DF0AD0001C38F450954095309540
:10E5B00021953F4F4F4F5F4F0895F6F79095809507
:10E5C000709561957F4F8F4F9F4F08952F923F9287
:10E5D0004F925F926F927F928F929F92AF92BF9273
:10E5E000CF92DF92EF92FF920F931F93CF93DF931F
:10E5F000CDB7DEB7CA1BDB0B0FB6F894DEBF0FBE7C
:10E60000CDBF09942A88398848885F846E847D84C8
:10E610008C849B84AA84B984C884DF80EE80FD80CA
:10E620000C811B81AA81B981CE0FD11D0FB6F89440
:10E63000DEBF0FBECDBFED010895EE0FFF1F0590A9
:08E64000F491E02D0994FFCFD5
:10E648005E010A0151756164726F00000164FF0187
:10E65800FFFF01FC01FC0101737373FF03007D00E0
:10E6680000C409C40964001048616C6C6F205765C8
:10E678006C740000000000000000000000000000B2
:10E688000000000000000000000000000000000082
:10E698000000000000000000000000000000000072
:10E6A8000000000000000000000000000000000062
:10E6B8000000000000000000010B050000ECFF64F2
:10E6C80040415A4664640A02969696960840403A33
:10E6D80010FB30380190D0030090D00300F401649F
:10E6E8000053706F727400004E6F726D616C0000A1
:10E6F800426567696E6E657200007800FF03640BFF
:10E708000A0D0B0C0E0B0F10010101010F70FF0019
:00000001FF
